:100000000C948B050C94B3050C94B3050C94B305B8
:100010000C94B3050C94B3050C94B3050C94B30580
:100020000C9405090C94B3050C94B3050C94B3051A
:100030000C94B3050C94B3050C94B3050C94B30560
:100040000C94B3050C94B3050C9462630C94B30543
:100050000C9463640C94AA640C94B3050C94B305DB
:100060000C94B3050C94B3050C944B600C94B3053D
:100070006376006A630064700063700063720075E9
:1000800070006A7000636F006A6F007370006A73BB
:1000900000636D006373006A6E006A6C00646C003C
:1000A000737500637500776561746865722E6F7093
:1000B000656E737072696E6B6C65722E636F6D0026
:1000C0002F776561746865720024442E70793F6CE7
:1000D0006F633D2445266B65793D2445266677761A
:1000E0003D244400485454502F312E3020323030BB
:1000F000204F4B0D0A43616368652D436F6E747228
:100100006F6C3A206D61782D6167653D363034380B
:1001100030302C207075626C69630D0A0D0A002462
:100120004600485454502F312E3020323030204F6A
:100130004B0D0A436F6E74656E742D547970653A79
:1001400020746578742F68746D6C0D0A5072616745
:100150006D613A206E6F2D63616368650D0A4163BE
:10016000636573732D436F6E74726F6C2D416C6C8D
:100170006F772D4F726967696E3A202A0D0A0D0A52
:10018000003C7363726970743E77696E646F772E9A
:100190006C6F636174696F6E3D222F223B3C2F733D
:1001A00063726970743E0A00485454502F312E30E7
:1001B00020323030204F4B0D0A436F6E74656E74E1
:1001C0002D547970653A206170706C69636174694F
:1001D0006F6E2F6A736F6E0D0A436F6E6E6E65637E
:1001E00074696F6E3A20636C6F73650D0A416363C7
:1001F0006573732D436F6E74726F6C2D416C6C6FF1
:10020000772D4F726967696E3A202A0D0A43616340
:1002100068652D436F6E74726F6C3A206E6F2D633C
:10022000616368650D0A0D0A0024467B22726573BE
:10023000756C74223A24447D0024467B22726573D7
:10024000756C74223A24447D0024462446002224FE
:1002500046223A24447D005D002C245300245300A0
:1002600024465B005D2C226E73746174696F6E733B
:10027000223A24447D002C0024440022736E223A4A
:100280005B0024465265626F6F74696E672E2E2E76
:10029000002C2264657870223A24442C226D657803
:1002A00070223A24447D002C00222446223A244421
:1002B00000222446223A244C0024467B003C6D65F3
:1002C0007461206E616D653D2276696577706F722D
:1002D000742220636F6E74656E743D227769647456
:1002E000683D6465766963652D77696474682C6917
:1002F0006E697469616C2D7363616C653D312E307C
:100300002C6D696E696D756D2D7363616C653D3122
:100310002E302C757365722D7363616C61626C6530
:100320003D6E6F223E0D0A003C736372697074204B
:100330007372633D2224452F686F6D652E6A7322A8
:100340003E3C2F7363726970743E0A3C2F626F6487
:10035000793E0A3C2F68746D6C3E0076617220769F
:1003600065723D24442C697061733D24443B3C2FED
:100370007363726970743E0A0024463C21444F4303
:10038000545950452068746D6C3E0A3C68746D6C1D
:100390003E0A3C686561643E0A24463C2F686561FC
:1003A000643E0A3C626F64793E0A3C736372697012
:1003B000743E005B302C305D5D2C226C72756E22B9
:1003C0003A5B24442C24442C24442C244C5D7D0092
:1003D0005B24442C244C2C244C5D2C00305D2C22BE
:1003E0007073223A5B0024442C00226465767422E8
:1003F0003A244C2C226E627264223A24442C2265E8
:100400006E223A24442C227264223A24442C227212
:1004100073223A24442C2272647374223A244C2CA2
:10042000226C6F63223A222445222C2277746B655A
:1004300079223A222445222C2273756E72697365E3
:10044000223A24442C2273756E736574223A244434
:100450002C227362697473223A5B005D7D00225D19
:1004600000225D2C00245300244C5D2C2200244CDF
:100470002C0024445D2C5B0024442C005B24442C81
:1004800024442C24442C5B00226E70726F6773220C
:100490003A24442C226E626F61726473223A2444BF
:1004A0002C226D6E70223A24442C226D6E737422BD
:1004B0003A24442C22706E73697A65223A24442CC3
:1004C000227064223A5B003C6872202F3E3C666FCB
:1004D000726D206E616D653D6F6620616374696F3A
:1004E0006E3D6375206D6574686F643D6765743E2D
:1004F0003C703E3C623E5363726970742055524CAE
:100500003A3C2F623E3C696E707574207479706558
:100510003D746578742073697A653D3332206D616E
:10052000786C656E6774683D3132372076616C7522
:10053000653D22244522206E616D653D6A73703EE3
:100540003C2F703E3C703E44656661756C7420695A
:10055000732024533C6272202F3E4966206C6F63E7
:10056000616C206F6E2075534420636172642C208F
:10057000757365202E2F3C2F703E3C703E3C623ED2
:1005800050617373776F72643A3C2F623E3C696EC0
:1005900070757420747970653D70617373776F72D4
:1005A000642073697A653D3332206E616D653D70FC
:1005B000773E3C696E70757420747970653D737513
:1005C000626D69743E3C2F703E3C6872202F3E3C49
:1005D0002F666F726D3E002446005D2C226D61789F
:1005E0006C656E223A24447D0073746E5F64697397
:1005F000006163745F72656C61790069676E6F7228
:10060000655F7261696E006D61736F70002C00220E
:100610002453220022736E616D6573223A5B002CB5
:10062000002444005D2C222446223A5B004E5450A4
:100630002053796E63696E672E2E2E0044657465B3
:100640006374696E67207553442E2E2E00302E2061
:1006500054657374202831206D696E29002E2000A6
:100660002000486F6C6420423320746F20737461E3
:10067000727400436C69636B20423320746F206C8A
:100680006973740052756E20612050726F677261D9
:100690006D3A0000010800060400014500008200D8
:1006A0000040002000504F5354202446204854540A
:1006B000502F312E300D0A486F73743A2024460DA6
:1006C0000A244624534163636570743A202A2F2A12
:1006D0000D0A436F6E74656E742D4C656E67746899
:1006E0003A2024440D0A436F6E74656E742D54795C
:1006F00070653A206170706C69636174696F6E2F08
:10070000782D7777772D666F726D2D75726C656EAB
:10071000636F6465640D0A0D0A2453004745542035
:100720002446245320485454502F312E300D0A486B
:100730006F73743A2024460D0A24460D0A0D0A00F0
:100740004163636570743A20746578742F68746DC2
:100750006C00E30004FA00010000000166777600F7
:10076000747A006E747000646863700069703100A0
:100770006970320069703300697034006777310046
:10078000677732006777330067773400687030002E
:100790006870310061720065787400736571007370
:1007A0006474006D6173006D746F6E006D746F66BC
:1007B000007572730072736F00776C0064656E0071
:1007C0006970617300646576696400636F6E006CC4
:1007D00069740064696D00726C7000757774006EE6
:1007E000747031006E747032006E747033006E7409
:1007F0007034007265736574004669726D7761725A
:1008000065207665722E00545A6F6E653A004E541C
:10081000503F0055736520444843503F0053746176
:100820007469632E6970313A005374617469632E80
:100830006970323A005374617469632E6970333A97
:10084000005374617469632E6970343A00476174AF
:10085000657761792E6970313A0047617465776117
:10086000792E6970323A00476174657761792E6933
:1008700070333A00476174657761792E6970343A54
:10088000004854545020706F72743A0000417574DF
:100890006F207265636F6E6E6563743F004578709C
:1008A0002E20626F6172643A0053657175656E74D3
:1008B00069616C3F0053746E2064656C61793A0025
:1008C0004D61732E2073746174696F6E3A004D61CF
:1008D000732E20206F6E2061646A2E3A004D617382
:1008E0002E206F66662061646A2E3A005261696E3E
:1008F0002073656E736F723A004E6F726D616C6C2F
:1009000079206F70656E3F002520576174657220F5
:1009100074696D653A0044657669636520656E614A
:10092000626C653F0049676E2070617373776F7208
:10093000643F004465762E2049443A004C434420ED
:10094000636F6E74726173743A004C434420626149
:10095000636B6C696768743A004C43442064696D4A
:100960006D696E673A0052656C61792070756C73C1
:10097000653A0055736520776561746865723F005C
:100980004E54502E6970313A004E54502E697032D8
:100990003A004E54502E6970333A004E54502E692E
:1009A00070343A00526573657420616C6C3F004D81
:1009B0006F6E005475650057656400546875004695
:1009C0007269005361740053756E00206D730020CE
:1009D00073656300207365630025004E6F005965E1
:1009E00073002B002B0020474D54003030003A009C
:1009F0002D002B000020202020002D44697361620F
:100A00006C6564212D003A0045004D433A003A00E0
:100A10002E002D0020002020003A002000486F6C9E
:100A20006420423320746F20736176650042312F59
:100A300042323A2B2F2D2C2042333A2D3E003D3DA1
:100A4000536574204F7074696F6E733D3D00506C38
:100A50006561736520576169742E2E2E005265738F
:100A6000657474696E672044657669636500436FD9
:100A70006E6E656374696E672E2E2E007C3C3E5E42
:100A80002B3D3F2F5B5D3B2C2A225C0000002100A8
:100A9000240027002A0000002200250028002B0047
:100AA00000002000230026002900020202020202A8
:100AB0000202040404040404040403030303030300
:100AC00003030101010101010101010204081020D9
:100AD0004080010204081020408001020408102018
:100AE0004080804020100804020100000001020044
:100AF00000000000000004030706000000000000E2
:100B000000000000000000000000A709BE2D263AEA
:100B1000FB4DE75E8A6511241FBECFEFD0E1DEBF3B
:100B2000CDBF13E0A0E0B1E0EEEDF2ED02C0059024
:100B30000D92A43EB107D9F71EE0A4EEB3E001C0C8
:100B40001D92A63AB107E1F71BE0C6E1DBE004C065
:100B50002297FE010E943269CA30D107C9F70E946C
:100B6000FA660C946D690C940000CF93DF93BC017E
:100B70008230910510F462E070E0A091A40EB09173
:100B8000A50EED0140E050E0E0E0F0E021C08881FA
:100B900099818617970769F48A819B81309719F0AC
:100BA0009383828304C09093A50E8093A40EFE01CC
:100BB00034C06817790738F44115510519F08417C6
:100BC000950708F4AC01FE018A819B819C01E90133
:100BD0002097E9F641155105A9F1CA01861B970B2B
:100BE000049708F4BA01E0E0F0E02AC08D919C91EE
:100BF000119784179507F9F46417750781F4129615
:100C00008D919C911397309719F09383828304C040
:100C10009093A50E8093A40EFD0132964CC0CA019C
:100C2000861B970BFD01E80FF91F619371930297E3
:100C30008D939C9340C0FD01828193819C01D901D9
:100C40001097A1F68091A20E9091A30E892B41F4EA
:100C50008091F2019091F3019093A30E8093A20EE4
:100C60004091F4015091F5014115510541F44DB702
:100C70005EB78091F0019091F101481B590B2091D2
:100C8000A20E3091A30ECA01821B930B8617970701
:100C900080F0AB014E5F5F4F8417950750F0420F15
:100CA000531F5093A30E4093A20EF90161937193C9
:100CB00002C0E0E0F0E0CF01DF91CF910895CF9343
:100CC000DF93009709F450C0EC0122971B821A822F
:100CD000A091A40EB091A50E109709F140E050E04C
:100CE000AC17BD0708F1BB83AA83FE0121913191A6
:100CF000E20FF31FAE17BF0779F48D919C91119706
:100D0000280F391F2E5F3F4F3983288312968D910C
:100D10009C9113979B838A834115510571F4D0935D
:100D2000A50EC093A40E20C012968D919C9113978E
:100D3000AD01009711F0DC01D3CFFA01D383C28358
:100D400021913191E20FF31FCE17DF0769F48881FB
:100D50009981280F391F2E5F3F4FFA01318320837D
:100D60008A819B8193838283DF91CF910895A0E054
:100D7000B0E0EDEBF6E00C9438696C01009729F4D3
:100D8000CB010E94B5056C01C1C08EEF882E8FEF9C
:100D9000982E8C0C9D1C8601060F171F081519052F
:100DA00008F4B2C0F401A081B181A617B707B8F06A
:100DB000A530B10508F4AAC0CD010497861797079E
:100DC00008F4A4C01297A61BB70BF801A193B19326
:100DD000D4016D937C93CF010E945F0697C07B0185
:100DE000EA1AFB0AEEEFFFEFEE0EFF1E36016A0E67
:100DF0007B1EC091A40ED091A50EAA24BB2444242E
:100E000055244AC0C615D705E1F5488159814E15CC
:100E10005F05B8F1CA0104978E159F05B0F41296CC
:100E2000A40FB51FF401B183A0832A813B81411433
:100E3000510431F0D20113963C932E93129766C061
:100E40003093A50E2093A40E61C08A819B81F80186
:100E500093838283425050404E195F0951834083EF
:100E60004114510431F0D20113961C930E93129742
:100E700004C01093A50E0093A40EF4017183608347
:100E800045C088819981A816B90608F45C012E0135
:100E90008A819B819C01E901209709F0B3CF809161
:100EA000A20E9091A30E86159705E9F4A616B70633
:100EB000D0F42091F4013091F5012115310541F470
:100EC0002DB73EB78091F0019091F101281B390BAD
:100ED00002171307C8F41093A30E0093A20ED401B7
:100EE0006D937C9313C0CB010E94B505EC01009774
:100EF00059F0F40140815181B6010E94E707C60113
:100F00000E945F066E0102C0CC24DD24C601CDB76D
:100F1000DEB7E0E10C945469FC0188279927E89436
:100F200021912032E9F3293010F02E30C8F32B3212
:100F300041F02D3239F4689404C00E949408820F65
:100F4000911D219120532A30C0F31EF49095819574
:100F50009F4F08951F93FC0199278827BC01E894AF
:100F600011911032E9F3193010F01E30C8F31B3222
:100F700051F01D3249F4689406C00E947F08610F49
:100F8000711D811D911D119110531A30B0F33EF463
:100F900090958095709561957F4F8F4F9F4F1F91D2
:100FA0000895FB01DC0102C005900D9241505040B4
:100FB000D8F70895FB01DC0104C08D9101908019E0
:100FC00021F441505040C8F7881B990B0895FB014C
:100FD000DC0102C001900D9241505040D8F70895B5
:100FE000DC0101C06D9341505040E0F70895FC01D1
:100FF0008191861721F08823D9F799270895319791
:10100000CF010895FB01DC0101900D920020E1F772
:101010000895FB01DC014150504030F08D9101906A
:10102000801919F40020B9F7881B990B0895FB016A
:10103000DC014150504048F001900D920020C9F76A
:1010400001C01D9241505040E0F70895A0E0B0E08B
:10105000ECE2F8E00C9440697C01EB018A01690143
:1010600009C0CE012196F6010995F70181937F0110
:101070000150104001151105A1F7CDB7DEB7E8E02A
:101080000C945C69A0E0B0E0E8E4F8E00C944069FE
:10109000EC017B018A01690109C0CE012196F701AB
:1010A00061917F01F601099501501040011511056C
:1010B000A1F7CDB7DEB7E8E00C945C69FB019F01B6
:1010C000E8944230C4F04532B4F44A3029F497FB36
:1010D0001EF4909581959F4F642F77270E94CC68CE
:1010E000805D8A330CF0895D8193CB010097A1F775
:1010F00016F45DE251931082C9010C94D708592F60
:10110000482F372F262F660F771F881F991F660FCE
:10111000771F881F991F620F731F841F951F660F0B
:10112000771F881F991F08957AE0979F902D879FBA
:10113000802D910D11240895FA01CF93FF93EF9321
:101140002230CCF02532BCF4C22F2C2F3327442779
:101150005527FF93EF930E94F368EF91FF91605D35
:101160006A330CF0695D6193B901CA016050704047
:101170008040904051F710828F919F91CF910C94B5
:10118000D708FB019F01423074F0453264F4642FAC
:1011900077270E94CC68805D8A330CF0895D81934B
:1011A000CB010097A1F71082C9010C94D708DC018C
:1011B000FC01672F71917723E1F7329704C07C918E
:1011C0006D9370836291AE17BF07C8F308959C01B9
:1011D000F999FECF32BD21BDF89A80B508959C01E2
:1011E000F999FECF1FBA32BD21BD60BD0FB6F8948C
:1011F000FA9AF99A0FBE0895FC01A681B7816D9302
:10120000B783A68381E090E008951F920F920FB6F6
:101210000F9211242F933F934F935F936F937F937C
:101220008F939F93AF93BF93EF93FF938091230886
:101230008F5F8093230880912308803128F0E0910C
:101240002108F09122080995FF91EF91BF91AF918C
:101250009F918F917F916F915F914F913F912F91CE
:101260000F900FBE0F901F901895A5EAB9E080E08F
:1012700090E0FC01EB5DF74F108211821282138225
:10128000FC01EB51F74F10821182128213821D92E2
:101290000496803C910569F71092DD091092DE09F1
:1012A0001092DF091092E009F999FECF81E090E0F9
:1012B00092BD81BDF89A80B5809324080895982F37
:1012C00080912408981708F041C0992309F43EC082
:1012D000892F90E0019727E430E0AC01429FC001E4
:1012E000439F900D529F900D11249C012E5F3F4F04
:1012F000875B9F4F24C0F999FECF32BD21BDF89A7C
:1013000050B5F999FECF72BD61BDF89A40B5F99913
:10131000FECF1FBA32BD21BD40BD0FB6F894FA9A78
:10132000F99A0FBEF999FECF1FBA72BD61BD50BDCB
:101330000FB6F894FA9AF99A0FBE2F5F3F4FB90192
:10134000695B7F4F2817390709F0D5CF08951092B0
:10135000E4071092E30785E593E09093E20780931A
:10136000E10789E18093EA071092ED0710920008E7
:1013700010920708109209080895AF92BF92DF9269
:10138000EF92FF920F931F93CF93DF9300D000D083
:1013900001EE17E0ADB7BEB712961C930E931197EE
:1013A0008BE792E014969C938E9313970E94B2362B
:1013B000FF240F900F900F900F90D02EE12E98E702
:1013C000A92E92E0B92EC6E7D2E04FC00F2D10E053
:1013D00000D000D000D0ADB7BEB71196EDB7FEB7C4
:1013E000D182E2821396BC92AE921297F80183E00A
:1013F000F595E7958A95E1F7ED53F54F808190E0FB
:1014000098012770307002C0959587952A95E2F76C
:101410008170907015969C938E9314970E94B236AB
:101420008091C20A90E001972DB73EB72A5F3F4FE7
:101430000FB6F8943EBF0FBE2DBF08171907A1F0D5
:1014400000D000D0ADB7BEB71196DC9211971296BE
:10145000EC9212971496DC93CE9313970E94B236B7
:101460000F900F900F900F90F3942091C20AF216F4
:1014700008F4ACCF00D000D000D0EDB7FEB7319665
:1014800081EE97E0ADB7BEB712969C938E931197FD
:1014900084E692E093838283248315820E94B2368D
:1014A000EDB7FEB736960FB6F894FEBF0FBEEDBF90
:1014B000DF91CF911F910F91FF90EF90DF90BF9040
:1014C000AF90089500D000D000D0EDB7FEB73196B0
:1014D00081EE97E0ADB7BEB712969C938E931197AD
:1014E00089EB92E09383828388EA91E095838483F9
:1014F0000E94B2368DB79EB706960FB6F8949EBF7F
:101500000FBE8DBF08950E94620A0E94BD0980E04F
:1015100008950F931F9300D000D000D0EDB7FEB711
:10152000319601EE17E0ADB7BEB712961C930E933D
:10153000119787ED95E09383828382E291E0958312
:1015400084830E94B23600D0EDB7FEB73196ADB7B6
:10155000BEB712961C930E93119787EC94E0938379
:10156000828384E494E09583848380E091E0978390
:1015700086830E94B2368DB79EB708960FB6F89450
:101580009EBF0FBE8DBF80E01F910F9108958F9277
:101590009F92AF92BF92DF92EF92FF920F931F93B1
:1015A000CF93DF93EB0100D000D000D0EDB7FEB7B2
:1015B000319601EE17E0ADB7BEB712961C930E93AD
:1015C000119724E236E033832283958384830E943B
:1015D000B236FF24EDB7FEB736960FB6F894FEBFCD
:1015E0000FBEEDBFD02EE12E31E2832E36E0932EDA
:1015F0002FE1A22E26E0B22E40C000D000D000D0B5
:10160000ADB7BEB71196EDB7FEB7D182E2821396A1
:101610009C928E9212970F2D10E0FE01E00FF11FA9
:10162000808114968C93149715961C920E94B23662
:101630008091C10A90E001972DB73EB72A5F3F4FD6
:101640000FB6F8943EBF0FBE2DBF08171907A1F0C3
:1016500000D000D0ADB7BEB71196DC9211971296AC
:10166000EC9212971496BC92AE9213970E94B236E7
:101670000F900F900F900F90F3948091C10AF8167D
:1016800008F4BBCFDF91CF911F910F91FF90EF90A6
:10169000DF90BF90AF909F908F9008950F931F930E
:1016A000DF93CF93CDB7DEB728970FB6F894DEBFA0
:1016B0000FBECDBF8091950A882329F486EA90E079
:1016C00060E00E948E3708E617E01C821B8285E5E9
:1016D00093E09A8389831E830D8318870F838DB7C8
:1016E0009EB70C970FB6F8949EBF0FBE8DBFEDB797
:1016F000FEB73196CE010196ADB7BEB712969C9358
:101700008E93119789EC90E09383828380910103FB
:101710008483158284E194E09783868384E894E04F
:101720009187808780914702828713860E94B23614
:10173000D8010D900020E9F71197A01BB10BA00F65
:10174000B11F2FED37E0EDB7FEB73C960FB6F8941A
:10175000FEBF0FBEEDBF50E342E395E213C08C9194
:10176000B90161507040803249F4F9015083FB01A6
:10177000408392939F012150304003C0F901808340
:101780009B011197F7E0A836BF0749F78C91D90163
:101790008C938091BB0A8F778093BB0A80EC90E09A
:1017A000B90146EA50E02FE43CE00E948E2E2896D4
:1017B0000FB6F894DEBF0FBECDBFCF91DF911F9162
:1017C0000F910895AF92BF92CF92DF92EF92FF9266
:1017D0000F931F937B018C018091BC0A82958F70BF
:1017E00079F58091BB0A83FD2BC087FF03C084E895
:1017F00093E002C08AE090E02091F10A3091F20A71
:101800004091F30A5091F40A211531054105510523
:1018100069F057016801A21AB30AC40AD50AA0E008
:10182000B0E08A159B05AC05BD0550F4E092F10AC5
:10183000F092F20A0093F30A1093F40A0E944E0BFE
:101840001F910F91FF90EF90DF90CF90BF90AF90DE
:1018500008950F931F9368E677E048E72FE131E0A2
:1018600000E010E00E944135882311F480E114C0AB
:1018700088E697E00E948C079C01181619065CF414
:101880008091240890E0281739072CF4822F0E94B9
:101890005F0981E001C081E11F910F9108950F93CD
:1018A0001F93CF93DF93EB01CC51DC4F01C0219606
:1018B0008881882309F47CC08632C9F76BC088E62A
:1018C00097E00E948C079C0185E0213A380720F4BC
:1018D0003093B40A2093B30ACE0168E677E048E774
:1018E00023E231E000E010E00E944135882369F0F6
:1018F00088E697E00E948C079C0185E0213A380732
:1019000020F43093B60A2093B50A0E94FE3DCE0122
:1019100068E677E048E72AE231E000E010E00E9464
:101920004135882359F088E697E00E948C078B3F69
:10193000910520F48093D1020E94A739CE0168E678
:1019400077E048E720E331E000E010E00E94413515
:101950008823D1F088E697E00E948C079C018136AD
:10196000910590F480914D0290E02817390761F0BD
:1019700020934D021092ED0A1092EE0A1092EF0A97
:101980001092F00A0E94A7398091BB0A8068809368
:10199000BB0A0EC0CE0168E677E048E723E331E0FA
:1019A00000E010E00E944135882309F495CF87CFED
:1019B000DF91CF911F910F9108956F927F928F9237
:1019C0009F92BF92CF92DF92EF92FF920F931F935D
:1019D000DF93CF93CDB7DEB728970FB6F894DEBF6D
:1019E0000FBECDBF80910703898380910D038A8349
:1019F000809113038B83809119038C83BB243E0158
:101A00000894611C711C45E0842E912C8C0E9D1E47
:101A100060913E026F5F60933E02C3010E940F31EE
:101A20000E94B6636B017C0188EE93E0A0E0B0E019
:101A3000C80ED91EEA1EFB1E0E945E478C010E9442
:101A4000AD31012B09F441C0C40160913E020E94F6
:101A5000422E8823D1F1ED80FE800F81188580EC25
:101A600098EDA4E5BCE7E80EF91E0A1F1B1F609164
:101A70004D0270E080E090E024E833E040E050E088
:101A80000E94A168E60EF71E081F191F08C0B39434
:101A900094E1B91609F0BCCFEE24FF248701B70109
:101AA000C80128960FB6F894DEBF0FBECDBFCF9108
:101AB000DF911F910F91FF90EF90DF90CF90BF903B
:101AC0009F908F907F906F9008950E94B6636C15E1
:101AD0007D058E059F0508F4AFCFD9CF0F931F93D7
:101AE000DF93CF93CDB7DEB76E970FB6F894DEBF16
:101AF0000FBECDBF8C0189EE97E0B8010E940F495F
:101B0000882309F47AC0CE010196B80141E00E9411
:101B10009D5E00D000D000D0EDB7FEB7319681EECB
:101B200097E0ADB7BEB712969C938E9311978FE155
:101B300091E09383828384EE90E0958384830E9476
:101B4000B2368DB79EB706960FB6F8949EBF0FBEFD
:101B50008DBF8091E7079091E8072091E5073091CC
:101B6000E607821B930B60E140E00E94812F1092F8
:101B7000E4071092E3078AE194E09093E6078093EC
:101B8000E5079093E8078093E7078E010B5F1F4FEF
:101B900019C0C8016AE174E040E052E00E9491512E
:101BA0009C01442737FD4095542F203092E039079F
:101BB00090E0490790E05907B0F0C90160E143E0C7
:101BC0000E94812F2F89388D498D5A8D8F85988954
:101BD000A989BA89281739074A075B07D1F620E097
:101BE00030E040E050E0C90161E143E00E94812F14
:101BF000CE0105960E946B5181E06E960FB6F89467
:101C0000DEBF0FBECDBFCF91DF911F910F91089521
:101C1000CF93DF939C0110926807FC01A081B181F2
:101C2000C0E0D0E00FC09C919D3231F09B3221F09A
:101C3000892F80538A3068F4FE01E859F84F908369
:101C400021961196F901808191810A96A817B9070A
:101C500050F3C859D84F18821196F901B183A08367
:101C600088E697E00E94AA07CB01DF91CF91089503
:101C70006F927F928F929F92AF92BF92CF92DF929C
:101C8000FF920F931F93DF93CF9300D00F92CDB7A6
:101C9000DEB75C016A01DE011196EEE5F3E083E058
:101CA00001900D928150E1F76983FF2452E0652E87
:101CB000712C6C0E7D1E4E010894811C911C1BC062
:101CC0008F2D90E0B3014AE050E00E945E08C5010C
:101CD00068E677E048E7940100E010E00E944135B3
:101CE000882341F088E697E00E948C07F601EF0D0B
:101CF000F11D8083F3948091C10AF81608F30F90C8
:101D00000F900F90CF91DF911F910F91FF90DF9077
:101D1000CF90BF90AF909F908F907F906F900895DD
:101D20000F931F930E94AB2B8DB79EB708970FB6EA
:101D3000F8949EBF0FBE8DBFEDB7FEB7319601EE92
:101D400017E0ADB7BEB712961C930E93119789E7B3
:101D500093E09383828382E291E0958384838DEB89
:101D600092E0978386830E94B236EDB7FEB7319634
:101D7000ADB7BEB712961C930E9311978BE593E007
:101D80009383828382ED90E0958384838091DD024A
:101D9000868317820E94B2360F900F90EDB7FEB780
:101DA0003196ADB7BEB712961C930E93119788E289
:101DB00093E09383828384E494E0958384830E94F8
:101DC000B2368DB79EB706960FB6F8949EBF0FBE7B
:101DD0008DBF80E01F910F9108954F925F926F9297
:101DE0007F928F929F92AF92BF92CF92DF92EF92AB
:101DF000FF920F931F93DF93CF930F92CDB7DEB770
:101E00000E94AB2B5B016C012DB73EB72C513040CB
:101E10000FB6F8943EBF0FBE2DBFEDB7FEB731969B
:101E200001EE17E0ADB7BEB712961C930E93119753
:101E30008AEE93E093838283A482B582C682D7829E
:101E40008091C10A808711868091BB0A8170828748
:101E500013868091BB0A8695817084871586809150
:101E6000BB0A869586958170868717868091B70A0A
:101E70009091B80AA091B90AB091BA0A808B918B5F
:101E8000A28BB38B84E194E0958B848B84E894E0FF
:101E9000978B868B8091B30A9091B40A918F808F33
:101EA0008091B50A9091B60A938F828F0E94B236C4
:101EB00090E0EDB7FEB77C960FB6F894FEBF0FBE6C
:101EC000EDBF780106EE13E023C000D000D000D0B3
:101ED000EDB7FEB73196ADB7BEB71196EC9211973C
:101EE0001296FC9213830283A92FB0E0AD53B54F35
:101EF0008C918483158299830E94B23699819F5F69
:101F0000EDB7FEB736960FB6F894FEBF0FBEEDBF25
:101F10008091C10AF1EE6F2EF7E07F2E9817A8F29C
:101F200000D000D0ADB7BEB712967C926E921197DA
:101F30008CED93E014969C938E9313970E94B23687
:101F400099240F900F900F900F90C301762C892E3B
:101F5000E0ED4E2EE3E05E2E64C0A92DB0E0FD0161
:101F6000EB55F64F6081662329F420E030E040E035
:101F700050E025C0CD01880F991F880F991FFC01E3
:101F8000EB5DF74FE080F18002811381FC01EB51A2
:101F9000F74FAE14BF04C006D10648F0208131814E
:101FA000428153812A193B094C095D0908C02081EF
:101FB0003181428153812E193F09400B510BEDB7FE
:101FC000FEB73E970FB6F894FEBF0FBEEDBF0DB73C
:101FD0001EB70F5F1F4F71828282F80153824282C7
:101FE000648315822683378340875187AA0FBB1FDE
:101FF000AA0FBB1FAB5DB74F8D919D910D90BC910A
:10200000A02D82879387A487B5870E94B2369394C8
:102010002DB73EB7225F3F4F0FB6F8943EBF0FBEBD
:102020002DBF8091C20A981608F497CF8DB79EB73E
:102030000E970FB6F8949EBF0FBE8DBFEDB7FEB7DB
:10204000319681EE97E0ADB7BEB712969C938E9312
:10205000119783EB93E0938382838091D5098483E6
:1020600015828091D609868317828091D709909135
:10207000D809918780878091D9099091DA09A09138
:10208000DB09B091DC0982879387A487B5870E941A
:10209000B236EDB7FEB73E960FB6F894FEBF0FBE50
:1020A000EDBF0F90CF91DF911F910F91FF90EF90B7
:1020B000DF90CF90BF90AF909F908F907F906F9068
:1020C0005F904F9008950E94620A0E94ED0E80E09A
:1020D0000895BF92CF92DF92EF92FF920F931F93DA
:1020E0006C01FC01B080E1800E94AB2B20E831E55F
:1020F00041E050E00E94F3682B0D311D411D511D40
:10210000FF2400E010E0CA01B901A80197010E9474
:10211000F368F60160831F910F91FF90EF90DF90BD
:10212000CF90BF9008958F929F92AF92BF92CF921F
:10213000DF92EF92FF920F931F934C01FC01A1805D
:10214000E080FF24EA0CF11C0027F7FC0095102F1B
:102150000E94AB2BBB24CC24DD2420E831E541E0F8
:1021600050E00E94F368CA01B901A60195010E94DE
:10217000F368E61AF70A080B190BC801B701A601A4
:1021800095010E94F368F40160831F910F91FF9005
:10219000EF90DF90CF90BF90AF909F908F90089579
:1021A0000E94AB2BAB01BC018091C20AE5EAF9E0C9
:1021B000A5EEB8E0282F30E02E0F3F1F0AC0808127
:1021C000882329F04D935D936D937C9313973196FB
:1021D0001496E217F30799F70895EF92FF920F9381
:1021E0001F93DF93CF93CDB7DEB7C857D0400FB65C
:1021F000F894DEBF0FBECDBF7C0168E677E048E70C
:102200002BE331E000E010E00E944135882311F417
:1022100080E127C0C7017E010894E11CF11CB701D1
:1022200048E72FE331E000E010E00E9441358823C9
:10223000B9F088E697E0B70140E150E00E94090854
:10224000009771F488E697E00E949635109288070F
:1022500084EF93E068E677E00E94F63881E001C001
:1022600083E0C858DF4F0FB6F894DEBF0FBECDBF76
:10227000CF91DF911F910F91FF90EF9008950F93F1
:102280001F9368E677E048E723E431E000E010E0E0
:102290000E9441358823C1F088E697E00E94963578
:1022A0001092A807A8E6B7E0FD018081803209F00E
:1022B0008D938081882311F03196F7CF84E494E0E8
:1022C00068E677E00E94F6388FEF1F910F9108952E
:1022D000EF92FF920F931F93CF93DF93EC0168E689
:1022E00077E048E727E431E000E010E00E94413564
:1022F000882311F00E94D010CE0168E677E048E70D
:102300002BE431E000E010E00E9441358823B9F170
:1023100088E697E00E948C071816190684F500D00D
:1023200000D000D0EDB7FEB7319681EE97E0ADB7A3
:10233000BEB712969C938E93119782E892E0938396
:10234000828382E291E0958384830E94B2368DB7C6
:102350009EB706960FB6F8949EBF0FBE8DBF8091B4
:10236000E7079091E8072091E5073091E607821B87
:10237000930B61E140E00E94812F0E94B038CE01B2
:1023800068E677E048E72FE431E000E010E00E94E3
:102390004135882399F080916807813339F4809121
:1023A000BB0A80FD0BC00E94D43908C0803331F4D1
:1023B0008091BB0A80FF02C00E94DF39CE0168E62F
:1023C00077E048E722E531E000E010E00E94413587
:1023D000882361F188E697E00E948C07EC011816CB
:1023E0001906F4F40E94AB2B7B018C01BE018827F7
:1023F00077FD8095982F20E13EE040E050E00E947C
:10240000A168E60EF71E081F191FE092B70AF092A6
:10241000B80A0093B90A1093BA0A0E94193E06C07E
:10242000009711F081E103C00E94093E81E0DF9135
:10243000CF911F910F91FF90EF9008952F923F92AF
:102440004F925F926F927F928F929F92AF92BF92C4
:10245000CF92DF92EF92FF920F931F93DF93CF9370
:10246000CDB7DEB728970FB6F894DEBF0FBECDBF4D
:102470007B018C014A830894E11CF11C011D111D94
:102480008091AD020E94053A9C018A818823A9F0BF
:102490008091DD099091DE09A091DF09B091E009FA
:1024A0000097A105B10549F079010027F7FC0095D7
:1024B000102FE80EF91E0A1F1B1F9091C20A998364
:1024C0008091BD0A282E33244091BB0A469546953B
:1024D0004695417050E081E0882E912C29016624B8
:1024E00057FC6094762C65C0E52FF0E02814390481
:1024F00009F45BC0CF01880F991F880F991FBC0199
:102500006B51774FDB01AD90BD90CD90DC90A11465
:10251000B104C104D10409F448C09C012B5D374FBC
:102520003C832B83D9018D919D910D90BC91A02D61
:102530000097A105B105C9F5A3E0F695E795AA9521
:10254000E1F7ED53F54F808190E0252F277002C011
:10255000959587952A95E2F780FD27C0D601C5019C
:102560008E0D9F1DA01FB11FEA81EE2391F0EB811C
:10257000FC81E082F18202831383FB0180839183DB
:10258000A283B3837C018D01E40CF51C061D171D8D
:102590000BC0EB81FC81E082F18202831383FB019B
:1025A00080839183A283B38341E05F5F0894811CA1
:1025B000911CF9815F1708F497CF4170440F440FC5
:1025C000440F8091BB0A877F842B8093BB0A289697
:1025D0000FB6F894DEBF0FBECDBFCF91DF911F9134
:1025E0000F91FF90EF90DF90CF90BF90AF909F90B2
:1025F0008F907F906F905F904F903F902F900895B5
:102600008F929F92AF92BF92CF92DF92EF92FF9202
:102610001F93CF93DF93C7E4D2E010E041EEE42EA6
:1026200047E0F42E37EA832E32E0932E29EAA22ED9
:1026300022E0B22E91EBC92E92E0D92E8881282F6C
:1026400030E040E050E0143129F42C533040404059
:1026500050403AC01E3159F4CA01B9012AE030E0B5
:1026600040E050E00E94A1689B01AC012DC01131F7
:1026700059F50E94053A2DB73EB72A5030400FB6A3
:10268000F8943EBF0FBE2DBFEDB7FEB73196ADB784
:10269000BEB71296FC92EE921197D382C2822C8121
:1026A0003D8135832483A0E0B0E086839783A087B3
:1026B000B1870E94B236EDB7FEB73A960FB6F894DE
:1026C000FEBF0FBEEDBF27C08DB79EB70A970FB6EE
:1026D000F8949EBF0FBE8DBFEDB7FEB73196ADB774
:1026E000BEB71296FC92EE921197B382A2828C81B1
:1026F0009D819583848326833783408751870E94F9
:10270000B236EDB7FEB73A960FB6F894FEBF0FBEDD
:10271000EDBF143291F000D000D0ADB7BEB7129625
:10272000FC92EE92119714969C928E9213970E94AF
:10273000B2360F900F900F900F901F5F26961532B4
:1027400009F07CCF0E94D53DEDB7FEB738970FB6A4
:10275000F894FEBF0FBEEDBF319621EE37E0ADB766
:10276000BEB712963C932E93119721E932E0338342
:1027700022838483158285E090E0978386830E947C
:10278000B236EDB7FEB738960FB6F894FEBF0FBE5F
:10279000EDBFDF91CF911F91FF90EF90DF90CF9031
:1027A000BF90AF909F908F9008950E94620A0E9400
:1027B000001380E008958F929F92AF92BF92CF92C4
:1027C000DF92FF920F931F93DF93CF9300D000D03F
:1027D000CDB7DEB76C0183E789831A821B821C8226
:1027E000FF2452E0852E912C8C0E9D1E5E010894D4
:1027F000A11CB11C1CC08F2D90E0B4014AE050E038
:102800000E945E08C60168E677E048E7950100E0AF
:1028100010E00E944135882349F088E697E00E9445
:1028200096358F2D68E677E00E94D438F394809136
:10283000C20AF81600F3C6016DE649EC5AE00E94A0
:10284000380E84EA97E069EC7AE00E94213EC601E6
:1028500069E64FEC5AE00E94380E8AEA97E06FEC86
:102860007AE00E94213EC60161E645ED5AE00E94F1
:10287000380E80EB97E065ED7AE00E94213EC601BC
:1028800064E64BED5AE00E94380E86EB97E06BED64
:102890007AE00E94213E81E00F900F900F900F9000
:1028A000CF91DF911F910F91FF90DF90CF90BF905C
:1028B000AF909F908F900895AF92BF92CF92DF928A
:1028C000EF92FF920F931F93CF93DF9300D000D02E
:1028D00001EE17E0ADB7BEB712961C930E93119799
:1028E00084E196E014969C938E9313970E94B236DF
:1028F000FF240F900F900F900F90E02E012F78E69D
:10290000A72E77E0B72E6FE0C62E66E0D62ECDE07C
:10291000D6E03EC08F2D68E677E00E94B63800D042
:1029200000D000D0EDB7FEB73196ADB7BEB7119667
:10293000EC92119712960C93D382C282B582A48234
:102940000E94B2362F2D30E08091C20A90E00197AC
:10295000EDB7FEB736960FB6F894FEBF0FBEEDBFCB
:1029600028173907A1F000D000D0ADB7BEB7119637
:10297000EC92119712960C9312971496DC93CE93C7
:1029800013970E94B2360F900F900F900F90F39410
:102990008091C20AF81608F4BDCF87E096E069EC92
:1029A0007AE00E94C70A8BEF95E06FEC7AE00E9414
:1029B000C70A81EF95E065ED7AE00E94C70A89EECB
:1029C00095E06BED7AE00E94C70A00D000D000D0FD
:1029D000EDB7FEB7319681EE97E0ADB7BEB7129670
:1029E0009C938E9311978AED95E09383828380E187
:1029F00090E0958384830E94B236EDB7FEB7369699
:102A00000FB6F894FEBF0FBEEDBFDF91CF911F91BF
:102A10000F91FF90EF90DF90CF90BF90AF9008950F
:102A20000E94620A0E945C1480E008950F931F9335
:102A30009C018091DD028823A9F4C90168E677E052
:102A400048E725E531E000E010E00E9441358823A9
:102A500051F088E697E00E94963588E697E00E945C
:102A60001B39811181E01F910F910895DF92EF9240
:102A7000FF920F931F93CF93DF93EC010E940D30D1
:102A80001092E4071092E3078AE194E09093E6073E
:102A90008093E5079093E8078093E707BE016B5F9B
:102AA0007F4FFD8080E2F81621F0EC2EDD2EFE0136
:102AB00004C0CB010E94900E18C18581882359F073
:102AC000803249F08A3039F08F3329F031968F32D5
:102AD000A1F752E1B1C050E0AFC0C52FD0E0FE0178
:102AE000EE0FFF1FEE0FFF1FEA50FE4F0190F08127
:102AF000E02D849190E08017910709F005C131968F
:102B0000849190E04C91242F332727FD3095821734
:102B1000930709F0F9C093E7F91669F44537D9F539
:102B2000CC0FDD1FCC0FDD1FC850DE4FE881F981CF
:102B3000CB01039641C0AAE6FA1669F54F3659F55E
:102B40008B010D5F1F4FC8010E941615882359F590
:102B50000E94620A8DB79EB708970FB6F8949EBF81
:102B60000FBE8DBFEDB7FEB7319681EE97E0ADB7E2
:102B7000BEB712969C938E9311978EE492E0938346
:102B8000828380914B0290914C0295838483809143
:102B9000470286834FC08B010D5F1F4FC8010E9403
:102BA0001615882361F1CC0FDD1FCC0FDD1FC85037
:102BB000DE4FE881F981C8010995282F882309F49F
:102BC00094C08F3FE9F4ADB7BEB718970FB6F8942D
:102BD000BEBF0FBEADBFEDB7FEB7319681EE97E039
:102BE00012969C938E93119789E492E0938382834B
:102BF00082E291E09583848381E891E06AC022E0DB
:102C0000ADB7BEB718970FB6F894BEBF0FBEADBF35
:102C1000EDB7FEB7319681EE97E012969C938E93B6
:102C2000119789E392E09383828388EA91E0958308
:102C30008483268317824FC00F2D112707FD10951F
:102C4000DB011196523109F048CF8091BB0A85FF14
:102C50004CC0C8E6D7E08E2D9D2D9C01D90101C046
:102C60008993EA2FEE1915968C911597803229F0E9
:102C7000119697E0C838D90799F7F0E0E859F84F6E
:102C8000108289EE97E068E571E040E00E942E49ED
:102C900088E697E00E946E0D8823C1F5ADB7BEB7F8
:102CA00018970FB6F894BEBF0FBEADBFEDB7FEB715
:102CB000319681EE97E012969C938E93119789E25C
:102CC00092E09383828388EA91E09583848380E213
:102CD00090E0978386830E94B2368DB79EB70896A0
:102CE0000FB6F8949EBF0FBE8DBF8091E7079091FD
:102CF000E8072091E5073091E607821B930B61E11D
:102D000040E00E94812F02C05F5F9CCFDF91CF9196
:102D10001F910F91FF90EF90DF9008958F929F92F7
:102D2000AF92BF92CF92DF92EF92FF920F931F93D9
:102D3000CF93DF93EC017A018B01CB01BA010E94A2
:102D4000982A4C01C801B7010E94922A5C0188812F
:102D500080FFACC0C801B7010E94862AC82EC801F6
:102D6000B7010E948C2AD82E88818295837090E0CA
:102D700082309105B1F083309105F1F0892BB1F5E6
:102D8000298130E08C2D90E0059667E070E00E948C
:102D9000E06802C0359527958A95E2F720FD26C0A8
:102DA00085C02D2D30E0898190E08F7190702817BB
:102DB000390709F07BC01AC0C801B70120E831E526
:102DC00041E050E00E94F368CA01B9012A8130E075
:102DD00040E050E00E94F368298130E040E050E09C
:102DE000621773078407950709F060C0888186958C
:102DF00086958370B9F0823019F4D0FE13C056C0A6
:102E0000813081F48FE1D81609F450C08DE1D816D5
:102E100009F05BC0C801B7010E94802A029709F03F
:102E200054C044C08CE390E0889E9001899E300D90
:102E3000989E300D11242A0D3B1D888186FD29C0E6
:102E40000D811E81EF81F8858B819C8128173907C0
:102E500068F10115110529F460E02817390739F5E3
:102E60001FC0309719F1281B390BC901BF010E94FF
:102E7000CC68AB016E9FC0016F9F900D7E9F900D3F
:102E800011248217930791F460E0041715077CF072
:102E900007C0FE0140E0838194812817390711F4AF
:102EA00061E005C04F5F32964430A9F760E0862F9D
:102EB000DF91CF911F910F91FF90EF90DF90CF9016
:102EC000BF90AF909F908F900895D0FCABCFEECF86
:102ED000982F9B0180912408981768F467E4969FC7
:102EE000B00111246E5F7F4FC90147E450E027EE27
:102EF00038E00E94260808952F923F924F925F92E9
:102F00006F927F928F929F92AF92BF92CF92DF92F9
:102F1000EF92FF920F931F93DF93CF93CDB7DEB75E
:102F2000C754D0400FB6F894DEBF0FBECDBF2DB74B
:102F30003EB72E5030400FB6F8943EBF0FBE2DBFA7
:102F4000EDB7FEB7319601EE17E0ADB7BEB71296FA
:102F50001C930E93119788E894E093838283809169
:102F60002408848315828091C10A868317828EE0AB
:102F700090E09187808784E090E0938782878CE05F
:102F800090E0958784870E94B236EE24EDB7FEB7B5
:102F90003E960FB6F894FEBF0FBEEDBFF02E012F88
:102FA00058E7C52E54E0D52E4CE0642E712C6C0EE3
:102FB0007D1E8F2C912E3EE5232E34E0332E21E60C
:102FC000422E24E0522E9AE1A92E94E0B92E57C148
:102FD0008E2DBE016F5F7F4F0E9468178981829599
:102FE0008370833039F48B81823020F0CE010296D9
:102FF0000E9493102DB73EB72A5030400FB6F89478
:103000003EBF0FBE2DBFEDB7FEB73196ADB7BEB711
:103010001196FC92119712960C932CE734E03383AF
:1030200022838981848315828A81868317828B819A
:10303000808711860E94B2360F900F900F900F90EC
:10304000EDB7FEB73196ADB7BEB71196FC921197AA
:1030500012960C93D382C2828C819D819583848346
:103060000E94B236EDB7FEB73196ADB7BEB7119636
:10307000FC92119712960C93D382C2828E819F810B
:10308000958384830E94B236EDB7FEB73196ADB713
:10309000BEB71196FC92119712960C93D382C282FE
:1030A00088859985958384830E94B236EDB7FEB7F3
:1030B0003196ADB7BEB71196FC92119712960C934C
:1030C00022E734E0338322838A859B85958384833A
:1030D0000E94B23610E04DB75EB74A5F5F4F26C020
:1030E000E60DF71D80810E94053AADB7BEB718976F
:1030F0000FB6F894BEBF0FBEADBFEDB7FEB73196A9
:103100001196FC92119712960C932EE634E03383BD
:103110002283A0E0B0E084839583A683B7830E94D6
:10312000B2361F5F4DB75EB7485F5F4F0FB6F8947A
:103130005EBF0FBE4DBFE12FF0E08091C20A90E06C
:103140000197E817F90764F2E60DF71D80810E94E8
:10315000053AADB7BEB718970FB6F894BEBF0FBE0D
:10316000ADBFEDB7FEB7319611968C9211971296BE
:103170009C9228E634E033832283A0E0B0E084838D
:103180009583A683B7830E94B2364DB75EB7485F7A
:103190005F4F0FB6F8945EBF0FBE4DBF88E697E055
:1031A000BE01645C7F4F4CE050E00E941708109213
:1031B000740700D000D000D0EDB7FEB73196ADB7A0
:1031C000BEB711968C92119712969C9225E634E028
:1031D0003383228348E657E0558344830E94B23606
:1031E0002E2D30E08091240890E00197ADB7BEB756
:1031F00016960FB6F894BEBF0FBEADBF281739079D
:1032000049F000D000D0EDB7FEB7F18202835482BE
:1032100043820EC000D000D0ADB7BEB71196FC926D
:10322000119712960C93129714963C922E92139724
:103230000E94B2360F900F900F900F908E2D63E08A
:103240000E94C0689230D1F48091E7079091E8071E
:103250002091E5073091E607821B930B60E140E087
:103260000E94812F1092E4071092E307B092E607C4
:10327000A092E507B092E807A092E707E394809157
:103280002408E81608F4A4CE00D000D081EE97E020
:10329000EDB7FEB7928381838BE594E094838383BB
:1032A0000E94B2360F900F900F900F90C95BDF4FC6
:1032B0000FB6F894DEBF0FBECDBFCF91DF911F9147
:1032C0000F91FF90EF90DF90CF90BF90AF909F90C5
:1032D0008F907F906F905F904F903F902F900895C8
:1032E0000E94620A0E947C1780E00895DF92EF92AC
:1032F000FF920F931F93DF93CF93CDB7DEB7C754E1
:10330000D0400FB6F894DEBF0FBECDBF2091240889
:10331000821708F046C0222309F443C090E00196CA
:1033200027E430E0829F8001839F100D929F100D53
:1033300011240E5F1F4F67E4D62E7E010894E11C16
:10334000F11C14C0C701B80147E450E027EE38E093
:103350000E942608C80187549040B70147E450E016
:103360002FEE38E00E944208095B1F4F209124088D
:103370002D9DC001112402960817190718F321503A
:1033800020932408F999FECF1FBA81E090E092BD06
:1033900081BD20BD0FB6F894FA9AF99A0FBE81E06C
:1033A00001C080E0C95BDF4F0FB6F894DEBF0FBEEF
:1033B000CDBFCF91DF911F910F91FF90EF90DF90E4
:1033C00008950F931F9368E677E048E72FE131E017
:1033D00000E010E00E944135882311F480E125C00F
:1033E00088E697E00E948C079C018FEF2F3F3807FB
:1033F00081F410922408F999FECF1FBA81E090E081
:1034000092BD81BD10BC0FB6F894FA9AF99A0FBE1E
:103410000BC08091240890E02817390714F081E14F
:1034200004C0822F0E94761981E01F910F910895A8
:10343000982F80912408981710F080E0089587E471
:10344000989FC0011124029647E450E02FEE38E027
:103450000E94420881E00895BC01909124089E30AA
:1034600010F080E0089587E4989FC001112402962F
:1034700047E450E02FEE38E00E94420820912408F3
:103480002F5F20932408F999FECF1FBA81E090E0C6
:1034900092BD81BD20BD0FB6F894FA9AF99A0FBE7D
:1034A00081E00895BF92CF92DF92EF92FF920F9347
:1034B0001F93DF93CF93CDB7DEB7C954D0400FB67B
:1034C000F894DEBF0FBECDBF7C0168E677E048E729
:1034D0002FE131E000E010E00E944135882309F43B
:1034E000D7C088E697E00E948C076C012FEF8F3FD2
:1034F00092070CF4CFC08091240890E0C816D9063A
:103500000CF0C8C0FA82E98284E690E0E80EF91E69
:103510000DC0C8016AE571E043E050E00E9409086F
:10352000009779F00F5F1F4F1A83098309811A8171
:10353000F8018081882309F4ABC00E151F0548F3FC
:10354000A7C00D5F1F4F1A8309838E010F5F1F4FA6
:10355000C8010E94080E8B83C8010E94080E8C834C
:10356000C8010E94080E8D8389819A8101969A83F1
:103570008983C8010E94080E9F838E83C8010E9420
:10358000080E99878887C8010E94080E9B878A8742
:10359000C8010E94080E9D878C8789819A810296B6
:1035A0009A838983FF24B02EE12E8E01025F1F4F84
:1035B0000BC08B2D9E2D0E94080E0E94E939F80148
:1035C000EF0DF11D8083F3948091C20AF81688F301
:1035D00089819A8102969A83898368E677E048E731
:1035E0002EE531E000E010E00E9441358E01025CE2
:1035F0001F4F882361F088E697E00E949635C80146
:1036000068E677E04CE050E00E9417081EC0C80151
:1036100063E671E00E940208FFEFCF16FFEFDF06BE
:1036200021F48091240890E001C0C6010196BE01FA
:103630006A5B7F4F4AE050E00E945E0806C0FC01D2
:10364000EF0DF11D1082F39402C0CE010E962FE211
:103650002F15A8F78B8182958370833039F48D8183
:10366000823020F0CE0104960E946910BE016D5F89
:103670007F4F8FEFC8168FEFD80621F4CB010E9441
:103680002C1A03C08C2D0E94181A882329F402C01A
:1036900080E103C081E101C081E0C75BDF4F0FB66D
:1036A000F894DEBF0FBECDBFCF91DF911F910F9178
:1036B000FF90EF90DF90CF90BF900895EF92FF9230
:1036C0000F931F93DF93CF93CDB7DEB727970FB636
:1036D000F894DEBF0FBECDBF7C0189EE97E068E5B0
:1036E00071E040E00E942E498E010F5F1F4FC8011C
:1036F00061E673E00E946868C801B7010E9425680E
:10370000C8016CE671E00E942568C80168E677E0B0
:1037100048E750E020E030E00E940967C8010E94BD
:103720009B6827960FB6F894DEBF0FBECDBFCF9132
:10373000DF911F910F91FF90EF9008952F923F928C
:103740005F926F927F928F929F92AF92BF92CF9231
:10375000DF92EF92FF920F931F93DF93CF93CDB73A
:10376000DEB76E970FB6F894DEBF0FBECDBF5C011B
:103770008091BB0A85FD02C080E220C1C50168E6D8
:1037800077E048E721E731E000E010E00E944135B2
:10379000882309F410C188E697E00E94AA076B010C
:1037A0007C01C50168E677E048E727E731E00E9441
:1037B0004135882309F4FFC0C701B60120E831E58F
:1037C00041E050E00E94156969017A0188E697E0BE
:1037D0000E94AA0720E831E541E050E00E94156907
:1037E00059012C153D0508F4E8C0C9018C199D0943
:1037F0008E56914008F0E1C000D000D000D0EDB767
:10380000FEB7319601EE17E0ADB7BEB712961C9326
:103810000E93119780E692E09383828388EA91E089
:10382000958384830E94B236EE24FF247724739418
:10383000EDB7FEB736960FB6F894FEBF0FBEEDBFDC
:10384000E8E62E2EE7E03E2E75E0872E912C8C0EBA
:103850009D1E502E612E0AE114E095C0C60168E657
:1038600077E04AE050E00E945E0888E697E00E9418
:103870005E1B89EE97E068E677E00E940F49882397
:1038800009F47EC01D821F821C821B828FEB93E095
:103890009A838983C40168E677E041E00E94675912
:1038A00001C07724C40168E677E047E750E020E0F4
:1038B00030E00E9484541816190624F0C4010E94B6
:1038C0006B515EC0FC01E959F84F80818A3009F4E0
:1038D0001082772081F000D000D000D0EDB7FEB785
:1038E0003196ADB7BEB711965C92119712966C9255
:1038F0008DE592E00FC000D000D000D0EDB7FEB74C
:103900003196ADB7BEB711965C92119712966C9234
:1039100089E592E093838283358224820E94B236C5
:10392000ADB7BEB716960FB6F894BEBF0FBEADBF0B
:103930000894E11CF11CC70169E170E00E94E06895
:10394000892B09F0AECF8091E7079091E80720918D
:10395000E5073091E607821B930B60E140E00E948F
:10396000812F1092E4071092E3071093E60700936B
:10397000E5071093E8070093E707EE24FF2491CFB3
:103980000894C11CD11CAC14BD0408F067CF00D052
:1039900000D081EE97E0EDB7FEB79283818387E593
:1039A00092E0948383830E94B23680E00F900F9060
:1039B0000F900F9003C080E101C081E16E960FB6B9
:1039C000F894DEBF0FBECDBFCF91DF911F910F9155
:1039D000FF90EF90DF90CF90BF90AF909F908F902F
:1039E0007F906F905F903F902F900895BF92CF92FD
:1039F000DF92EF92FF920F931F93DF93CF93CDB798
:103A0000DEB7A5970FB6F894DEBF0FBECDBFB82EB8
:103A10006A017B018091BB0A85FFCAC0CB01BA0154
:103A200020E831E541E050E00E94F368CA01B901A5
:103A300048E657E02AE030E00E949C0888E697E0DC
:103A40000E945E1B89EE97E068E571E040E00E940D
:103A50002E4989EE97E061E673E040E00E942E492E
:103A6000882351F489EE97E061E673E041E00E941B
:103A7000F048882309F49CC01C861E861B861A8683
:103A80008FEB93E0998788878E01045F1F4FC801F1
:103A900068E677E042E40E9467594E8D5F8D68A129
:103AA00079A1C8010E94034F8E010F5F1F4FC8010B
:103AB0006BE771E00E946868C8016CE771E00E94E2
:103AC000826881E0B81619F1B81628F082E0B816BD
:103AD00009F041C02AC0C8016091D6090E94F96767
:103AE000C8016EE771E00E942568C8016091D509A0
:103AF0000E94F967C8016EE771E00E942568609135
:103B0000D7097091D809C8010E94CB6724C0C801A9
:103B100060E871E00E9425688091E10A9091E20AD4
:103B2000A091E30AB091E40A0DC0C80168E871E011
:103B30000E9425688091E50A9091E60AA091E70A23
:103B4000B091E80AB701A601481B590B6A0B7B0B21
:103B5000C8010E9499678E010F5F1F4FC8016EE771
:103B600071E00E942568C801B701A6010E9499670B
:103B7000C80160E971E00E942568C80162E971E04E
:103B80000E942568C80168E677E048E750E020E039
:103B900030E00E940967CE01089668E677E00E944F
:103BA000785ECE010C960E946B51C8010E949B6802
:103BB000A5960FB6F894DEBF0FBECDBFCF91DF91B3
:103BC0001F910F91FF90EF90DF90CF90BF900895DD
:103BD000CF93DF93EC018091BB0A85FF28C0CE0113
:103BE00065E971E043E050E00E940908009771F434
:103BF00089EE97E061E673E040E00E942E49882359
:103C0000B1F087E098E00E94E55311C0CE010E9418
:103C10005E1B89EE97E068E677E00E940F498823F3
:103C200031F089EE97E068E677E00E94EC48DF919A
:103C3000CF9108950F931F9368E677E048E729E94D
:103C400031E000E010E00E944135882311F480E16A
:103C500005C088E697E00E94E81D81E01F910F9162
:103C600008950E9471390E94653FA5EAB9E080E09D
:103C700090E0FC01EB5DF74F1082118212821382FB
:103C8000FC01EB51F74F10821182128213821D92B8
:103C90000496803C910569F71092DD091092DE09C7
:103CA0001092DF091092E00908952F923F924F92EF
:103CB0005F926F927F928F929F92AF92BF92CF92BC
:103CC000DF92EF92FF920F931F93DF93CF9300D079
:103CD00000D000D0CDB7DEB74C01A7E4EA2EA2E0B9
:103CE000FA2E7724CC2466242224AA24BB24F2E0D2
:103CF0004F2E512C4C0E5D1EDA2C84E2A81609F4CE
:103D000088C098E1A91609F484C02A2D9B2DF701DB
:103D100030808181813009F41082D201E9E5F3E03D
:103D200085E001900D928150E1F7822FBE016D5F19
:103D30007F4F4AE050E00E945E08C40168E677E0E9
:103D400048E7920100E010E00E944135882309F421
:103D50003FC0F7018181813011F4808339C088E64A
:103D600097E00E94AA079B01AC01F4E1DF1629F459
:103D7000245C3F4F4F4F5F4F1BC08EE1D81669F454
:103D8000CA01B9012AE030E040E050E00E94156924
:103D9000C901DA019C01AD010BC091E1D91641F4D2
:103DA000C9010E94E939282F30E040E050E002C00C
:103DB00057FD0CC0F701818190E0A0E0B0E08217D0
:103DC0009307A407B50714F0208302C0222423948C
:103DD000F70180818315E9F08D2D8150823010F438
:103DE000772473948D2D8052843010F4772473944B
:103DF0008D2D83508B3010F466246394FAE1DF1626
:103E000019F46624639405C08FE1D81611F4CC240C
:103E1000C3940894A11CB11CE6E0F0E0EE0EFF1E76
:103E2000F5E2AF16B10409F067CFC40168E677E0A8
:103E300048E72DE931E000E010E00E944135882399
:103E4000B1F088E697E00E9496351092980788E6D0
:103E500097E064E174E00E943539882341F084E101
:103E600094E068E677E00E94F638CC24C394198287
:103E7000C40168E677E048E721EA31E08E010F5F90
:103E80001F4F0E9441358823B9F088E697E00E94D1
:103E900096351092880788E697E064E874E00E94FF
:103EA00035398823A1F084E894E068E677E00E9441
:103EB000F638CC24C3940BC08981882341F010923A
:103EC000680784E894E068E677E00E94F63880911D
:103ED0005302882331F5C40168E677E048E727EA12
:103EE00031E000E010E00E9441358823D1F088E6FF
:103EF00097E00E94AA07162F072FF82EE92E0E949E
:103F0000311E612F702F8F2D9E2D0E947E2B809150
:103F1000BB0A84FF06C0612F702F8F2D9E2D0E943B
:103F20007E2D222011F081E121C00E94A739772047
:103F300041F01092ED0A1092EE0A1092EF0A1092E0
:103F4000F00ACC2041F01092F10A1092F20A10927D
:103F5000F30A1092F40A662041F01092F50A1092CA
:103F6000F60A1092F70A1092F80A81E026960FB628
:103F7000F894DEBF0FBECDBFCF91DF911F910F919F
:103F8000FF90EF90DF90CF90BF90AF909F908F9079
:103F90007F906F905F904F903F902F900895DF92A9
:103FA000EF92FF920F931F93DF93CF9300D0CDB783
:103FB000DEB79A83898324E6E22EF12CE80EF91EFF
:103FC0000DC0C8016BEA71E043E050E00E940908AF
:103FD000009779F00F5F1F4F1A83098309811A81B7
:103FE000F8018081882309F453C00E151F0548F39A
:103FF0004FC00D5F1F4F1A8309830E94311E10E0CE
:1040000000E07E010894E11CF11C8EEFD82E2EC03A
:10401000C7010E94080EBC01009739F1412F50E002
:10402000E12FE695E695E695F0E0E552F54F8081C3
:1040300090E0212F277002C0959587952A95E2F789
:1040400080FD13C0FA01EE0FFF1FEE0FFF1FEB51B3
:10405000F74FCB01A0E0B0E080839183A283B383CC
:104060004B55564FFA01D08201E01F5F8091C20A82
:10407000181770F2002361F00E94AB2B4091BB0A2D
:1040800042954695469541700E941E1281E001C0FE
:1040900080E10F900F90CF91DF911F910F91FF90D2
:1040A000EF90DF900895AF92BF92CF92DF92EF92A0
:1040B000FF920F931F93DF93CF93CDB7DEB7C75413
:1040C000D0400FB6F894DEBF0FBECDBFE82E0E94E1
:1040D000311E8E2D81508E3F28F4BE016F5F7F4FC1
:1040E0000E946817DD24FF24EEEFCE2E7CE0A72E81
:1040F000B12CAC0EBD1E3CC00F2D10E08FEFE816AA
:1041000019F442E050E00CC0EE2009F443C0F50180
:10411000E00FF11F80810E94053AAC01009739F150
:10412000F80163E0F695E7956A95E1F7E552F54FFA
:10413000808190E02F2D277002C0959587952A9554
:10414000E2F780FD14C0F801EE0FFF1FEE0FFF1F16
:10415000EB51F74FCA01A0E0B0E080839183A283C6
:10416000B3830B55164FF801C082DD24D394F3942A
:104170008091C20AF81608F4BFCFDD2071F00E94CA
:10418000AB2B4091BB0A42954695469541700E94E3
:104190001E1203C04CE350E0C3CFC95BDF4F0FB624
:1041A000F894DEBF0FBECDBFCF91DF911F910F916D
:1041B000FF90EF90DF90CF90BF90AF9008958F92D7
:1041C0009F92AF92BF92CF92DF92EF92FF920F93A6
:1041D0001F93CF93DF93B82EA62E79018A01C82EA4
:1041E000DD2460E00E944D39F601EE0FFF1FEE0F57
:1041F000FF1FEB5DF74F20813181428153812115F3
:1042000031054105510509F49AC02E153F054007B7
:10421000510708F07BC0C60143E0959587954A9504
:10422000E1F7982E87E0882E8B20CA2DD0E0C601BA
:104230000196C817D90709F444C0B092D509F60110
:10424000EB55F64F80818093D609C701821B930BF3
:104250009093D8098093D709E092D909F092DA09AE
:104260000093DB091093DC0980E0B801A7010E94EC
:10427000F61CE92DF0E0E753F54F808190E0082C23
:1042800002C0959587950A94E2F780FF1AC0809145
:10429000BB0A86FF16C0CC0FDD1FCC0FDD1FCF5130
:1042A000D74F8091BF0290E0A0E0B0E0CC97A10989
:1042B000B1098E0D9F1DA01FB11F88839983AA830A
:1042C000BB83E92DF0E0EB52F54F808190E002C016
:1042D000959587958A94E2F780FF18C08091FB023C
:1042E000882381F08EE061E00E94BB626091FB0256
:1042F0002AE0629FB0011124882777FD8095982FCE
:104300000E94C4638EE060E00E94BB62F601EE0F83
:10431000FF1FEE0FFF1FDF01AB5DB74F1D921D9218
:104320001D921C921397EB51F74F1082118212824B
:10433000138285EA99E0C80ED91EF6011082DF913A
:10434000CF911F910F91FF90EF90DF90CF90BF9092
:10435000AF909F908F900895AF92BF92CF92DF92CF
:10436000EF92FF920F931F93CF93DF937C0168E648
:1043700077E048E72FEA31E000E010E00E944135A5
:10438000882309F492C088E697E00E948C07EC012C
:1043900097FD89C08091C20A90E0C817D9070CF038
:1043A00082C0C70168E677E048E72FE431E00E9469
:1043B0004135882309F479C088E697E00E948C078C
:1043C000182F0E94AB2B5B016C01112309F462C012
:1043D000C70168E677E048E723EB31E000E010E052
:1043E0000E944135882309F460C088E697E00E9466
:1043F000AA07CB01019780529D4F08F054C08091CD
:10440000BD0A90E09E012F5F3F4F8217930709F48A
:104410004EC0FE0113E0F595E7951A95E1F7F0E03F
:10442000ED53F54F808190E0AE014770042E02C03D
:10443000959587950A94E2F780FD39C0FE01EE0F4D
:10444000FF1FEE0FFF1FEB51F74F80819181A2817B
:10445000B3810097A105B10551F5FE01EE0FFF1FD5
:10446000EE0FFF1FEB51F74FCB01A0E0B0E08083D0
:104470009183A283B383CB55D64F83E68883409143
:10448000BB0A4295469546954170C601B5010E940A
:104490001E1207C08C2F6091BD0AA60195010E94D3
:1044A000DF2081E005C081E103C080E101C080E33D
:1044B000DF91CF911F910F91FF90EF90DF90CF9000
:1044C000BF90AF9008954F925F926F927F928F92BC
:1044D0009F92AF92BF92CF92DF92EF92FF920F9393
:1044E0001F93CF93DF935B016C019091BB0A44242F
:1044F0004394492291FD0CC08091C502882311F498
:10450000FF2408C0F92EF694F69481E0F82211F009
:10451000FF24F394EE245BC08E2D90E0FC01E15368
:10452000F54F3081FC01ED53F54F20815E2C550C89
:10453000550C550C00E010E0622E7724832E992450
:10454000252D200FC22FD0E0FE01EB55F64FE08164
:10455000E336B0F5442059F0FF2091F1C401002E5C
:1045600002C0959587950A94E2F780FD29C0C301A2
:10457000002E02C0959587950A94E2F780FF08C047
:10458000822F6091BD0AA60195010E94DF2018C00C
:10459000EE23B1F0FE01EE0FFF1FEE0FFF1FDF0154
:1045A000AB5DB74F1D921D921D921C921397EB515C
:1045B000F74F1082118212821382CB55D64F188288
:1045C0000F5F1F4F0830110509F0BACFE3948091B7
:1045D000C10AE81608F4A0CFDF91CF911F910F9187
:1045E000FF90EF90DF90CF90BF90AF909F908F9013
:1045F0007F906F905F904F900895AF92BF92CF924F
:10460000DF92EF92FF920F931F935B016C018091F9
:10461000BB0A83FDBAC08091F50A9091F60AA09179
:10462000F70AB091F80A0097A105B10511F40E94AC
:104630004B412091BC0A22952F7061E070E002C0CE
:10464000660F771F2A95E2F7882777FD8095982FC8
:104650002091F50A3091F60A4091F70A5091F80A34
:1046600086017501E21AF30A040B150B2EE130E006
:1046700040E050E00E94A1686E157F058007910719
:1046800008F083C08091E109882359F48EE99AE00B
:104690006FE041E00E9484458EE99AE064E00E9468
:1046A0004045A092F50AB092F60AC092F70AD0925D
:1046B000F80A89E89AE00E9460310E94B6637B01A3
:1046C0008C010E945E470E94AD3189E89AE00E9409
:1046D0002234882361F40E94B6636E197F09800B2F
:1046E000910B683C71058105910558F33AC08091A2
:1046F000BC0A8F7002C08F7080668093BC0A809164
:10470000BC0A82958F7090E00397ACF48091F90A0F
:104710009091FA0AA091FB0AB091FC0AA6019501BA
:10472000281B390B4A0B5B0BDA01C901815C984AE3
:10473000A040B04050F180919B02882331F1A092BB
:10474000F90AB092FA0AC092FB0AD092FC0A0E94BF
:104750004B418823D1F08091BC0A8F708093BC0AB2
:1047600014C08091BC0A282F22952F702F5F2F70C4
:10477000922F9295907F8F70892B8093BC0A30E0A6
:10478000273031050CF0B7CFBACF1F910F91FF90B2
:10479000EF90DF90CF90BF90AF900895EF92FF928F
:1047A0000F931F939B01AC0180915302882309F45E
:1047B00047C08091BC0A82958F7009F041C08091FA
:1047C000BB0A83FD3DC08091ED0A9091EE0AA09155
:1047D000EF0AB091F00A0097A105B10569F07901DF
:1047E0008A01E81AF90A0A0B1B0BD801C701815884
:1047F0009145A140B04020F12093ED0A3093EE0A9C
:104800004093EF0A5093F00A8091E109882329F43C
:104810008DE296E061E00E94033B0E94DD0C7B018B
:104820008C01611571058105910551F00E947E2B67
:104830008091BB0A84FF04C0C801B7010E947E2D8D
:104840001F910F91FF90EF90089584B7877F84BFE9
:104850000E940E400E94463E0E9435096CE370E0C3
:1048600080E090E00E94752B8091BB0A84FD03C01C
:1048700080E090E002C08EE99DE20E941E2C64EF71
:1048800071E080E090E00E94C46380E00E94C43F39
:104890008091600088618093600081E28093600075
:1048A000809160008064809360008CE396E061E01A
:1048B0000E94033B89EE97E060E044E00E947D495E
:1048C000882329F08091BB0A80628093BB0A0E94F2
:1048D0004B41882321F08091BC0A8F7004C08091E5
:1048E000BC0A8F7080618093BC0A64EF71E080E045
:1048F00090E00E94C4630E94653F0E94AB2B6093CE
:10490000E90A7093EA0A8093EB0A9093EC0A0895FF
:10491000BF92CF92DF92EF92FF920F931F93DF939C
:10492000CF93CDB7DEB7C754D0400FB6F894DEBFF3
:104930000FBECDBF6B017C018091E90A9091EA0A1C
:10494000A091EB0AB091EC0A0097A105B105D9F04E
:104950000F96A11DB11D8C159D05AE05BF0598F4E0
:104960008091F5026FEF70E0681B71098CE00E9486
:104970001C621092E90A1092EA0A1092EB0A109255
:10498000EC0A1092E10982E00E94743AB82E082FD6
:1049900010E086FFBFC0C092E90AD092EA0AE09216
:1049A000EB0AF092EC0A8091EF026FEF70E0681B67
:1049B00071098CE00E941C628091E109833020F42F
:1049C000813008F063C004C0833009F0A3C052C036
:1049D000C8018F70907082309105F1F0843091059C
:1049E00051F1019709F096C0B7FE0CC08EE10E940C
:1049F0000F63892B21F48FEF0E9453208BC00E94FC
:104A0000D01088C060914502709146028DE79AE00F
:104A10000E948D3D81E00CC0B7FE03C00E94B038FB
:104A200079C089E89AE060E070E00E948D3D82E004
:104A30008093E1096FC0B7FE0CC084E896E060E0A7
:104A40000E94033B83E796E061E00E94033B83E022
:104A5000EFCF2091BC0A822F8F7090E06091C10A45
:104A6000019670E00E94E0688F70207F282B2093D1
:104A7000BC0A50C00F7010700430110509F04AC014
:104A8000B7FE07C08091EC090E9453201092E10903
:104A900041C08091EC0990E06091240870E06F5F64
:104AA0007F4F01960E94E0688093EC0982E696E0D1
:104AB00060E00E94033B8091EC09882331F1815032
:104AC000BE016F5F7F4F0E94681780E696E061E04D
:104AD0000E94033B8EE99AE060E041E00E94844539
:104AE0006091EC098EE99AE070E04AE050E00E94A3
:104AF000E4668DE596E00E94F33A8EE99AE0BE0105
:104B0000645C7F4F0E94F76605C08DE496E061E02B
:104B10000E94033BC95BDF4F0FB6F894DEBF0FBEA8
:104B2000CDBFCF91DF911F910F91FF90EF90DF905C
:104B3000CF90BF9008952F923F924F925F926F92C5
:104B40007F928F929F92AF92BF92CF92DF92EF921D
:104B5000FF920F931F93DF93CF93CDB7DEB7C1556D
:104B6000D0400FB6F894DEBF0FBECDBF8091A70234
:104B700081708295880F880F807C9091BB0A9F7B03
:104B8000982B9093BB0A8091B3028093BD0A0E9438
:104B90005E470E94AD319093E3098093E20900974C
:104BA00021F08C519C4F0E943615A8951092230835
:104BB0000E94AB2B4B015C010E9488248091E80984
:104BC0009091E909A091EA09B091EB09881599053E
:104BD000AA05BB0509F452C38092E8099092E9093D
:104BE000A092EA09B092EB098091E109882311F4BF
:104BF0000E94C43F8091BB0A81FF10C08091B70A18
:104C00009091B80AA091B90AB091BA0A881699068B
:104C1000AA06BB0690F00E94093E0FC08091B70A19
:104C20009091B80AA091B90AB091BA0A881699066B
:104C3000AA06BB0610F40E94193E0E94BD3A90914C
:104C4000BB0A969591708091BE0A869581708917EE
:104C5000C9F0992349F08092E50A9092E60AA09261
:104C6000E70AB092E80A05C082E0B501A4010E94FB
:104C7000F61C9091BB0A92708091BE0A8D7F892BA1
:104C80008093BE0A9091BB0A9695969591708091FB
:104C9000BE0A8695869581708917C9F0992349F0D7
:104CA0008092E10A9092E20AA092E30AB092E40AAA
:104CB00005C081E0B501A4010E94F61C9091BB0AD9
:104CC00094708091BE0A8B7F892B8093BE0AC501A8
:104CD000B4012CE330E040E050E00E94F368790139
:104CE0008A018091E4099091E509A091E609B091CB
:104CF000E709E816F9060A071B0709F4B0C0E092B5
:104D0000E409F092E5090093E6091093E7096624A7
:104D100055241E010894211C311C90C0862DB10120
:104D20000E946817C101B501A4010E948E16882354
:104D300009F483C07724462C43947AC0C72CDD2421
:104D40008091BD0A90E096012F5F3F4F8217930735
:104D500009F46DC0D60123E0B695A7952A95E1F731
:104D6000272D2770FD01ED53F54F808190E0022E35
:104D700002C0959587950A94E2F780FD58C0A55228
:104D8000B54F8C9190E002C0959587952A95E2F7F2
:104D900080FD4DC0ECE0F0E0EC0FFD1FEC0DFD1DC3
:104DA0002081222309F443C0F601EE0FFF1FEE0F0E
:104DB000FF1FEB51F74F80819181A281B381009752
:104DC000A105B105A1F5822F0E94053A7C0100E002
:104DD00010E0898181FF13C02091D10230E040E0D2
:104DE00050E0C801B7010E94A16824E630E040E02D
:104DF00050E00E94F368C901DA017C018D01F601DF
:104E0000EE0FFF1FEE0FFF1FEB51F74FE082F18215
:104E100002831383E114F1040105110541F025EA31
:104E200039E0C20ED31ED6014C925524539473948C
:104E30008091C20A781608F481CF63948091240887
:104E4000681608F46BCF552051F04091BB0A42958B
:104E5000469546954170C501B4010E941E1280918D
:104E6000BB0A83FFA3C12A961FAE2A972EC12A969A
:104E7000BFAD2A978B2F90E0FC01ED53F54F2081B9
:104E8000EB2FEE0FEE0FEE0F2B96EFAF2B97442488
:104E90005524422F50E02E965FAF4EAF2E97DC0187
:104EA000AB52B54F6096BFAFAEAF6097FC01E75312
:104EB000F54F6296FFAFEEAF62972B961FAD2B9723
:104EC000140D612E7724F301EB55F64F8081882372
:104ED000B9F0F301EE0FFF1FEE0FFF1FEB51F74F7D
:104EE00080819181A281B38188169906AA06BB06AA
:104EF00038F0812F6091BD0AA50194010E94DF2046
:104F00002C964FAE2C972E968EAD9FAD2E97042CDF
:104F100002C0959587950A94E2F780FDC7C093017A
:104F2000220F331F220F331FA5E2EA2EA8E0FA2E2C
:104F3000E20EF31EF70180819181A281B381881670
:104F40009906AA06BB0608F4B1C0F5EE2F2EF8E0CC
:104F50003F2E220E331EF10180819181A281B38107
:104F600088169906AA06BB0608F0A0C0812F61E04A
:104F70000E944D390091BD0A002309F471C0202F11
:104F800030E0C30101962817390709F469C0629619
:104F9000AEADBFAD62978C9190E02C960FAC2C9784
:104FA00002C0959587950A94E2F780FF59C08091D9
:104FB000BB0A86FF55C0015029960FAF299710E014
:104FC0008091B902F7012081318142815381280FFC
:104FD000311D411D511DB801660F771F660F771FE8
:104FE000FB01EB5DF74F2083318342835383809134
:104FF000BF02C82EDD24EE24FF2484EC9FEFAFEF28
:10500000BFEFC80ED91EEA1EFB1EF10180819181FF
:10501000A281B381C80ED91EEA1EFB1E6B51774FC9
:10502000DB01CD92DD92ED92FC9213970B55164F5A
:10503000E5EAF9E06E0E7F1ED3018C91F8018083C2
:1050400082169306A406B50658F08C149D04AE048F
:10505000BF0430F429968FAD299761E00E944D3945
:105060006096AEADBFAD60978C9190E02C960FAC82
:105070002C9702C0959587950A94E2F780FF16C099
:105080008EE061E00E94BB628091FB02882371F098
:10509000BAE08B9FB0011124882777FD8095982F67
:1050A0000E94C4638EE060E00E94BB620894411CD1
:1050B000511CE8E04E16510409F0FFCE2A96FFADD0
:1050C0002A97FF5F2A96FFAF2A978091C10A2A96F6
:1050D0002FAD2A97281708F4CACEC501B4010E9443
:1050E00063220E94653F8091C20AE5EEF8E060E02D
:1050F000EE24FF24870190E0880F991F880F991FE5
:105100008E0F9F1F12C020813181428153818216F0
:105110009306A406B50640F4E216F3060407150745
:1051200010F479018A0161E03496E817F90759F71C
:10513000E092DD09F092DE090093DF091093E009A7
:105140006623A1F50E9471390E94653FA5EAB9E086
:1051500080E090E0FC01EB5DF74F1082118212823B
:105160001382FC01EB51F74F1082118212821382DD
:105170001D920496803C910569F71092DD0910920A
:10518000DE091092DF091092E0099091BB0A80912C
:10519000B3028093BD0A8091A70281708295880F27
:1051A000880F807C977B982B9093BB0A7091BD0AE7
:1051B0007723E9F18091BB0A86FD39C06091C20A6C
:1051C00040E021E030E0072F10E02AC0842F90E07B
:1051D0000217130711F1DC0193E0B695A7959A9594
:1051E000E1F7542F5770FD01ED53F54F808190E0AA
:1051F000052E02C0959587950A94E2F780FF0DC0B1
:10520000A753B54F8C9190E002C0959587955A951C
:10521000E2F780FF02C061E006C04F5F2F5F3F4FA3
:105220004617A0F260E0872F81500E944D39C501DA
:10523000B4010E9463220E94653F8091E1098823A6
:1052400089F4C501B40123E030E040E050E00E9461
:10525000F3689B01AC0128593C4F81E0D9016C9166
:105260000E94F93CC501B4010E94FD22C501B401B0
:105270000E94CE23C501B4010E94E20BCF5ADF4F3A
:105280000FB6F894DEBF0FBECDBFCF91DF911F9157
:105290000F91FF90EF90DF90CF90BF90AF909F90D5
:1052A0008F907F906F905F904F903F902F900895D8
:1052B0008F929F92AF92BF92CF92DF92EF92FF9226
:1052C0000F931F93CF93DF937B018C01EA012CE3B3
:1052D00030E040E050E00E94F3686883C801B70105
:1052E0002CE330E040E050E00E94F368122F032FDF
:1052F000F42EE52E622F732F842F952F2CE330E0B0
:1053000040E050E00E94F3686983612F702F8F2D79
:105310009E2D2CE330E040E050E00E94F368122F15
:10532000032FF42EE52E622F732F842F952F28E163
:1053300030E040E050E00E94F3686A83612F702FF4
:105340008F2D9E2D28E130E040E050E00E94F36870
:1053500079018A01C801B7016C5F7F4F8F4F9F4F62
:1053600027E030E040E050E00E94F3686F5F6B831D
:1053700020E0AA24BB24650101C02F5F822E99245E
:10538000F401EE54F84FCF0183709070892B99F49B
:10539000CF0164E670E00E94E068892B39F4CF0108
:1053A00060E971E00E94E068892B29F48EE691E0C3
:1053B000A0E0B0E004C08DE691E0A0E0B0E0A80E6F
:1053C000B91ECA1EDB1EC501A0E0B0E0E816F90652
:1053D0000A071B0790F62E83F401EE54F84F83E082
:1053E000882E912C8E229F228114910499F4CF0152
:1053F00064E670E00E94E068892B39F4CF0160E92F
:1054000071E00E94E068892B29F48EE691E0A0E02B
:10541000B0E004C08DE691E0A0E0B0E0A81AB90ABF
:10542000CA0ADB0A980187010A191B092C093D09E0
:10543000CF0164E670E00E94E0687C01CF0160E982
:1054400071E00E94E068AC01EBE6F3E060E06130FF
:1054500051F48114910449F4E114F10441F441152B
:10546000510529F002C0808103C08CE101C08DE1AB
:1054700090E0A0E0B0E0081719072A073B0740F0CA
:10548000081B190B2A0B3B0B6F5F31966C30F9F63A
:105490006F5F6D83802F8F5F8C83DF91CF911F9122
:1054A0000F91FF90EF90DF90CF90BF90AF909F90C3
:1054B0008F900895EF92FF920F931F937B018C01C1
:1054C0008091040A9091050AA091060AB091070AFA
:1054D000E816F9060A071B0771F0C801B70149EF82
:1054E00059E00E945829E092040AF092050A0093BC
:1054F000060A1093070A1F910F91FF90EF900895ED
:105500000E945A2A8091FE0990E008950E945A2A2A
:105510008091FC0990E008950E945A2A8091FD092B
:1055200090E008950E945A2A8091FA0990E0089527
:105530000E945A2A8091FB0990E008954F925F9251
:105540006F927F928F929F92AF92BF92CF92DF9293
:10555000EF92FF920F931F93CF93DF934C01DC01E7
:1055600016961C91612F70E080E090E020E833E314
:1055700041EE51E00E94A1685B016C0122EB37E033
:10558000E12FF0E0EE54F84F1DC0C9018370907018
:10559000892BB1F4C90164E670E00E94E068892BB0
:1055A00039F4C90160E971E00E94E068892B41F497
:1055B00080E891E5A1E0B0E0A80EB91ECA1EDB1E8E
:1055C0002F5F3F4F2E173F0701F7D40115968C919F
:1055D000482E5524C90164E670E00E94E0687C0111
:1055E000C90160E971E00E94E0688C01C1E0D0E08F
:1055F00093E0692E712C6222732227C0C230D1053C
:1056000091F46114710479F4E114F10419F40115B1
:10561000110549F480E89BE3A6E2B0E0A80EB91EAC
:10562000CA1EDB1E11C0FE01E659FC4F608170E00E
:1056300080E090E020E831E541E050E00E94A16880
:10564000A60EB71EC81ED91E2196C415D505B4F2E4
:10565000D40112966C9170E080E090E020E13EE091
:1056600040E050E00E94A1687B018C01F40161815F
:1056700070E080E090E02CE330E040E050E00E94F9
:10568000A168E60EF71E081F191FD4018C91E80EC1
:10569000F11C011D111D14966C9170E06150704059
:1056A000882777FD8095982F20E831E541E050E08C
:1056B0000E94A168E60EF71E081F191FEA0CFB1CCA
:1056C0000C1D1D1DB701C801DF91CF911F910F91D6
:1056D000FF90EF90DF90CF90BF90AF909F908F9012
:1056E0007F906F905F904F90089560933F0270930A
:1056F0004002809341029093420208956093EF0923
:105700007093F0098093F1099093F20920913F0280
:10571000309140024091410250914202260F371FC2
:10572000481F591F2093F3093093F4094093F5095A
:105730005093F60982E090E09093F8098093F7097E
:105740000E94B6636093000A7093010A8093020A74
:105750009093030A0895EF92FF920F931F931CC03A
:105760002F5F3F4F4F4F5F4F2093EF093093F0096A
:105770004093F1095093F20988EE93E0A0E0B0E085
:10578000E80EF91E0A1F1B1FE092000AF092010AA0
:105790000093020A1093030A0E94B663E090000A85
:1057A000F090010A0091020A1091030A6E197F0914
:1057B000800B910B2091EF093091F0094091F10994
:1057C0005091F209685E73408040904048F68091A5
:1057D000F3099091F409A091F509B091F609281701
:1057E00039074A075B07E8F0E091ED09F091EE090F
:1057F0003097B9F00995611571058105910519F08A
:105800000E947E2B0EC020E030E08091F70990913D
:10581000F809892B11F021E030E03093F80920934A
:10582000F7096091EF097091F0098091F109909169
:10583000F2091F910F91FF90EF9008959093EE0958
:105840008093ED098091EF099091F009A091F10901
:10585000B091F2098093F3099093F409A093F509AC
:10586000B093F6090E94AB2B0895482F6AE00E947E
:10587000C068282F30E084E0220F331F8A95E1F7BB
:10588000842F0E94C068892F820F0895CF93DF93E1
:10589000EC018091080A9091090A8836910559F522
:1058A00088E79DE068E670E00E94AD5E88E79DE0D5
:1058B00060E00E942F5F88810E94352C682F70E085
:1058C0006F77707088E79DE00E942F5F89810E944A
:1058D000352C682F88E79DE00E942F5F8A810E9407
:1058E000352C682F88E79DE00E942F5F8B810E94F6
:1058F000352C682F2DC08F36910509F04AC088E7F6
:105900009DE06FE670E00E94AD5E88E79DE060E09C
:105910000E942F5F88810E94352C682F606888E77D
:105920009DE00E942F5F89810E94352C682F88E7B7
:105930009DE00E942F5F8A810E94352C682F88E7A6
:105940009DE00E942F5F8B810E94352C682F68603C
:1059500088E79DE00E942F5F8C810E94352C682F84
:1059600088E79DE00E942F5F8D810E94352C682F73
:1059700088E79DE00E942F5F8E818E510E94352C1A
:10598000682F88E79DE00E942F5F88E79DE00E94D6
:10599000725FDF91CF91089588E690E09093090AB5
:1059A0008093080A88E79DE068E670E00E94AD5E9B
:1059B00088E79DE060E00E942F5F88E79DE00E94FD
:1059C000725F8823D9F08FE690E09093090A809364
:1059D000080A88E79DE06FE670E00E94AD5E88E708
:1059E0009DE060E00E942F5F88E79DE00E94725F6B
:1059F000882321F01092090A1092080A08951F9333
:105A0000CF93DF93EC016091080A7091090A611548
:105A1000710509F46FC088E79DE00E94AD5E88E7DC
:105A20009DE060E00E942F5F88E79DE00E94725F2A
:105A30006091080A7091090A88E79DE047E050E00C
:105A40000E94835F88E79DE00E94C05E282F2F7729
:105A500022952F701AE0219F900111248F70820FE0
:105A6000888388E79DE00E94C05E282F22952F70D2
:105A7000219F900111248F70820F898388E79DE018
:105A80000E94C05E282F2F7322952F70219F9001B6
:105A900011248F70820F8A8388E79DE00E94C05E88
:105AA00087708B8388E79DE00E94C05E282F229537
:105AB0002F70219F900111248F70820F8C8388E7B3
:105AC0009DE00E94C05E282F22952F70219F90019B
:105AD00011248F70820F8D8388E79DE00E94C05E45
:105AE000282F2F70225E82958F70819FC001112414
:105AF000280F2E83DF91CF911F9108950F931F934D
:105B0000DF93CF93CDB7DEB727970FB6F894DEBFFC
:105B10000FBECDBF8E010F5F1F4FA8010E945829F5
:105B2000C8010E94462C27960FB6F894DEBF0FBE20
:105B3000CDBFCF91DF911F910F9108950F931F93C8
:105B4000DF93CF93CDB7DEB727970FB6F894DEBFBC
:105B50000FBECDBF8E010F5F1F4FC8010E94FF2CEB
:105B6000C8010E949E2A27960FB6F894DEBF0FBE8A
:105B7000CDBFCF91DF911F910F91089588E79DE0F0
:105B80000E94875F0895DF92EF92FF920F931F9319
:105B9000CF93DF93D82E862FBA01213041F4675F6F
:105BA0007F4F9B0140E050E0695070400EC02230B2
:105BB00029F020E030E040E050E007C06250704043
:105BC0009B0140E050E06E5F7F4FE82EFF2484EEA3
:105BD00093E0E80EF91E8B01E7010FC0F881E0E0C9
:105BE000898190E08E2B9F2BA0E0B0E0280F391F19
:105BF0004A1F5B1F2296025010400230110570F7B9
:105C0000CB018E7FD701A80FB91F6817790779F0EC
:105C10008C9190E0A0E0B0E0BA2FA92F982F8827B0
:105C200002C040E050E0280F391F4A1F5B1FCA0125
:105C3000AA27BB270097A105B10599F7C90180954F
:105C40009095ED2DF0E0EC51FC4F90838183DF9136
:105C5000CF911F910F91FF90EF90DF9008951092D8
:105C6000FC031092FD0380E48093F8031092F90383
:105C70008093FA0388E16EE044E150E020E00E9466
:105C8000C32D0895282F662321F0809109048617DB
:105C9000E1F480910A048823C1F480910B048833D5
:105CA000A1F4809107048B3781F4E22FF92F8091C2
:105CB0003604838380913704828380913804818302
:105CC00080913904808381E0089580E00895809177
:105CD0000A0A86958095817008958091810A809541
:105CE00090917D0A892B8093850A8091820A809504
:105CF00090917E0A892B8093860A8091830A8095F1
:105D000090917F0A892B8093870A8091840A8095DD
:105D10009091800A892B8093880A089590931F0A96
:105D200080931E0A7093290A6093280A5093210ACF
:105D30004093200A80E497E09093230A8093220AFC
:105D40001092250A1092240A3093270A2093260ADB
:105D500030914502209146028DEF94E39093120A10
:105D60008093110A8DE394E39093140A8093130AAD
:105D700020930D0A30930E0A81E080930B0A8091E4
:105D80000C0A8F5F877080930C0A80931D0A089518
:105D90000F931F93BC0104EE13E0C8010E94D93594
:105DA000C801069667E77AE00E94D9351F910F91E6
:105DB0000895EF92FF920F931F937B010E94C82ECC
:105DC00002E014E0C801B7010E94E135C801049760
:105DD0006DE77AE00E94E1351F910F91FF90EF90FF
:105DE0000895EF92FF920F931F93CF93DF937C015F
:105DF000EB018A0185E19AE00E94D92E8881807F9B
:105E0000803E49F088819981AA81BB818F5F9F4F35
:105E1000AF4FBF4F31F484EE93E067E773E00E9429
:105E2000D93588E08093F0031092F10382EF93E07C
:105E30006BE976E049E050E00E94D1071092F4034C
:105E400081E18093FB031093080400930904F0920E
:105E50000604E092070410920A0410920C041092B7
:105E60000D04DF91CF911F910F91FF90EF90089556
:105E7000EF92FF920F931F930AEE13E0C8010E9466
:105E8000C82E74E1E72EF12CE00EF11EC8014896F1
:105E9000B7010E94E135C7016DE77AE00E94E13564
:105EA0000E942F2E1F910F91FF90EF900895BC013B
:105EB00010929C0A10929B0A81E080930A0A89E85A
:105EC0009AE00E94E13508950F931F938C01889604
:105ED0009093F4038093F5030E942F2E10921604E2
:105EE00010921704045E1F4F82E36AE1A80122E0CA
:105EF0000E94C32DC8014A960E94E7471F910F9147
:105F00000895FF920F931F93CF93DF93EC01F62E2A
:105F1000042F10E080912A0A90912B0AA0912C0A5C
:105F2000B0912D0A2B2F33274427552720930A049D
:105F3000A0930B0490930C0480930D04F09213042F
:105F4000CE010E94642F1F5F011720F79E0140E0E1
:105F500050E080912A0A90912B0AA0912C0AB091CE
:105F60002D0A820F931FA41FB51F80932A0A9093B6
:105F70002B0AA0932C0AB0932D0ADF91CF911F9189
:105F80000F91FF900895CF93DF939C01862F80613E
:105F900080931304643029F02115310511F421E0B8
:105FA00030E0909108048091060480930804909357
:105FB000060490910904809107048093090490934A
:105FC0000704CDE0D4E08881A901480F511D2C8140
:105FD0004C832883252F3327219754E0C930D507D8
:105FE00091F71D861E8680E589871092F40388E26A
:105FF0008093F5030E94382F84E08B871C8682E310
:106000006AE14CE150E022E00E94C32D86E390E07B
:106010000E94E747DF91CF91089580911B0A9091EC
:106020001C0A60E00E94C32F80910A0490E0A0E067
:10603000B0E0BA2FA92F982F882720910B04820F48
:10604000911DA11DB11DBA2FA92F982F882720912E
:106050000C04820F911DA11DB11DBA2FA92F982FDD
:10606000882720910D04820F911DA11DB11D8093E1
:106070002A0A90932B0AA0932C0AB0932D0A089514
:10608000E82F4091080450E0292F30E042175307D1
:1060900009F092C0809109048E1709F08DC080919B
:1060A0001304E82F81FF4EC01092F4038CE280931A
:1060B000F5030E94382F82E1809313049091080425
:1060C000809106048093080490930604909109043B
:1060D000809107048093090490930704EDE0F4E0B5
:1060E00021E030E08081A901480F511D44831082D6
:1060F000252F3327319754E0E930F50799F71586B6
:1061000016861182128280914402838314828D5FED
:106110008093440282E0818B84E0828B95E0938BB4
:10612000148A80E68187938788E7848782E36AE11F
:1061300040E250E022E00E94C32D8AE390E00E94FA
:10614000E7473AC084FF38C09091F40380E0209183
:10615000F50330E0282B392B80911204482F50E0B2
:10616000A4E055954795AA95E1F7CA01880F991FB4
:10617000880F991F281B390B2451304037FF02C06C
:1061800020E030E030931C0A20931B0A232B69F097
:106190009A01220F331F220F331F2E5D3F4F68508D
:1061A00070406217730740F009C0E0FF05C080E04F
:1061B00090E060E00E94C32F20E030E0C901089524
:1061C0000F931F93DF93CF930F92CDB7DEB78C0160
:1061D000045E1F4F1093F4030C511040802F845E17
:1061E0008093F50389830E942F2E085F1F4F109321
:1061F0000A048981845180930B04085F1F4F88E251
:106200006AE1A80121E00E94C32DC8014A960E94BC
:10621000E7470F90CF91DF911F910F910895FF9263
:106220000F931F939C01F62E85E19AE0B9010E941D
:10623000D92E00EF13E088E08093F0031092F10371
:10624000C80102966BE976E049E050E00E94D10770
:106250008CE48093F50381E18093FB030E942F2E51
:10626000109208048BE7809309048AE08093060467
:10627000F092070410920A0488E380930B041092B2
:106280000C0410920D04025E1F4F80E3F80111927E
:106290008A95E9F7C80162E577E04AE050E00E949C
:1062A000D10788E26AE140E450E021E00E94C32D7A
:1062B0008AE590E00E94E7471F910F91FF900895B3
:1062C000EF92FF920F931F93BC0185E19AE00E9429
:1062D000D92E00EF13E088E0F82EF092F003109230
:1062E000F103C80102966BE976E049E050E00E94B4
:1062F000D10784E58093F503EE24E394E092FB0359
:106300000E942F2EF09206041092070410920804A7
:106310001092090485E080930A048091800A80939A
:106320000B0410920C04E0920D04C8014E9662E436
:1063300070E048E350E00E94F00784E262E240E44B
:1063400050E020E00E94C32D82E690E00E94E747E3
:106350001F910F91FF90EF900895DF92EF92FF92BF
:106360000F931F93CF93DF93EC018091990A8823B9
:1063700019F0CE010E94CF42209709F0BFC0809152
:106380000A0A8570F1F180919B0A90919C0A892BF1
:10639000C1F50E941F478823A1F187E793E00E947F
:1063A000C82E88E08093F003E6E0FE2EF092F10321
:1063B00082EF93E063E976E048E050E00E94D10785
:1063C00004E014E0D8011D92FA94E9F7C8010A9795
:1063D00067E77AE00E94D935C801069669E87AE055
:1063E0000E94E135C80104976DE77AE00E94E1352B
:1063F00080910A0A886080930A0A8AE290E00E94EB
:10640000E74780919B0A90919C0A019690939C0A81
:1064100080939B0A80910B0A813009F003C280911E
:106420000A0A81FFFFC102E000930B0A8091430238
:106430008F5F809343028F7110910C0A1295110F98
:10644000107E182BE0900D0AD0900E0A85E19AE09C
:1064500065E97AE00E94D92E78E0F72EF092F003F9
:106460001092F10382EF93E06BE976E049E050E0AF
:106470000E94D1078CE28093F50386E08093FB03B2
:106480000E942F2EE0920804D09209048BE08093A2
:10649000060410930704EAE0F4E0DF011D92FA9489
:1064A000E9F78091440280930C048D5F809344024D
:1064B00080E6809312040093130483E08093140415
:1064C00010921504109216041092170410921804DA
:1064D0001092190400931A0484E080931B04009323
:1064E0001C0486E280931D0482E36AE140E250E0EE
:1064F00022E00E94C32D8AE390E0AFC0C932D105EB
:1065000008F490C11091F003183009F096C1809101
:10651000F103863009F091C18AE094E06DE77AE0FA
:1065200044E050E00E94DA07009709F086C18091AC
:10653000F903813029F58AEE93E00E94C82E10926B
:10654000F80382E08093F90384E094E06AEF73E05B
:106550000E94D9358AEF93E067E77AE00E94D93547
:106560008AE094E060E074E00E94E13580E094E02D
:106570006DE77AE00E94E1358AE290E00E94E74709
:1065800080910A0A83FF4EC11091F903123009F07D
:1065900049C180E094E069E87AE044E050E00E947C
:1065A000DA07009709F03EC185E19AE06AEF73E0EF
:1065B0000E94D93510930A0A35C1183009F032C14A
:1065C0008091F103882309F02DC18091F203853475
:1065D00009F028C182E094E06DE77AE044E050E001
:1065E0000E94DA070097A9F082E094E065E87AE07B
:1065F00044E050E00E94DA07009759F082E094E00E
:1066000067E773E044E050E00E94DA07009709F082
:1066100009C18091FB03813019F58091060488300F
:10662000F9F4E0910F0AF091100A309719F08EEF0B
:1066300093E009950E94382F109206048091080477
:10664000883F28F0809109048F5F8093090480912E
:106650000804885F80930804CE010E94E747E2C0E7
:106660000E94ED35882351F08091FB03813131F494
:10667000CE010E94F235882309F0D4C0C633D1057B
:1066800028F48091FB03863009F0CCC08091080487
:106690008B3009F0BEC08EEF93E065E97AE044E00C
:1066A00050E00E94DA07009709F0BCC08091130403
:1066B000382F82FF13C0E091110AF091120A30972F
:1066C00059F08091090482958695877063E040E0D7
:1066D00050E020E030E0099585E090C09091F4030F
:1066E00080E02091F503022F10E0082B192B8091F8
:1066F0001204482F50E064E0559547956A95E1F7FC
:10670000CA01880F991F880F991F081B190B045184
:10671000104017FF02C000E010E080910B0A8230A9
:1067200079F531FF21C034FF1FC080E090E060E0C8
:106730000E94C32F88E180931304E091130AF09123
:10674000140A309719F420E030E007C08091070464
:1067500082958695877009959C0183E080930B0A4A
:10676000C9010E94642F5EC081E080930B0A34FF50
:1067700003C080E090E002C0C801019664E046C01A
:10678000833081F50115110579F1E091110AF0913D
:10679000120A309749F1440F551F440F551FCE017F
:1067A00008974E5D5F4F8417950708F4AC01C80148
:1067B000840F951FC817D90710F0980103C09E01D8
:1067C000241B350B8091090482958695877060E0C3
:1067D000099580919A0A882319F0C80168E016C0CB
:1067E000C80108C08530F1F030FF0BC08330D1F014
:1067F000C801019669E00E94C32F86E080930B0ACE
:1068000011C00115110571F0C80160E00E94C32F8D
:1068100009C08091450290914602BE010E9440301D
:106820009C0102C020E030E0C901DF91CF911F91AF
:106830000F91FF90EF90DF900895CA32D10508F0D4
:10684000BCCEF0CFBC018091FB038130A1F48091DC
:106850000604882381F480910E04823461F48EEF63
:1068600093E044E050E00E94DA079C0180E0232B93
:1068700019F481E0089580E00895CF92DF92EF92BD
:10688000FF920F931F93DF93CF93CDB7DEB7289777
:106890000FB6F894DEBF0FBECDBF2AE134E03E83D1
:1068A0002D8338872F8390911D0A891709F08FC097
:1068B0001C821B8285E593E09A8389834091240A98
:1068C0005091250A41155105A9F58DB79EB70C9732
:1068D0000FB6F8949EBF0FBE8DBFEDB7FEB73196D1
:1068E000CE010196ADB7BEB712969C938E931197C9
:1068F0008CE197E09383828380911E0A90911F0A16
:10690000958384838091280A9091290A97838683AE
:106910008091200A9091210A918780878091220A94
:106920009091230A938782870E94B2368DB79EB7D3
:106930000C9648C02091220A3091230AE0901E0A4A
:10694000F0901F0A0091200A1091210A21153105AB
:1069500019F065EB71E004C068EB71E024EA36E001
:10696000DA010D900020E9F76D010894C108D10803
:10697000C41AD50A8DB79EB740970FB6F8949EBF3C
:106980000FBE8DBFEDB7FEB73196CE010196ADB704
:10699000BEB712969C938E93119785EA96E09383E7
:1069A0008283F582E4821783068331872087738789
:1069B0006287D586C486578746870E94B2368DB7D0
:1069C0009EB740960FB6F8949EBF0FBE8DBF2F8125
:1069D00038858D819E81281B390BC90128960FB6F9
:1069E000F894DEBF0FBECDBFCF91DF911F910F9105
:1069F000FF90EF90DF90CF9008950F931F93CF9368
:106A0000DF93890190911D0A891759F0E091260AB8
:106A1000F091270A84E060E070E040E050E00995E2
:106A20002AC0662341F52D30310528F1C091260A90
:106A3000D091270A2097F9F043515C4F89EB91E000
:106A4000BA0143E050E00E9409089C0180E0232B3A
:106A500009F081E06091120470E0B4E075956795EB
:106A6000BA95E1F7660F771F660F771F6E5D7F4F50
:106A7000A801FE01099580E0DF91CF911F910F9150
:106A800008950F931F93CF93DF93DC01EB01722FD7
:106A9000532F822F932F9C01F90160E016C0808153
:106AA000981771F431968081882371F411968C9136
:106AB0008D3331F4872F952F9C01F90161E004C0DB
:106AC000872F952F9C01F90111969C91992339F0FC
:106AD000903229F09A3019F0662309F304C061302E
:106AE00011F030E018C07A2F50E04150504002C001
:106AF000299311963A2F371B2C91222359F02032DB
:106B000049F02A3039F0263229F0832F90E084179B
:106B1000950774F318820115110511F0F8016083CF
:106B2000832FDF91CF911F910F910895CF93DF9322
:106B3000FC01EC0137C08B3211F480E231C08532A8
:106B400079F5DF0111969181392F30533A3070F089
:106B5000892F8156863010F4375208C0892F81540E
:106B6000863010F030E002C0392F3753FD013196E6
:106B700011962C91922F90539A3070F0822F81565B
:106B8000863010F4975208C0822F8154863010F05E
:106B900090E002C0922F9753832F8295807F892B9C
:106BA000899331968081882331F61882DF91CF91C5
:106BB0000895DC01FB0186E001900D928150E1F720
:106BC00008959C01FB0180819181A281B381F9012B
:106BD00080839183A283B38308958091560A8111A3
:106BE00081E00895CF92DF92EF92FF920F931F936F
:106BF000CF93DF93CEE2DAE030E0CC24DD2429C06D
:106C00002A814B818091080490E0042F10E08017C6
:106C10009107D9F4909109049217B9F48C818823D3
:106C2000A1F020910B0430E028503040F0900A048D
:106C3000EE242E0D3F1DE881F981892F942F6EEFF0
:106C400073E04EE054E0099531E00894C11CD11C7A
:106C500025968091560A90E0C816D9068CF2832FAB
:106C6000DF91CF911F910F91FF90EF90DF90CF9028
:106C70000895EF92FF920F931F93CF93DF93FC0140
:106C8000EB018A0179011092990A009729F08DE7AA
:106C90009AE0BF010E94E135209719F0CE010E94D1
:106CA000572F0115110529F081E99AE0B8010E94DA
:106CB000E135E114F10429F081E89AE0B7010E947E
:106CC000E1350E946D2E10929C0A10929B0A81E081
:106CD000DF91CF911F910F91FF90EF900895AF92A8
:106CE000BF92CF92DF92FF920F931F93CF93DF93C8
:106CF0008C01EB01F42E1092990A38E341E050E048
:106D000060E070E018C0832F90E0FC01B3E0F595DF
:106D1000E795BA95E1F7E95AF54F877090705A01F7
:106D20006B0104C0AA0CBB1CCC1CDD1C8A95D2F7DD
:106D300020812A292083315031F787E79AE0BE016C
:106D40000E94D935C80167E77AE04F2D0E94434879
:106D5000DF91CF911F910F91FF90DF90CF90BF9067
:106D6000AF900895CF92DF92EF92FF920F931F930F
:106D7000DF93CF93CDB7DEB7EB84FC84CD84DE8484
:106D8000DE011F9601C0D801F6018491882309F421
:106D9000BCC00894C11CD11C843209F099C0F60112
:106DA0000894C11CD11C8491863409F45FC08734D7
:106DB00034F4843469F0853409F08AC06EC08C34B0
:106DC000C9F1833509F445C0883409F081C00DC08C
:106DD0008D010E5F1F4FF701668177818D919C9128
:106DE0004AE050E00E945E087EC02C91822F9927D5
:106DF00087FD909514E0959587951A95E1F78F702A
:106E00002F702A300CF0295F8A300CF0895F8D01D9
:106E10000E5F1F4FF701A681B781805DFD01819351
:106E2000205D11962C933196D7011796FC93EE9323
:106E30001697A9CF8D010C5F1F4F6D917D918D919C
:106E40009C91F701468157812AE030E00E949C081E
:106E50004AC08D010E5F1F4F6D917C91D701169630
:106E60008D919C9117970E9402083DC08D010E5F85
:106E70001F4F2D913C910AC0D7011696ED91FC91C0
:106E8000179781931796FC93EE931697F9012F5F4E
:106E90003F4F8491882381F776CF8D010E5F1F4F7E
:106EA0002D913C910AC0D7011696ED91FC91179750
:106EB00081931796FC93EE931697F999FECF32BD06
:106EC00021BDF89A80B52F5F3F4F882361F75BCFD4
:106ED000F70126813781F90181939F01F7013783FB
:106EE00026838D0150CFD70116968D919C911797CF
:106EF000FC0101900020E9F73197E81BF90B8E0F98
:106F00009F1FF701978386833ECFCF91DF911F911B
:106F10000F91FF90EF90DF90CF900895FF920F9325
:106F20001F93CF93DF938C01F62E0E94B663EB0183
:106F30000CC00E945E470E94AD310E94B6636C1B7C
:106F40007D0B6053754708F0EFC00E941F478823F0
:106F500081F30E94B663EB010CC00E945E470E9461
:106F6000AD310E94B6636C1B7D0B6053754708F012
:106F7000DBC00E94672E882381F71092950A109239
:106F8000960A1092970A1092980A80919D0A8F5F34
:106F900080939D0A8091910A882361F488E098E0AB
:106FA000A8E0B8E08093910A9093920AA093930A84
:106FB000B093940A80919D0A90E0906E61E97AE026
:106FC00045E350E00E94F12EEEE0F4E08CE0DF01BA
:106FD0001D928A95E9F7DF011C9690E0FF2019F0D9
:106FE000F801808102C0F80184910F5F1F4F8E323B
:106FF00041F0882331F09F5FFD01E90FF11D80838F
:10700000EDCFFD019193DF01A90FB11D882329F771
:10701000FD01119211961C92DF01119641E041830E
:10702000FD01319611961C92418386ED24EE33E0EA
:10703000821B32968E0F80930E0490919D0A90933E
:107040000F04409310044093130490E00E94E0303A
:107050000E94B6638B0161C00E94B663601B710B16
:107060006053754708F060C00E945E47EC010097CE
:1070700009F453C00E94AD31892B09F04EC0C634CB
:10708000D10508F44AC080910704853309F045C052
:1070900080910804803E09F040C0909109048091DD
:1070A0009D0A9817D1F580910F048917B1F5809149
:1070B000110490E08F709070892BB1F580910E04CF
:1070C000E82FF0E0E25FFB4F9E012C513C4F8081A6
:1070D000807C39F0329609C08081882311F4319682
:1070E00004C03196E217F307B8F3CF010E962817C4
:1070F000390798F08181813051F48185843039F4E9
:107100003A9685E99AE0BF010E94E13506C0818583
:1071100090E00A96E80FF91FDACF8091950A88234C
:1071200009F49ACF81E001C080E0DF91CF911F91F7
:107130000F91FF9008959C01F999FECF32BD21BDBA
:10714000F89A80B508959C01F999FECF1FBA32BD17
:1071500021BD60BD0FB6F894FA9AF99A0FBE089552
:10716000E091FD0AF091FE0A09950895FB0190E077
:1071700024E0880F991F2A95E1F7108A9C012C556D
:107180003B4FAC014C545B4FF999FECF32BD21BD52
:10719000F89A80B58083882331F02F5F3F4F319676
:1071A0002417350789F70895FB0190E034E0880F34
:1071B000991F3A95E1F7108A9C012C553B4F8C544E
:1071C0009B4F4081F999FECF1FBA32BD21BD40BD12
:1071D0000FB6F894FA9AF99A0FBE442331F031961B
:1071E0002F5F3F4F2817390761F70895AC01FB0166
:1071F0000FC0F999FECF1FBADA01A80FB11DB2BDB9
:10720000A1BD20BD0FB6F894FA9AF99A0FBE319637
:107210008E2F861B2081222361F7F999FECF1FBA9A
:10722000480F511D52BD41BD10BC0FB6F894FA9ADB
:10723000F99A0FBE0895FC0184EF93E0F999FECF0F
:1072400092BD81BDF89A30B52081332339F02223D5
:1072500051F00196321739F43196F0CF80E02223B5
:1072600019F481E0089580E00895FC01CB01F999BB
:10727000FECF92BD81BDF89A30B52081332349F00D
:10728000222339F00196321711F081E008953196EA
:10729000EECF80E0321381E00895282F2770869585
:1072A0008695869590E0662369F0FC01ED53F54FD5
:1072B00081E090E002C0880F991F2A95E2F72081B3
:1072C000282B0DC0FC01ED53F54F81E090E002C08A
:1072D000880F991F2A95E2F7809520812823208323
:1072E00008951092C30A1092C40A1092C50A10920F
:1072F000C60A1092C70A1092C80A0895E7E4F2E09D
:107300002CEB37E0F999FECF32BD21BDF89A80B55C
:1073100080832F5F3F4F369687E0213E380791F7F5
:107320008091A1028F5F8093C10A90E043E0880FB3
:10733000991F4A95E1F78093C20A9091D702917004
:107340008091BB0A8E7F892B8093BB0A0895EFE161
:10735000F3E080EE97E02081F999FECF1FBA92BD4D
:1073600081BD20BD0FB6F894FA9AF99A0FBE3697F0
:10737000019722E0E134F20771F78091A1028F5F5B
:107380008093C10A90E053E0880F991F5A95E1F766
:107390008093C20A9091D70291708091BB0A8E7F30
:1073A000892B8093BB0A08958091BB0A81608093EA
:1073B000BB0A81E08093D7020E94A739089580918B
:1073C000BB0A8E7F8093BB0A1092D7020E94A73916
:1073D00008958C33910510F4682F15C02AE280338C
:1073E000920730F46CE370E00E94CC68655C0BC0DF
:1073F0002DEF8032920710F06EEF05C060E17EE065
:107400000E94CC686451862F0895282F30E08C3379
:10741000D8F08F3E68F48CE390E0A901489F90017A
:10742000499F300D589F300D1124245D3D400CC004
:1074300080E19EE0A901489F9001499F300D589F2F
:10744000300D1124205C364FC90108951092A10A15
:107450001092A00A87EA93E090939F0A80939E0A75
:107460000895EF92FF920F931F93CF93DF93E82E2F
:10747000162F042FF22E662321F0623081F422238E
:1074800071F08E2D0E940F63892B11F000E024C053
:10749000FF2011F480E001C080E8082B1DC0C0E08F
:1074A000D0E08E2D0E940F63892B81F4113031F0D2
:1074B000123061F484E0C03BD80744F461E070E02E
:1074C00080E090E00E94C4632196EBCFFF2019F486
:1074D000C05BD4400CF00068802FDF91CF911F91EA
:1074E0000F91FF90EF9008950F931F93082F109125
:1074F000FF0A107861E070E080E090E00E94C463D1
:107500008FE10E940F63892B21F48FE1602F41E00E
:1075100013C08EE10E940F63892B21F48EE1602F4E
:1075200042E00AC08DE10E940F63892B11F040E018
:1075300007C08DE1602F44E0212F0E94313A482F8F
:107540008091FF0A90E08F709070242F30E0892B9B
:1075500039F42F703070232B71F0842F806406C0B3
:107560002F703070232B39F4842F80624093FF0AF0
:107570001F910F910895842FF9CF8BE00E940F6324
:1075800040E02091CB0230E08217930709F041E000
:10759000440F440F8091BB0A8B7F842B8093BB0ADE
:1075A0000895EF92FF920F931F938C016EE9E62EE0
:1075B0006AE0F62E6AE070E00E94E068C7014AE0E7
:1075C00050E00E94E466C8016AE070E00E94E06852
:1075D000BC01C7014AE050E00E94E4661F910F9190
:1075E000FF90EF900895CF93DF93EC0104C08EE9F4
:1075F0009AE00E940466FE01219664916623B9F721
:10760000DF91CF9108950F931F93CF93DF938C0158
:10761000462F8EE99AE060E00E948445E80104C0AC
:107620008EE99AE00E9404669E01201B822FFE01D3
:10763000219664916623A1F7992787FD9095C0E173
:10764000D0E0C81BD90B05C08BE19AE00E94F33A49
:107650002197D7FFF9CFDF91CF911F910F91089517
:107660000F931F93CF93DF938C01FC01EE0FFF1F4D
:10767000E00FF11FEE0FFF1FE75BFD4F808191814F
:1076800060E00E94033B84EF99E061E00E94033BCD
:107690008EE99AE060E041E00E94844503311105E3
:1076A00009F465C0043111056CF40C30110509F4BE
:1076B00073C00131110509F480C00130110509F0D2
:1076C000C0C015C00B31110509F49FC00C31110564
:1076D0002CF40431110509F0B4C050C00C3111056F
:1076E00009F49CC00E31110509F0ABC05DC080915A
:1076F0004D02C82FD0E0E097D7FD05C082EF99E09A
:107700000E94F33A07C080EF99E00E94F33AD095C7
:10771000C195DF4FCE0164E070E00E94E0688EE921
:107720009AE04AE050E00E94E4668EEE99E00E9402
:10773000F33ACE0164E070E00E94E068BC01B4E07E
:10774000660F771FBA95E1F7681B790B29F48BEE6A
:1077500099E00E94F33A06C08EE99AE04AE050E0D0
:107760000E94E46686EE99E00E94F33A8EC084EEB1
:1077700099E00E94F33A6091B9025BC08091BF0228
:107780008C3320F082EE99E00E94F33A6091BF02C0
:1077900070E06C5370400EC07091950260E0809173
:1077A0008F02680F711D06C06091FB028AE0689F1E
:1077B000B00111248EE99AE03FC08091AD02682F9C
:1077C00070E08C33D8F08F3E68F48CE390E09B013E
:1077D000289FB001299F700D389F700D1124645DA2
:1077E0007D400CC080E19EE09B01289FB001299F55
:1077F000700D389F700D1124605C764F8EE99AE011
:107800004AE050E00E94936640C06091E9028DE03A
:1078100070E00E941C626091E9020BC08091EF024F
:107820006FEF70E0681B71098CE00E941C62609130
:10783000EF028EE99AE070E04AE050E00E94E466D0
:1078400024C0F801EE0FFF1FE00FF11FEE0FFF1F26
:10785000E95BFD4F81816081813051F4662319F429
:107860008BED99E002C08EED99E00E94F33A07C0DB
:107870008EE99AE070E04AE050E00E94E466073149
:10788000110519F489ED99E012C0C80143970297D8
:1078900018F484ED99E00BC00131110519F48FEC57
:1078A00099E005C00E31110521F48BEC99E00E949E
:1078B000F33ADF91CF911F910F910895EF92FF92CC
:1078C0000F931F93182F092F0E94303B212F302F29
:1078D000C9018C016AEAE62E82E00E94743A482FC0
:1078E00050E09A012F70307022303105E1F02430E1
:1078F000310569F12130310509F068C00115110524
:1079000009F467C0F801EE0FFF1FE00FF11FEE0F43
:10791000FF1FE95BFD4F90818181891709F459C0F0
:107920009F5F908356C00115110509F44FC0F801FF
:10793000EE0FFF1FE00FF11FEE0FFF1FE95BFD4F82
:107940009081992309F442C0915090833FC086FFF3
:107950003DC087FF0BC080911F03882311F0E09288
:107960001F030E94A739FF24F39434C0033011058C
:1079700041F480915902882309F1FF240CE010E0C2
:1079800029C00C30110521F4FF240EE010E022C0C4
:107990000531110541F48091C502882379F4FF2453
:1079A00007E110E017C00231110541F48091B302E4
:1079B000882321F4FF2405E110E00CC0C8010196E2
:1079C00065E270E00E94E0688C0103C0882309F43E
:1079D00083CFFF24C8010E94303BFF2009F47CCFF5
:1079E0008EE99AE00E9472451F910F91FF90EF90EF
:1079F00008950F931F93CF93DF93482F062F8EE99F
:107A00009AE060E00E9484458091BC0A8F7019F46E
:107A10008AE09AE010C088E09AE00E94F33A609110
:107A2000BC0A6F708EE99AE070E04AE050E00E9474
:107A3000E46686E09AE00E94F33A8091BB0A80FDFA
:107A400006C08AEF99E061E00E94033B26C0E09106
:107A5000BC0AEF70F0E0ED53F54F1081C1E0D0E0CB
:107A60008091BC0A8F7051F48091B30290E0C817E6
:107A7000D90721F410FD06C06DE405C010FD02C059
:107A80006FE501C0602F8EE99AE00E94046621969E
:107A9000C930D10511F01695E3CF85EF99E00E942A
:107AA000F33A8EE99AE06DE041E00E9484458091CE
:107AB000BB0A81FD06C082FF09C08091C5028823F0
:107AC00029F08EE99AE063E00E9440458EE99AE051
:107AD0006EE041E00E9484458091BB0A85FF05C0AD
:107AE0008EE99AE062E00E9440458EE99AE06FE0FC
:107AF00041E00E94844560E08091BC0A82958F70CD
:107B000090E003970CF061E08EE99AE00E94404516
:107B1000DF91CF911F910F910895EF92FF920F93F4
:107B20001F93CF93DF938C017B018EE99AE00E9433
:107B3000B3458EE99AE060E040E00E948445C0E0F1
:107B4000D0E0F801EC0FFD1F60818EE99AE070E053
:107B50004AE050E00E94E46680E19AE00E94F33A35
:107B60002196C330D10569F7F80163818EE99AE067
:107B700070E04AE050E00E94E4668EE99AE060E03E
:107B800041E00E9484458EE09AE00E94F33A8EE93B
:107B90009AE0B7014AE050E00E94E466DF91CF919D
:107BA0001F910F91FF90EF90089584E00E94FA6179
:107BB0009C0183E02E3B380710F080E0089583E0BD
:107BC0002734380710F081E0089582E02B3E380713
:107BD00010F082E0089582E0223A380710F083E046
:107BE000089582E02536380710F084E00895235385
:107BF000324010F085E008958FEF089588EE93E00D
:107C000063EB7AE048E050E023EA38E30E94420860
:107C100008958091BB0A8D7F8093BB0A1092B70AAA
:107C20001092B80A1092B90A1092BA0A0E94FE3D48
:107C300008958091BB0A82608093BB0A0E94FE3D3A
:107C4000089546E050E023EA38E30E944208089590
:107C500083EB9AE068EE73E048E050E02BE938E30C
:107C60000E942608AEEBBAE0EBEBFAE083E001906D
:107C70000D928150E1F708959C01CB01B90146E0D6
:107C800050E02BE938E30E942608089564EF71E084
:107C900080E090E00E94C463F999FECF8CEB97E0FE
:107CA00092BD81BDF89A80B5823D59F4F999FECF15
:107CB00080EE97E092BD81BDF89A80B58A3A09F0CE
:107CC00096C08DE59AE060E00E94033B8EE49AE066
:107CD00061E00E94033B80E090E0F999FECF1FBA7B
:107CE00092BD81BD10BC0FB6F894FA9AF99A0FBEF6
:107CF000019628E08030920781F70E94FE3D84EFD4
:107D000093E06DEB71E00E94F63884E194E066EC5C
:107D100071E00E94F63884E494E060ED71E00E9426
:107D2000F63884E894E06FEE71E00E94F63824EAB9
:107D300034E0E1E0F0E043E5F999FECF1FBA32BD4F
:107D400021BD40BD0FB6F894FA9AF99A0FBEF99981
:107D5000FECF1FBA2F5F3F4F32BD21BD21503040B3
:107D6000CF016AE070E00E94E068605D60BD0FB620
:107D7000F894FA9AF99A0FBEF999FECF1FBA2E5FBE
:107D80003F4F32BD21BDCF016AE070E00E94E06844
:107D9000805D80BD0FB6F894FA9AF99A0FBE225F03
:107DA0003F4F87E0243A380711F03196C5CF8FEF67
:107DB000F999FECF1FBA32BD21BD80BD0FB6F89430
:107DC000FA9AF99A0FBE2F5F3F4F97E02A3A390788
:107DD00079F70E94A73964EF71E080E090E00E949B
:107DE000C463E091FD0AF091FE0A09951CC00E944F
:107DF0007E3984EA97E069EC7AE00E943C3E8AEAA8
:107E000097E06FEC7AE00E943C3E80EB97E065EDF6
:107E10007AE00E943C3E86EB97E06BED7AE00E94B0
:107E20003C3E0E94283E80E00E94743A90E08F70B1
:107E300090708130910519F0049779F503C084E2C0
:107E400090E020C08EE39AE060E00E94033B60ED8A
:107E500077E080E090E00E94C4638DE29AE060E009
:107E60000E94033B8DE19AE061E00E94033B80E0C9
:107E70000E94743A86FFFBCF8EE99AE00E94B345D8
:107E800080E090E00E945E3C80911F03882329F0EF
:107E9000E091FD0AF091FE0A09958CE061E00E94F4
:107EA0007C628DE061E00E947C626091E9028DE07D
:107EB00070E00E941C628091EF026FEF70E0681B1F
:107EC00071098CE00E941C620895EF92FF920F935B
:107ED0001F93CF93DF9383E060E00E94BB6208ECC6
:107EE0001AE08091BB0A80FD02C060E002C0F80188
:107EF0006081C7E0D0E0E62EFF2486E160E00E94CA
:107F0000BB62B7010C2E02C0759567950A94E2F723
:107F1000617085E10E94BB6286E161E00E94BB6204
:107F20002197FFEFCF3FDF0741F7015010408AE074
:107F3000023C1807B1F683E061E00E94BB62DF916A
:107F4000CF911F910F91FF90EF900895DF93CF9302
:107F5000CDB7DEB727970FB6F894DEBF0FBECDBF03
:107F6000CE0101960E94FF2C8C8190E0059667E07F
:107F700070E00E94E06827960FB6F894DEBF0FBE4F
:107F8000CDBFCF91DF910895DF92EF92FF920F93D3
:107F90001F93D82E0E94AB2B7B018C018EE99AE0B7
:107FA00060E04D2D0E948445C801B7010E94982AC7
:107FB0000E94D13A89E19AE00E94F33AC801B701E0
:107FC0000E94922A0E94D13A86E19AE00E94F33AF6
:107FD0000E94A63FE82FF0E0EE0FFF1FEB5DFC4F85
:107FE000808191810E94F33A84E19AE00E94F33A01
:107FF000C801B7010E94802A0E94D13A82E19AE02A
:108000000E94F33AC801B7010E948C2A0E94D13A1B
:108010001F910F91FF90EF90DF9008958F92AF9294
:10802000CF92EF920F931F93DF93CF93CDB7DEB72D
:10803000A0970FB6F894DEBF0FBECDBF81E061E020
:108040000E947C6281E061E00E94BB6283E061E0AB
:108050000E947C6283E061E00E94BB6286E161E095
:108060000E947C6285E161E00E947C621092C30AFA
:108070001092C40A1092C50A1092C60A1092C70A3A
:108080001092C80A0E94653F81E060E00E94BB62D6
:1080900080E061E00E947C6280E061E00E94BB625F
:1080A00081E0809381008CE061E00E947C628DE041
:1080B00061E00E947C626091E9028DE070E00E94C4
:1080C0001C628091EF026FEF70E0681B71098CE019
:1080D0000E941C6200D000D0EDB7FEB73196ADB75C
:1080E000BEB711961C921182128213828EE99AE019
:1080F00061E043E12FEF02E1B4E1EB2EA5E1CA2EEE
:10810000F6E1AF2EE7E18E2E0E942A460F900F90E7
:108110000F900F908EE99AE060E142E020E00E942B
:10812000BB458BE060E00E947C628BE061E00E94D6
:10813000BB6288E79DE00E94875F8091BB0A8164F3
:108140008093BB0AAEEBBAE0EBEBFAE083E0019080
:108150000D928150E1F788E691E09093B40A809304
:10816000B30A88E394E09093B60A8093B50A81E05D
:108170008093C10A88E08093C20ADE011196E5E986
:10818000F3E001900D928150E1F7DE011996EDE8E0
:10819000F3E088E001900D928150E1F7DE01519605
:1081A000E5E8F3E088E001900D928150E1F7DE010F
:1081B0005996EDE7F3E088E001900D928150E1F7E8
:1081C0008EE99AE061E08E010F5F1F4FA8010E94C7
:1081D0004A451A821B8281E08C838EE99AE060E036
:1081E000A8010E944A458EE99AE062E0AE01475F2D
:1081F0005F4F0E944A458EE99AE063E0AE014F5E10
:108200005F4F0E944A458EE99AE064E0AE01475E06
:108210005F4F0E944A458CE161E00E947C628CE1E4
:1082200060E00E94BB628EE061E00E947C628EE0B2
:1082300060E00E94BB628FE160E00E947C628EE1A0
:1082400060E00E947C628DE160E00E947C628FE1D0
:1082500061E00E94BB628EE161E00E94BB628DE141
:1082600061E00E94BB620E94CC2C882329F480919B
:10827000BB0A80618093BB0AA0960FB6F894DEBF5C
:108280000FBECDBFCF91DF911F910F91EF90CF9097
:10829000AF908F900895DF93CF93CDB7DEB7289737
:1082A0000FB6F894DEBF0FBECDBF8EE69AE061E058
:1082B0000E94033B0E94AB2B6093F50A7093F60A71
:1082C0008093F70A9093F80A6093F90A7093FA0A78
:1082D0008093FB0A9093FC0A8091E3028093380319
:1082E00084E893E063E373E044E00E946F36882300
:1082F00011F490E03AC09091950280E020918F02B5
:10830000820F911D909346028093450280915902FD
:10831000882319F00E944F4422C080915F02898314
:10832000809165028A8380916B028B8380917102B8
:108330008C83809177028D8380917D028E838091E2
:1083400083028F83809189028887AE014B5F5F4FE4
:10835000CE010196BA0120E030E00E94393690E06B
:10836000882309F491E081E09827892F28960FB699
:10837000F894DEBF0FBECDBFCF91DF910895DF939C
:10838000CF9300D000D000D0CDB7DEB7DE0111967C
:10839000EDE9F3E086E001900D928150E1F786E18E
:1083A00091E0E4EEF3E0DF019C011D9221503040AA
:1083B000E1F78091000B833019F46DE87AE003C097
:1083C000BE016F5F7F4F84E490E043E450E00E9481
:1083D000F12E8091000B833039F084EE93E0BE01E2
:1083E0006F5F7F4F0E94D93581E080930E048093A8
:1083F0000F0486E08093100480910D0B90910E0B7A
:10840000A0910F0BB091100B809312049093130462
:10841000A0931404B09315048091000B833039F4B9
:108420008EE094E00C966DE77AE00E94E1358AE2F6
:1084300094E067E77AE00E94D935AAEFB4E0EAE475
:10844000F3E002C081918D9333E0E035F307D1F77B
:108450009091000B992311F083E001C081E080939B
:1084600000058DE38093010587E08093020581E09C
:1084700080930305A4E0B5E0E7E7FAE002C081914C
:108480008D938AE0ED37F807D1F78CE080930A05E9
:1084900080E180930B05E9E3F3E0ACE0B5E002C0D6
:1084A00081918D9323E0E934F207D1F72CE135E097
:1084B0003093150B2093140B913069F582E3809370
:1084C0001C0584E080931D05D9011296EDE7FAE0C2
:1084D00002C081918D933AE0E138F307D1F786E34A
:1084E0008093220584E08093230584E295E09093B5
:1084F000150B8093140BDC01EDE8FAE002C08191CA
:108500008D938AE0E139F807D1F788E295E09093FE
:10851000150B8093140B2091130B222311F094E080
:1085200001C093E0A091140BB091150BFD0187E3FE
:10853000819311969C93DF01119681E08183FD0167
:10854000319683E011968C93DF01119686E081834A
:10855000CD0101969093150B8093140B222339F0D3
:1085600011962C9301969093150B8093140BE09128
:10857000140BF091150B8FEF8193F093150BE09393
:10858000140BCF018E5094400E94E03026960FB617
:10859000F894DEBF0FBECDBFCF91DF910895EF926B
:1085A000FF920F931F93CF93DF938C018091000B69
:1085B000823009F4F8C0833030F4882351F18130DF
:1085C00009F066C14BC0833021F0843009F060C1EE
:1085D000EAC00E94B6632091050B3091060B4091D2
:1085E000070B5091080BE090010BF090020B0091EB
:1085F000030B1091040B2E0D3F1D401F511F6217DE
:1086000073078407950708F443C10E94BF4184E0C3
:1086100018C00E94B66360930D0B70930E0B80938D
:108620000F0B9093100B10927D0A10927E0A1092FD
:108630007F0A1092800A0E94BF4181E00E940E478B
:1086400081E08093000B0E94B6636093090B7093E6
:108650000A0B80930B0B90930C0B1AC10634110577
:1086600008F4D5C080910704833409F0D0C020916C
:108670001204309113044091140450911504809118
:108680000D0B90910E0BA0910F0BB091100B2817B2
:1086900039074A075B0709F0BAC0CEEFD4E0FE0104
:1086A000A8014C515C4FDF01119691819D012F5F14
:1086B0003F4F8081853329F411968C91823009F4E3
:1086C000C5C0F901E90FF11DE417F50760F39FC07C
:1086D000FE019191E980EF0121969333D9F0943313
:1086E00040F4933089F0963091F0913009F046C013
:1086F00008C09A3379F09F3F09F451C09633F1F5E1
:1087000037C081E89AE036C089E89AE033C081E951
:108710009AE030C0618170E080E090E0982F872F70
:10872000762F66272981620F711D811D911D982F5B
:10873000872F762F66272A81620F711D811D911D5B
:10874000982F872F762F66272B81620F711D811D31
:10875000911D28EE33E040E050E00E94A168609354
:10876000050B7093060B8093070B9093080B89C041
:108770008DE89AE0BE010E94E13583C0E091110BC3
:10878000F091120B309709F47CC08091130B98176D
:1087900009F077C0892FBE014E2D099572C00E9445
:1087A000BF4182E04ECF0634110588F18091070465
:1087B000833469F52091120430911304409114041C
:1087C0005091150480910D0B90910E0BA0910F0B01
:1087D000B091100B281739074A075B07C1F4EEEF79
:1087E000F4E0A8014C515C4FDF01119691819D018D
:1087F0002F5F3F4F8081853321F411968C91853016
:1088000071F1F901E90FF11DE417F50768F30E9412
:10881000B6632091090B30910A0B40910B0B5091DC
:108820000C0B205F384D4F4F5F4F26173707480717
:10883000590748F02DC089E89AE00E94572F83E03D
:108840008093000B25C01092000B22C08DE79AE0A8
:108850006EE174E00E94E1350C511C4F39CF81E08C
:108860000E94FD460E94B6636093010B7093020B59
:108870008093030B9093040B8091890A8823F9F26B
:10888000DACFCE0DD11DC017D10708F421CF87CF85
:10889000DF91CF911F910F91FF90EF900895CF93AB
:1088A000DF9381E08093990A90917C0A892F8295C9
:1088B0008F70805D809347039F70905D9093480315
:1088C0001092000B0E94B663EB0104C00E945E4749
:1088D0000E94CF428091000B833061F00E94B6630A
:1088E0006C1B7D0B6053754728F40E941F4788233B
:1088F00089F3ECCF0E946D2E10929C0A10929B0A75
:1089000090E08091000B833009F491E0892FDF9192
:10891000CF9108950F931F938C01FC01868160E035
:108920000E94BB6281E090E00E941D64F801868194
:1089300061E00E94BB6281E090E00E941D64F8014A
:10894000868160E00E94BB6284E690E00E941D6424
:108950001F910F910895CF92DF92EF92FF920F93A4
:108960001F93CF93DF93D82EC92E282F392FC901FB
:108970008C01C0E0D0E0E62EFF24F801878161E0A1
:108980000E947C62B7010C2E02C0759567950A940F
:10899000E2F76170F80187810E94BB6221960F5F48
:1089A0001F4FC830D10549F78D2D9C2D0E948A4458
:1089B000DF91CF911F910F91FF90EF90DF90CF90BB
:1089C0000895CF92DF92EF92FF920F931F93CF9370
:1089D000DF93D82EC92E282F392FC9018C01C0E072
:1089E000D0E0E62EFF24F801878161E00E947C62DE
:1089F000B7010C2E02C0759567950A94E2F7617075
:108A0000F80187810E94BB6221960F5F1F4FC4301F
:108A1000D10549F78D2D9C2D0E948A44DF91CF917D
:108A20001F910F91FF90EF90DF90CF9008951F93CB
:108A3000CF93DF93EC01162F8C81642F0E94BB62D1
:108A40008D818F3F19F060E00E94BB628F8584FFAB
:108A500005C0CE01612F0E94AB440EC0612F70E0B3
:108A600084E0759567958A95E1F7CE010E94E1440F
:108A7000CE01612F0E94E144DF91CF911F910895B3
:108A800041E00E94174581E090E0089540E00E9497
:108A900017450895EF92FF920F931F93CF93DF93A3
:108AA0008C017A016770660F660F660F60640E9422
:108AB0004645C0E0D0E0D801ED91FC91D701AC0F64
:108AC000BD1F0190F081E02DC8016C9109952196A0
:108AD000C830D10581F7DF91CF911F910F91FF90A1
:108AE000EF900895FC0160896E7F608B68600E9442
:108AF00046450895FC016089862F8460808B6C60F8
:108B0000CF010E9446450895DF93CF93CDB7DEB7DE
:108B100028970FB6F894DEBF0FBECDBF9C01FE01B3
:108B20003196ABEAB3E088E00D9001928150E1F715
:108B3000F9018389481710F0482F4150E42FF0E0E5
:108B4000EE0FFF1FEC0FFD1F8181680F6068C901E8
:108B50000E94464528960FB6F894DEBF0FBECDBFE3
:108B6000CF91DF91089561E00E94464580ED97E046
:108B70000E941D640895CF93DF93EC01423018F0FA
:108B80008F8588608F874B8B1C8A222329F0413088
:108B900019F48F8584608F8780E593EC0E941D64B3
:108BA0008C8160E00E94BB628E8160E00E94BB62AB
:108BB0008D818F3F19F060E00E94BB626F8564FD7C
:108BC0001DC0CE0163E00E94E14484E991E10E946E
:108BD0001D64CE0163E00E94E14484E991E10E94BA
:108BE0001D64CE0163E00E94E14486E990E00E94AA
:108BF0001D64CE0162E00E94E14416C06062CE01B5
:108C00000E94464584E991E10E941D646F8560627F
:108C1000CE010E94464586E990E00E941D646F8562
:108C20006062CE010E9446456F856062CE010E945F
:108C3000464584E0888BCE010E947A45CE010E9491
:108C4000B34582E0898BCE0166E00E944645DF9104
:108C5000CF9108956F927F928F92AF92CF92EF92C1
:108C60000F931F93DF93CF93CDB7DEB73C01162F41
:108C7000842FF301448325830683E782C086A1867F
:108C800082869D8593879E8594879F859587988901
:108C9000968761E00E947C62F30185818F3F19F025
:108CA00061E00E947C62F301868161E00E947C6247
:108CB000112319F0F301178603C080E1F3018787C0
:108CC000C30160E141E020E00E94BB45CF91DF910C
:108CD0001F910F91EF90CF90AF908F907F906F90FA
:108CE00008958091190B61E00E94BB627894089509
:108CF000FF920F931F93082F162FF42EF894809154
:108D0000190B60E00E94BB621F71102B1EBD0DB4D9
:108D100007FEFDCFFEBC0DB407FEFDCF0E947146DD
:108D20001F910F91FF9008951F93182F282F30E067
:108D30002076307080911A0B90E02817390799F04F
:108D400080EA6FE143E00E947846412F40764093ED
:108D50001A0B50E085E0559547958A95E1F780E834
:108D60006FE10E9478461F9108950F931F93182F6B
:108D7000062F0E94944680E4612F402F0E9478467F
:108D80001F910F9108950F931F93182F072F0E9483
:108D9000B546812F8F5F602F0E94B5461F910F91BE
:108DA00008950F931F93182F062FF8948091190B95
:108DB00060E00E94BB62802F8F71812B8EBD0DB44D
:108DC00007FEFDCF1EBC0DB407FEFDCF07FF04C09C
:108DD0001EBC0DB407FEFDCF1EB50E947146812F4B
:108DE0001F910F9108951F93182F0E94944680E0C1
:108DF000612F0E94D1461F910895882311F410928B
:108E0000180B8091180B882341F488E30E94F346E5
:108E1000682F6E7F88E30E94B54608951F93182F30
:108E200088E30E94F346682F616088E30E94B5469C
:108E3000112319F481E08093180B1F91089584ED9C
:108E400061E10E94B54682ED61E00E94B5468AEE7E
:108E50000E94F34680FDFBCF82ED60E00E94B546A4
:108E600089ED0E94F34690E09695879596958795B3
:108E7000817008950F931F93CF93DF93EC018B01C3
:108E8000F8948091190B60E00E94BB628AE38EBD6A
:108E90000DB407FEFDCF09C01EBC0DB407FEFDCF0B
:108EA0008EB5F80181938F0121972097A9F70E9431
:108EB0007146DF91CF911F910F9108950F931F93EA
:108EC000DF93CF9300D000D000D0CDB7DEB789E3D9
:108ED0000E94F346882319F400E010E048C0609136
:108EE0001B0B70911C0B80E00E94C34686E090E053
:108EF000BE016F5F7F4F0E943A4789819A819093AC
:108F00001C0B80931B0B2B813C81E091160BF09185
:108F1000170B8D8187FD03C000E010E00EC02450C8
:108F200030408F01015010402017310708F48901AB
:108F3000C80164EE73E00E943A47F801EC51FC4F1F
:108F4000108260911B0B70911C0B8CE061307807D4
:108F500024F08CE06FEF7BE003C0615070408CE048
:108F60000E94C34680E86EE140E40E947846C80152
:108F700026960FB6F894DEBF0FBECDBFCF91DF911E
:108F80001F910F9108950F931F93CF93DF938C013F
:108F9000EB01F8948091190B60E00E94BB628AE7B4
:108FA0008EBD0DB407FEFDCF08C088818EBD0DB407
:108FB00007FEFDCF21960150104001151105A9F7BC
:108FC0000E947146DF91CF911F910F910895CF9329
:108FD000DF93EC010FC08CE10E94F34681FF0AC0D1
:108FE00080E86FE140E80E94784680EA6FE140E85F
:108FF0000E94784680E06FE10E94D14683FDEBCF6E
:1090000082E060E07CE00E94C346BE016050744F85
:1090100086E00E94C3468AE760E040E00E9478460E
:10902000CE0164EE73E00E94C34780E86FE148E040
:109030000E947846DF91CF91089584E061E00E941C
:109040007C6284E061E00E94BB6285E061E00E9496
:109050007C6287E061E00E947C6286E060E00E94C2
:109060007C6285E061E00E94BB6285E060E00E9476
:10907000BB6287E060E00E94BB6280E58CBD8DB57D
:1090800081608DBD08951F93CF93DF93EB01142F63
:109090009093170B8093160B0CB406FC02C00E9431
:1090A0001D481093190B812F61E00E947C620E9481
:1090B00071468FEF60E04FEF0E94784662E070E00B
:1090C00080E090E00E94C46380E06DE10E94D146A0
:1090D0008823D1F310921C0B10921B0B88E060E0E8
:1090E00070E00E94C3468CE060E070E00E94C346DE
:1090F0008AE06FEF7BE00E94C34684E060E07CE0A2
:109100000E94C34686E06FEF71E10E94C34680E093
:109110000E940E4788E26FE370E30E94C34680E33B
:1091200069EF77EF0E94C34680EC6DE00E94B54680
:1091300081EC60E00E94B54680E862EC42E30E9468
:10914000784686EC62E17CE00E94C34684EC62E1F2
:109150000E94B5468AEC6CED75E00E94C34684EE31
:1091600068810E94B54685EE69810E94B54682EE0F
:109170006A810E94B54683EE6B810E94B54680EEFF
:109180006C810E94B54681EE6D810E94B54684EDEA
:1091900060E10E94B54686ED60E071E00E94C34642
:1091A0008AEE0E94F34680FDFBCF8FE10E94944639
:1091B00080E86BE140EC0E94784680E86FE144E093
:1091C0000E94784682E70E94F346863008F08F5F5F
:1091D000DF91CF911F9108954E960E943F590895B7
:1091E000DF93CF93CDB7DEB76A970FB6F894DEBFA3
:1091F0000FBECDBFFB01242F19821B82BC01625E12
:109200007F4FCE010196AF010E94265A6A960FB693
:10921000F894DEBF0FBECDBFCF91DF9108954E967B
:109220000E9477590895CF93DF93EC01662331F0C4
:109230006E96D0932E0DC0932D0D6E9788A1882326
:1092400021F0CE014E960E946B51CE014E9625968E
:10925000BE010E94BB4EDF91CF910895DF92EF9245
:10926000FF920F931F93DF93CF93CDB7DEB76A972B
:109270000FB6F894DEBF0FBECDBF9C01FB01D42E0C
:1092800019821B8280818F3241F48181882329F4E5
:10929000C901642F0E94134922C08901025E1F4F39
:1092A0007E010894E11CF11CC701B801AF0121E067
:1092B0000E947758882391F08B81823078F0D80112
:1092C000F7018AE101900D928150E1F7DD2021F054
:1092D00010932E0D00932D0D81E001C080E06A9661
:1092E0000FB6F894DEBF0FBECDBFCF91DF911F91B7
:1092F0000F91FF90EF90DF9008950F931F93CF93FE
:10930000DF93EC010E94B45D8823C9F08E010B5FEE
:109310001F4FC801BE0141E00E94604A882339F412
:10932000C801BE0140E00E94604A882341F0CE019E
:1093300061E00E941349882319F081E001C080E0B8
:10934000DF91CF911F910F9108958FEF9FEFAFEFB6
:10935000BFEF8093220D9093230DA093240DB09323
:10936000250D1092260D08950F931F938C01CB01AC
:10937000BA016250704080409040F801248130E092
:1093800040E050E00E94A1689B01AC01F801828599
:109390009385A485B585280F391F4A1F5B1FB90126
:1093A000CA011F910F9108958091260D80FF3DC045
:1093B0004091220D5091230D6091240D7091250D47
:1093C0008091270D9091280D22E23BE00E94095DDB
:1093D000882369F18091260D81FF22C080911D0BA9
:1093E0008230F0F040911E0B50911F0B6091200BCA
:1093F0007091210B8091220D9091230DA091240D4D
:10940000B091250D480F591F6A1F7B1F8091270DB2
:109410009091280D22E23BE00E94095D882339F0FB
:109420008091260D8E7F8093260D81E0089580E047
:1094300008950E94D4490895DF92EF92FF920F930E
:109440001F937B018C01D42E8091220D9091230DCE
:10945000A091240DB091250D8E159F05A007B10791
:10946000E1F00E94D449882311F1D2FC0CC0809114
:10947000270D9091280DB801A70122E23BE00E9440
:10948000805D8823A1F01092260DE092220DF092CB
:10949000230D0093240D1093250D83E0D822809195
:1094A000260D8D298093260D22E23BE002C020E0AC
:1094B00030E0C9011F910F91FF90EF90DF90089568
:1094C0006F927F928F929F92AF92BF92CF92DF92D4
:1094D000EF92FF920F931F93CF93DF93EC01142F22
:1094E0007093280D6093270D1A8A82E090E0A0E027
:1094F000B0E088839983AA83BB831092260D8FEFF7
:109500009FEFAFEFBFEF8093220D9093230DA093B9
:10951000240DB093250D442321F4662477244301C0
:1095200036C0453008F0EFC060E070E080E090E0C9
:1095300040E00E941C4ADC01009709F4E4C0412F7E
:1095400050E041505040FA0174E0EE0FFF1F7A9551
:10955000E1F7E80FF91FE254FE4F808190E08F772A
:109560009070892B09F0CFC064E0440F551F6A95B5
:10957000E1F7A40FB51FAA53BE4F6D907D908D905B
:109580009C90611471048104910409F4BCC0C4016D
:10959000B30140E00E941C4A5C01009709F4B3C08B
:1095A000FC01838594858050924009F0ACC0F501A0
:1095B0002089222309F4A7C0468557854115510506
:1095C00009F4A1C020931D0B85858C83198691E039
:1095D00060E070E00AC0990F6F5F7F4F68307105DF
:1095E00009F491C089858F5F89878C81891799F7E4
:1095F000F501668977896115710519F080E090E0C1
:1096000005C0F50164A175A186A197A160931E0B09
:1096100070931F0B8093200B9093210B6A01EE2413
:10962000FF24C60CD71CE81CF91CCE86DF86E88A0E
:10963000F98AF501018912891C8B0B8B30E040E01F
:1096400050E00E94A1686C0D7D1D8E1D9F1D6D8BCD
:109650007E8B8F8B988F35E0000F111F3A95E1F7C5
:1096600001501E4F012F11270695980140E050E050
:10967000260F371F481F591F2A873B874C875D8756
:10968000F50183899489009721F07C0100E010E0C6
:1096900005C0F501E0A0F1A002A113A1C401B3012E
:1096A000621B730B840B950B6E0D7F1D801F911F2A
:1096B000098404C096958795779567950A94D2F7A3
:1096C0006D837E838F839887653FFFE07F07F0E09F
:1096D0008F07F0E09F0718F48CE08A8B14C0655F59
:1096E0007F4F8040904010F480E10AC0F50184A5CE
:1096F00095A5A6A5B7A58D8B9E8BAF8BB88F80E265
:109700008A8B81E001C080E0DF91CF911F910F91A2
:10971000FF90EF90DF90CF90BF90AF909F908F9091
:109720007F906F90089542600E941C4A08958F9226
:109730009F92AF92BF92CF92DF92EF92FF920F93E0
:109740001F93CF93DF93EC016A017B01480159011C
:10975000423051056105710508F44BC08D819E8131
:10976000AF81B8850196A11DB11D84179507A60785
:10977000B70708F43EC08A89803129F4252F362F97
:10978000472F55270BC08032A1F59A01AB0117E096
:1097900056954795379527951A95D1F78E859F85CC
:1097A000A889B989280F391F4A1F5B1FCA01B9014F
:1097B00041E00E94934B9C010097D9F08A89803147
:1097C00049F4F601F070EE0FFF1FE20FF31F9182D4
:1097D00080820DC0F601EF77F070EE0FFF1FEE0FE5
:1097E000FF1FE20FF31F80829182A282B38281E089
:1097F00001C080E0DF91CF911F910F91FF90EF901A
:10980000DF90CF90BF90AF909F908F900895CF92B0
:10981000DF92EF92FF920F931F93CF93DF93EC01B0
:109820007A018B016901423051056105710508F427
:1098300053C08D819E81AF81B8850196A11DB11D58
:1098400084179507A607B70708F446C08A898031B0
:1098500029F45527412F302F2F2D0BC08032E1F5F1
:109860009A01AB0167E056954795379527956A951C
:10987000D1F78E859F85A889B989280F391F4A1F7E
:109880005B1FCA01B90140E00E94934B9C01009705
:1098900019F18A89803159F4F701F070EE0FFF1F3A
:1098A000E20FF31F80819181A0E0B0E00EC0F701CC
:1098B000EF77F070EE0FFF1FEE0FFF1FE20FF31FA9
:1098C00080819181A281B381BF70F60180839183F1
:1098D000A283B38381E001C080E0DF91CF911F912B
:1098E0000F91FF90EF90DF90CF9008958F929F920D
:1098F000AF92BF92CF92DF92EF92FF920F931F939E
:10990000DF93CF9300D000D0CDB7DEB75C016A0102
:109910007B014E010894811C911CC501B701A60171
:1099200094010E94074C8823B1F1C501B701A6013B
:1099300000E010E020E030E00E94974B882359F1CE
:10994000F50180819181A281B381C816D906EA060A
:10995000FB0620F4C082D182E282F382C980DA80E1
:10996000EB80FC80F5018289803151F4F8EFCF164D
:10997000FFEFDF06F0E0EF06F0E0FF0670F209C04F
:1099800088EFC8168FEFD8068FEFE8068FE0F8064D
:1099900020F281E001C080E00F900F900F900F90B7
:1099A000CF91DF911F910F91FF90EF90DF90CF90BB
:1099B000BF90AF909F908F9008952F923F924F92BB
:1099C0005F926F927F928F929F92AF92BF92CF924F
:1099D000DF92EF92FF920F931F93DF93CF93CDB758
:1099E000DEB766970FB6F894DEBF0FBECDBF1C0181
:1099F00049875A876B877C873E872D87DC011596C0
:109A00002D913D914D915C9118972F5F3F4F4F4F96
:109A10005F4F2D833E834F835887ED85FE85008100
:109A2000118122813381011511052105310549F08C
:109A3000480159010894811C911CA11CB11C10E023
:109A400006C0DC018D909D90AD90BC9011E0750139
:109A50006401442455243201F10185819681A78156
:109A6000B085481659066A067B0608F09DC02D8110
:109A70003E814F8158852C153D054E055F0550F4FC
:109A8000F2E08F2E912CA12CB12CE2E0CE2ED12C25
:109A9000E12CF12CC101B701A6019E012F5F3F4FC0
:109AA0000E94074C882309F47FC089819A81AB8189
:109AB000BC810097A105B10571F08C149D04AE0422
:109AC000BF0409F010E0460157010894811C911C65
:109AD000A11CB11C16C0D701C6010196A11DB11D64
:109AE0008B8B9C8BAD8BBE8B88199909AA09BB09FE
:109AF00029853A854B855C8582179307A407B507AE
:109B000059F00894411C511C611C711C0894C11C23
:109B1000D11CE11CF11CA0CF112349F08B899C8939
:109B2000AD89BE89F10180839183A283B383C10192
:109B3000B701A6010FEF1FEF2FEF3FE00E94974BF9
:109B4000882399F431C0260137010894410851084F
:109B500061087108C101B301A201970186010E9449
:109B6000974B882309F1730162018C149D04AE04A4
:109B7000BF0448F3AD85BE854D915D916D917C919B
:109B8000411551056105710539F0C1019501840147
:109B90000E94974B882341F0ED85FE85808291825B
:109BA000A282B38281E001C080E066960FB6F8948D
:109BB000DEBF0FBECDBFCF91DF911F910F91FF9000
:109BC000EF90DF90CF90BF90AF909F908F907F905D
:109BD0006F905F904F903F902F9008958091C100BB
:109BE00085FDFCCF8091C00085FFF8CF6093C60053
:109BF00081E090E0089510922C0D10922B0D87EBD0
:109C000093E090932A0D8093290D08950F931F934D
:109C1000CF93DF93DC01EB018A0180E090E020E24A
:109C2000FE01E80FF91F208301968B309105C1F7E3
:109C300057E040E024C0622F2E3219F08CE79AE002
:109C400007C05A3051F15AE048E018C0321729F1E4
:109C5000FC01019634913323C9F75417F0F02132F7
:109C6000E0F02F37D0F4822F81568A3110F4622F22
:109C70006052FE01E40FF11D60834F5F11962C913D
:109C8000222311F02F32B9F6F801B183A08390E0BE
:109C90008881803219F091E001C090E0892FDF9136
:109CA000CF911F910F910895CF92DF92EF92FF9283
:109CB0000F931F93DF93CF9300D000D0CDB7DEB7C3
:109CC0007C01FC0186899789A08DB18D89839A8357
:109CD000AB83BC8300E010E06E010894C11CD11C72
:109CE00049815A816B817C81D70114968D919C9119
:109CF000159796010E94074C882379F1D701149695
:109D0000ED91FC9115978481080F111DB0E1003091
:109D10001B0718F529813A814B815C81828980314A
:109D200031F4285F3F4F40405040D0F205C0285FDB
:109D30003F4F4F4F5F40A0F2C801A0E0B0E029E0E4
:109D4000880F991FAA1FBB1F2A95D1F7F701828B95
:109D5000938BA48BB58B81E001C080E00F900F90B6
:109D60000F900F90CF91DF911F910F91FF90EF9087
:109D7000DF90CF900895CF93DF93EC01FB018A81B0
:109D80008823D1F57D836C8382898031C9F582E097
:109D90008A831E8A1F8A188E198E83899489A0E06F
:109DA000B0E035E0880F991FAA1FBB1F3A95D1F785
:109DB0008A8B9B8BAC8BBD8B0FC083E08A8385899C
:109DC0009689A789B08D8E8B9F8BA88FB98FCE0176
:109DD0000E94544E882381F081E089831E821F8275
:109DE000188619861A861B861C861D861E861F8667
:109DF000188A198A1B8201C080E0DF91CF910895F3
:109E00008032D1F7DACF6F927F928F929F92AF928A
:109E1000BF92CF92DF92EF92FF920F931F93CF9357
:109E2000DF93EC017A018B012A81222309F480C09F
:109E30008A899B89AC89BD8984179507A607B707CE
:109E400008F476C085C0E114F1040105110551F450
:109E50001E821F82188619861A861B861C861D86FE
:109E600081E067C02A853B854C855D85EC81FD815D
:109E7000818590E0099621503040404050403901A2
:109E80004A01082E04C096948794779467940A94A4
:109E9000D2F72F5F3F4F4F4F5F4F0894E108F10813
:109EA000010911095701680104C0D694C794B794F9
:109EB000A7948A95D2F70894E11CF11C011D111D8D
:109EC000A614B704C804D90428F0211531054105AA
:109ED000510549F48E899F89A88DB98D8E839F8302
:109EE000A887B98716C0A618B708C808D90811C02E
:109EF0004E815F81688579858C819D8194010E9466
:109F0000074C0894A108B108C108D108882331F48E
:109F10000FC046E0842E912C8C0E9D1EA114B1041E
:109F2000C104D10429F7EA86FB860C871D8798CFE8
:109F300080E0DF91CF911F910F91FF90EF90DF9024
:109F4000CF90BF90AF909F908F907F906F9008952B
:109F5000223009F078CFE7CFCF93DF93EC01462F83
:109F60006E857F85888999890E941C4AAC0100977B
:109F700019F420E030E00AC08B81282F30E065E042
:109F8000220F331F6A95E1F7240F351FC901DF91B6
:109F9000CF9108950F931F93CF93DF938C01FC0112
:109FA00082818823F1F1818187FF38C0C80161E097
:109FB0000E94AC4FEC010097A1F18881853E89F1A8
:109FC000F8018281823040F482899389A489B5891D
:109FD0008C8F9D8FAE8FBF8FF801868997899B8F5D
:109FE0008A8F86899789A08DB18DCD01AA27BB273D
:109FF0009D8B8C8BE0912F0DF091300D309751F0AF
:10A00000BE016A5E7F4FCE0148960995888D998D75
:10A010009B8B8A8BF80181818F7781830E94D44941
:10A0200004C081E0F801808380E0DF91CF911F912F
:10A030000F9108956F927F928F929F92AF92BF92ED
:10A04000CF92DF92EF92FF920F931F93DF93CF9304
:10A0500000D000D0CDB7DEB77C015A016B01DC0126
:10A0600012968C911297813009F091C011968C91C3
:10A0700081FF8DC0A0C00097A105B10511F481E05A
:10A0800087C0F7016284738484849584C701B60114
:10A09000A5010E94034F882309F479C0D7011496C3
:10A0A0008D919C911597A114B104C104D10489F438
:10A0B00056964D915D916D917C9159970E94764C89
:10A0C000882309F464C0F701168A178A108E118E4E
:10A0D00044C0D70116964D915D916D917C91199771
:10A0E0009E012F5F3F4F0E94074C882309F44FC009
:10A0F000D7011496ED91FC91159749815A816B8196
:10A100007C818289803149F4483FBFEF5B07B0E032
:10A110006B07B0E07B0748F020C0483F8FEF58073F
:10A120008FEF68078FE07807C0F4CF010E94764C6C
:10A13000882369F1D70116964D915D916D917C91BF
:10A14000199714968D919C9115970FEF1FEF2FEF94
:10A150003FE00E94974B8823D1F0F701A28AB38A8F
:10A16000C48AD58A818180688183C7010E94CA4FD1
:10A17000882369F0B601A5016A147B048C049D0450
:10A1800010F4B401A301C7010E94034F01C080E095
:10A190000F900F900F900F90CF91DF911F910F9123
:10A1A000FF90EF90DF90CF90BF90AF909F908F90F7
:10A1B0007F906F900895F70182899389A489B5896A
:10A1C00084179507A607B70708F055CFE0CF1F9370
:10A1D000CF93DF93EC01142F262F30E0F90185E0B7
:10A1E000EE0FFF1F8A95E1F7EE5DF44F83858171D5
:10A1F00021F0842F827109F064C08091220D90912A
:10A20000230DA091240DB091250D8E879F87A88BDB
:10A21000B98B6B83F901B5E0EE0FFF1FBA95E1F73B
:10A22000EE5DF44F2489358940E050E0A9013327E1
:10A2300022272E8B3F8B488F598F828D938DA0E0E4
:10A24000B0E0282B392B4A2B5B2B2E8B3F8B488F72
:10A25000598F838590E088719070009751F4848DB8
:10A26000958DA68DB78D8A8B9B8BAC8BBD8B81E03A
:10A2700008C0409731F5CE010E94544E882309F161
:10A2800084E08A83812F8F7089831E821F821886C3
:10A2900019861A861B861C861D8614FF18C0CE01DF
:10A2A00040E050E060E070E00E941A50882379F4AA
:10A2B00008C04A895B896C897D89CE010E94034F61
:10A2C00002C01A8280E0DF91CF911F91089515FDA1
:10A2D000F0CF81E0F8CF0F931F938C010E94CA4FFB
:10A2E000F80112821F910F910895CF93DF93EC0133
:10A2F00040E050E060E070E00E941A50882369F06E
:10A30000CE0161E00E94AC4FFC01009731F085EE78
:10A3100080831A820E94D44901C080E0DF91CF91EE
:10A3200008952F923F924F925F927F928F929F92C9
:10A33000AF92BF92CF92DF92EF92FF920F931F9353
:10A34000DF93CF93CDB7DEB728970FB6F894DEBF73
:10A350000FBECDBF98878F835E834D83DC0112963D
:10A360008C911297882309F41EC111968C9180FF5D
:10A370001AC134C1F501EE19FF09FE83ED837A831A
:10A3800069838F81988506969C838B834D805E8040
:10A3900003C1AF81B8851A962D913D914D915C9185
:10A3A0001D978FEF282E81E0382E2222332214961B
:10A3B000ED91FC91159759016A0109E0D694C79473
:10A3C000B794A7940A95D1F774807A947A2012965C
:10A3D0008C91823049F4E588F6880789108DEA0C63
:10A3E000FB1C0C1D1D1D35C02114310411F57720F7
:10A3F00001F5211531054105510559F4EF81F88525
:10A4000086899789A08DB18D86839783A087B18730
:10A4100010C0AF81B88516964D915D916D917C917C
:10A420001997CF012B813C810E94074C882309F4A6
:10A43000BAC0EF81F8854681578160857185848136
:10A4400095810E94B4497B018C01E70CF11C011D30
:10A45000111D2114310499F4F0E04F16F2E05F066B
:10A4600070F02091220D3091230D4091240D5091D8
:10A47000250DE216F3060407150709F0CFC0C80141
:10A48000B70140E00E941C4A009709F48CC040E0EC
:10A4900052E04219530942014415550508F44A0196
:10A4A0009C01220D331D89819A81B901A4010E946A
:10A4B000E70759C08091270D9091280DB801A70199
:10A4C00029813A810E94805D882309F46CC0812C27
:10A4D00012E0912E48C0D52CD694AF81B885129643
:10A4E0008C911297823049F01496ED91FC9115975A
:10A4F000848187198D1508F4D82EE216F306040717
:10A50000150770F02D0D311D411D511DE216F3068A
:10A510000407150728F40E94D449882309F443C08E
:10A520008091270D9091280DB801A7010E945D5DD3
:10A530008823C9F109811A81FF2408C0B8010E944B
:10A540005B5C00501E4F882371F1F3948091270DBE
:10A550009091280DFD1490F30E94435D882319F11A
:10A560009D2C990C8824E981FA81E80DF91DFA8364
:10A57000E983940140E050E0EF81F885828593857E
:10A58000A485B585820F931FA41FB51F828793876B
:10A59000A487B587481859084114510409F0F9CE29
:10A5A0004D815E8102C04FEF5FEFCA0128960FB662
:10A5B000F894DEBF0FBECDBFCF91DF911F910F91F9
:10A5C000FF90EF90DF90CF90BF90AF909F908F90D3
:10A5D0007F905F904F903F902F900895AF81B88506
:10A5E0005296AD90BD90CD90DC9055971A96ED9017
:10A5F000FD900D911C911D97ED81FE819F0140E022
:10A6000050E0D601C5018E199F09A00BB10B281788
:10A6100039074A075B0708F0ADCEB1CEF0E04F1620
:10A62000F4E05F0608F057CF45CFDF93CF930F924A
:10A63000CDB7DEB7BE016F5F7F4F41E050E00E94B3
:10A640009151019719F02FEF3FEF03C08981282F17
:10A6500030E0C9010F90CF91DF910895EF92FF9202
:10A660000F931F93CF93DF93EC018A81823038F1EF
:10A67000EA84FB840C851D85CE010E94155397FD4D
:10A680001EC08A859B85AC85BD854F96A11DB11DD9
:10A690008A879B87AC87BD8725E016950795F79439
:10A6A000E7942A95D1F72E2D30E02F70307095E089
:10A6B000220F331F9A95E1F72E5D344F02C020E040
:10A6C00030E0C901DF91CF911F910F91FF90EF9082
:10A6D0000895CF93DF93EC018A81843071F5CE0128
:10A6E00040E050E060E070E00E94034F10C0CE01F7
:10A6F0000E942E53FC01009701F180818823A1F074
:10A70000853E29F08E3219F0838583FF16C02A8595
:10A710003B854C855D858A899B89AC89BD892817D5
:10A7200039074A075B0718F381E08A8389818260D1
:10A730008983CE010E94755101C080E0DF91CF91E5
:10A740000895DF92EF92FF920F931F93CF93DF93C1
:10A750008C01EB017A01D22E8C819D81F8019583C9
:10A7600084838281882329F56115710559F521C0FB
:10A77000A70165E0440F551F6A95E1F760E070E0BE
:10A78000CE010E94034F8823A1F0CE010E942E53D8
:10A79000FC01009771F08081882359F0853E49F0D3
:10A7A0008E3239F06E2D6F70C8014D2D0E94E7502A
:10A7B00001C080E0DF91CF911F910F91FF90EF904A
:10A7C000DF90089527FFD4CFF4CFAF92BF92CF92FE
:10A7D000DF92EF92FF920F931F93DF93CF93CDB74A
:10A7E000DEB76A970FB6F894DEBF0FBECDBF8C01FF
:10A7F00019821B8240E050E060E070E00E94034F4D
:10A800005E010894A11CB11C52C0C8010E942E53C5
:10A81000FC01009709F466C08081882309F456C0C2
:10A82000853E09F444C08E3209F441C0838583FD1E
:10A830003EC0A7019601F5E05695479537952795B7
:10A84000FA95D1F77901C501B801A90121E00E946B
:10A85000A153882309F446C08B81843021F4C501BB
:10A860000E94E55306C08A8182608A83C5010E94E6
:10A8700075518823B9F10894E11CF11CA70160E02F
:10A8800070E0E5E0440F551F661F771FEA95D1F78A
:10A89000F80182859385A485B58584179507A60759
:10A8A000B70729F0C8010E94034F8823D9F0F801A7
:10A8B000C284D384E484F58482899389A489B58988
:10A8C000C816D906EA06FB0608F49FCFF801828174
:10A8D0008250823028F0C8010E946953882319F001
:10A8E00081E001C080E06A960FB6F894DEBF0FBE2B
:10A8F000CDBFCF91DF911F910F91FF90EF90DF902F
:10A90000CF90BF90AF9008952F923F924F925F9259
:10A910006F927F928F929F92AF92BF92CF92DF926F
:10A92000EF92FF920F931F93DF93CF930F92CDB7C8
:10A93000DEB72C015B013A01490100E010E0EE2492
:10A94000EA94FE2C1E010894211C311C13C00A0D30
:10A950001B1DF80160838114910419F46A3049F4D5
:10A960001EC0772767FD7095C4010E94F707009706
:10A97000B1F4860168010894C11CD11CC614D70427
:10A9800044F5C201B10141E050E00E9491517C01C7
:10A9900081309105F1F469816D30C9F6EBCF860104
:10A9A000A00EB11EF5011082C8010F90CF91DF916A
:10A9B0001F910F91FF90EF90DF90CF90BF90AF90DD
:10A9C0009F908F907F906F905F904F903F902F90CF
:10A9D0000895F7FEE5CF0FEF1FEFE6CFCF93DF939C
:10A9E000EC019C012A5F3F4F8C819D8141E050E04A
:10A9F00060E070E00E94DD4C8823A1F08E899F8981
:10AA0000A88DB98D0097A105B10559F48E819F815C
:10AA1000A885B9858E8B9F8BA88FB98F8981806817
:10AA2000898381E0DF91CF9108953F924F925F92A9
:10AA30006F927F928F929F92AF92BF92CF92DF924E
:10AA4000EF92FF920F931F93DF93CF93CDB7DEB7B3
:10AA50002A970FB6F894DEBF0FBECDBF4C01162F5C
:10AA6000072F5A874987DC0112968C911297813003
:10AA700009F0B0C111968C9181FFACC1C9C1F4013C
:10AA8000428953896489758982859385A485B585B2
:10AA900084179507A607B70731F0C4010E94034F3A
:10AAA000882309F497C1812F902F9C0138872F8329
:10AAB00029853A853E832D8351C1D4011496ED91A9
:10AAC000FC911597DA01C90119E0B695A7959795FC
:10AAD00087951A95D1F7F480FA94F82289011170BC
:10AAE000FF2009F052C00115110509F04EC0D40134
:10AAF00016964D915D916D917C9119974115510577
:10AB00006105710571F1CF019E012F5F3F4F0E94DA
:10AB1000074C882309F45EC129813A814B815C810D
:10AB2000D4011496ED91FC9115978289803149F4F6
:10AB3000283FBFEF3B07B0E04B07B0E05B0748F0B2
:10AB400019C0283FEFEF3E07EFEF4E07EFE05E073B
:10AB500088F4D40116962D933D934D935C931997E9
:10AB600014C0F40186899789A08DB18D0097A10545
:10AB7000B10531F4C4010E94EE54882331F42AC196
:10AB8000F40186839783A087B187D40116964D91EF
:10AB90005D916D917C91199714968D919C9115976B
:10ABA0000E94B4495B016C01AF0CB11CC11CD11CEB
:10ABB00001151105C9F4ED81FE81E050F240D8F590
:10ABC000D4011A962D913D914D915C911D9752960D
:10ABD0008D919D910D90BC91A02D281739074A07A2
:10ABE0005B0710F045E001C041E0C601B5010E94DD
:10ABF0001C4A009709F4EEC040E052E0401B510BA4
:10AC00004D805E804415550508F42A019C01200FF3
:10AC1000311FC9016F817885A2010E94E707040DE9
:10AC2000151D0050124009F07DC00E94194A88236A
:10AC300009F078C0CFC0ED81FE81E050F44000F50E
:10AC40008091220D9091230DA091240DB091250D9E
:10AC50008A159B05AC05BD0511F40E94A54980919C
:10AC6000270D9091280DB601A5012F8138850E94EE
:10AC7000095D882309F4AEC0412CF2E05F2E52C07A
:10AC8000D4011496ED91FC91159784818F193E8023
:10AC90003694831508F4382E032D10E020E030E0C0
:10ACA0008091270D9091280DB601A5010E94C15CED
:10ACB000882309F48FC06F8078848601750122C0D3
:10ACC0008091220D9091230DA091240DB091250D1E
:10ACD000E816F9060A071B0711F40E94A54980919E
:10ACE000270D9091280DB3010E94355CE0E0F2E061
:10ACF0006E0E7F1E0894E11CF11C011D111D88239E
:10AD000009F468C08E2D8A198315D0F28091270D21
:10AD10009091280D0E940F5C882309F45BC0532C8E
:10AD2000550C4424920140E050E0F4018285938563
:10AD3000A485B585820F931FA41FB51F82879387B3
:10AD4000A487B5872F813885240D351D38872F833B
:10AD50008D819E81841995099E838D83D4011A96D5
:10AD60002D913D914D915C911D97ED81FE81EF2BD1
:10AD700009F0A3CE52968D919D910D90BC91A02D7E
:10AD800082179307A407B50740F4D40152962D9378
:10AD90003D934D935C9355970BC080912F0D9091EF
:10ADA000300D892B59F0E985FA85EF2B39F0D40164
:10ADB00011968C911197806811968C93F401818182
:10ADC00083FF05C0C4010E94CA4F882319F049853A
:10ADD0005A8505C081E0D4018C934FEF5FEFCA0123
:10ADE0002A960FB6F894DEBF0FBECDBFCF91DF918C
:10ADF0001F910F91FF90EF90DF90CF90BF90AF9099
:10AE00009F908F907F906F905F904F903F900895AC
:10AE100082FD35CE48CE9F92AF92BF92CF92DF9205
:10AE2000EF92FF920F931F93CF93DF938C01FC015E
:10AE300082899389A489B589805E9F4FAF41B040D4
:10AE400008F05CC0C8010E94EE54882309F456C083
:10AE5000D80116964D915D916D917C91199714963C
:10AE60008D919C9115970E94B4495B016C0145E05E
:10AE70000E941C4AEC01009709F442C080E092E075
:10AE8000FE019C01119221503040E1F79C2EED2EE5
:10AE9000FF24F39411C0B601A5014F0D511D611D92
:10AEA000711D8091270D9091280D292D3E2D0E9416
:10AEB000095D882319F1F394D8011496ED91FC9162
:10AEC00015972481F21638F330E040E050E089E035
:10AED000220F331F441F551F8A95D1F752968D912B
:10AEE0009D910D90BC91A02D820F931FA41FB51FA3
:10AEF000F801828B938BA48BB58B02C0C0E0D0E0AD
:10AF0000CE01DF91CF911F910F91FF90EF90DF90D5
:10AF1000CF90BF90AF909F9008953F924F925F92D5
:10AF20006F927F928F929F92AF92BF92CF92DF9259
:10AF3000EF92FF920F931F93CF93DF934C01EB019E
:10AF4000442E352E522E8C819D81F401958384836D
:10AF5000CB0140E050E060E070E00E94034F7724B6
:10AF60004FC0CE010E94155397FDABC08A859B85CB
:10AF7000AC85BD8581509E4FAF4FBF4F8A879B8761
:10AF8000AC87BD87A090220DB090230DC090240DFA
:10AF9000D090250D22E2E22E2BE0F22E00E010E010
:10AFA000602EF7018081882311F0853E79F47720A7
:10AFB00041F4F401A686B786C08AD18A63827724D9
:10AFC0007394F7018081882391F428C0B80195E03B
:10AFD000660F771F9A95E1F76E5D744F842D932D60
:10AFE0004BE050E00E94DA07009709F47DC00F5F44
:10AFF0001F4F80E290E0E80EF91E0031110581F646
:10B000002A853B854C855D858A899B89AC89BD896C
:10B01000281739074A075B0708F4A3CF56FE51C02B
:10B0200051FE4FC0772051F0F4016380C40161E00C
:10B030000E94AC4FEC01009761F443C08A818230DA
:10B0400009F43FC0CE010E940B570097D1F1EC01EB
:10B05000662480E2FE0111928A95E9F7DE01242D33
:10B06000332DC901FC018BE001900D928150E1F775
:10B07000E0912F0DF091300D309739F0BE01625FF5
:10B080007F4FCE014096099508C081E298E2998BE6
:10B09000888B80E098E09F878E87888999899B8B31
:10B0A0008A8B998F888F8E859F859F8B8E8B0E9430
:10B0B000D449882331F0C401662D452D0E94E75004
:10B0C00001C080E0DF91CF911F910F91FF90EF9031
:10B0D000DF90CF90BF90AF909F908F907F906F90B8
:10B0E0005F904F903F90089557FEE5CFEACF2F92A3
:10B0F0003F924F925F926F927F928F929F92AF9208
:10B10000BF92CF92DF92EF92FF920F931F93DF9344
:10B11000CF93CDB7DEB7C454D0400FB6F894DEBF9E
:10B120000FBECDBF3C016B01DE01A05CBF4F11968D
:10B130005C934E9323962FAF23976115710509F405
:10B1400083C01E8618A6FC018281882309F07CC07A
:10B150001C861EA2FA0180818F32F1F086015CE02C
:10B16000E52EF12CEC0EFD1E40E4A42EB12CAC0E0D
:10B17000BD1E4E010894811C911C2596FFAEEEAEBB
:10B18000259736E2232E312C2C0E3D1E270124C09C
:10B190001196B183A08301C0FD01A081B1818C9182
:10B1A0008F32B1F3D60112968C9112978250823071
:10B1B000A8F28E010A5D1F4F14966D917C91159730
:10B1C000C8010E94BB4E882351F63EC0342D252D68
:10B1D0008701832F922F7C01F50180819181B40139
:10B1E000A5010E94064E882329F42EC03196D50170
:10B1F000ED93FC93D501ED91FC9180818F32B1F3F9
:10B200008823C9F0C701B801A40121E00E948D572D
:10B210008823D1F00C151D0519F0C8010E946B514F
:10B220002596EEADFFAD2597EE16FF0679F6C10126
:10B23000322D292FCDCFC301B801A40123962FAD04
:10B2400023970E948D5701C080E0CC5BDF4F0FB683
:10B25000F894DEBF0FBECDBFCF91DF911F910F914C
:10B26000FF90EF90DF90CF90BF90AF909F908F9026
:10B270007F906F905F904F903F902F9008950F9325
:10B280001F93DF93CF93CDB7DEB76A970FB6F894CD
:10B29000DEBF0FBECDBF9C01AB0119821B828E01A8
:10B2A0000F5F1F4FC801B90122E00E947758882321
:10B2B00019F0C8010E9475516A960FB6F894DEBF66
:10B2C0000FBECDBFCF91DF911F910F910895FB016C
:10B2D000242F60912D0D70912E0DAF010E94775893
:10B2E0000895FC01128210820E9467590895DF932D
:10B2F000CF93CDB7DEB76A970FB6F894DEBF0FBE17
:10B30000CDBF9C01AB0119821B82CE010196B90110
:10B3100021E00E9477586A960FB6F894DEBF0FBE00
:10B32000CDBFCF91DF910895EF92FF920F931F93BE
:10B33000DF93CF93CDB7DEB7A0970FB6F894DEBFFB
:10B340000FBECDBF8C017B01FB018281823008F4EE
:10B350006FC0C80123EC0E948D57882309F468C090
:10B3600081E0F801818384E08283C8010E940B5749
:10B37000892B09F45DC0C8010E94CA4F882309F4D3
:10B3800057C0C80161E00E94AC4FFC01009709F46E
:10B390004FC080E18387DE01119680E201900D921B
:10B3A0008150E1F78EE28983FE01329620E2CE01E0
:10B3B0000C962193E817F907E1F7F80146895789B8
:10B3C000608D718D848195810E94B44941E00E9415
:10B3D0001C4A9C01009761F1DC01FE01319680E27C
:10B3E00001900D928150E1F78EE28A83F70182810C
:10B3F0008250823028F41C8E1B8E1E8A1D8A0CC03F
:10B40000F70186899789A08DB18D9C8F8B8FCD0197
:10B41000AA27BB279E8B8D8BD9019096FE01319672
:10B4200080E201900D928150E1F70E94D44901C061
:10B4300080E0A0960FB6F894DEBF0FBECDBFCF91CF
:10B44000DF911F910F91FF90EF9008952F923F92FF
:10B450004F925F926F927F928F929F92AF92BF9224
:10B46000CF92DF92EF92FF920F931F93DF93CF93D0
:10B47000CDB7DEB7C454D0400FB6F894DEBF0FBED0
:10B48000CDBF3C016B01DE01A05CBF4F11965C9308
:10B490004E9323962FAF23976115710509F487C04A
:10B4A0001E8618A6FC018281882309F080C09AC0FC
:10B4B0008601FCE0EF2EF12CEC0EFD1EE0E4AE2E3A
:10B4C000B12CAC0EBD1E4E010894811C911C25961A
:10B4D000FFAEEEAE259776E2272E312C2C0E3D1EC8
:10B4E000270124C01196B183A08301C0FD01A08172
:10B4F000B1818C918F32B1F3D60112968C91129753
:10B5000082508230A8F28E010A5D1F4F14966D9111
:10B510007C911597C8010E94BB4E882351F647C005
:10B52000342D252D8701832F922F7C01F5018081F9
:10B530009181B401A5010E94064E882329F437C0E9
:10B540003196D501ED93FC93D501ED91FC9180816D
:10B550008F32B1F3882329F1C701B801A40121E09A
:10B560000E948D57882361F42396BFAD2397BB2398
:10B57000F1F0C701B801A4010E9494598823B9F0E1
:10B580000C151D0519F0C8010E946B512596EEADF2
:10B59000FFAD2597EE16FF0619F6C101322D292FB2
:10B5A000C1CFC301B801A4010E94945901C080E039
:10B5B000CC5BDF4F0FB6F894DEBF0FBECDBFCF918F
:10B5C000DF911F910F91FF90EF90DF90CF90BF9090
:10B5D000AF909F908F907F906F905F904F903F9033
:10B5E0002F9008951C861EA2ED91FC9111978081E9
:10B5F0008F3209F05DCF7ACF40E082E002C0880F41
:10B600004F5F861710F44630D1F7242F30E0C90180
:10B610009595879580658CBD40FF02C080E004C091
:10B6200080E0463009F081E08DBD089584E061E05E
:10B630000E94BB6284E061E00E947C6286E060E080
:10B640000E947C6285E061E00E947C6287E061E0AC
:10B650000E947C620895FF920F931F93CF93DF9314
:10B660008B010E94B663EB01FF24FA9409C00E948B
:10B67000B6636C1B7D0B6017710710F080E008C08B
:10B68000FEBC0DB407FEFDCF8EB58F3F81F781E084
:10B69000DF91CF911F910F91FF900895FC01808160
:10B6A00061E00E94BB628FEF8EBD0DB407FEFDCF3F
:10B6B0000895CF93DF93EC01DA016EBD0DB407FE60
:10B6C000FDCF8C918EBD1196EC91119782E090E0A8
:10B6D0000DB407FEFDCFEEBD22E08030920731F0C1
:10B6E000FD01E80FF91FE0810196F2CF0DB407FECE
:10B6F000FDCF8FEF8EBD0DB407FEFDCF8FEF8EBD5A
:10B700000DB407FEFDCF8FEF8EBD0DB407FEFDCF4C
:10B710008EB58B838F71853011F481E006C083E193
:10B720008983CE010E944E5B80E0DF91CF91089526
:10B73000BF92CF92DF92EF92FF920F931F93CF931E
:10B74000DF93EC016B017A010E94B6638B01BB248D
:10B75000BA9409C00E94B663601B710B6D527140B0
:10B7600010F081E10BC0BEBC0DB407FEFDCF8EB55D
:10B770008B838F3F79F38E3F39F08FE08983CE0141
:10B780000E944E5B80E030C0D7011197EF28D9F0BE
:10B790008FEF8EBD20E030E09FEF0BC00DB407FEB1
:10B7A000FDCF8EB59EBDF601E20FF31F80832F5FA4
:10B7B0003F4F2A173B0790F30DB407FEFDCF8EB520
:10B7C000AC0DBD1D8C931B828FEF8EBD0DB407FE9B
:10B7D000FDCF8EB58FEF8EBD0DB407FEFDCF8EB5BC
:10B7E000CE010E944E5B81E0DF91CF911F910F91BE
:10B7F000FF90EF90DF90CF90BF9008950F931F932D
:10B800008C0181E39DE0F80162810E94FC5AF801FD
:10B81000808160E00E94BB621F910F910895CF93D9
:10B82000DF93EC010E94FE5BCE0168E572E00E94AE
:10B830002B5B882389F08DEF8EBD0DB407FEFDCF05
:10B84000CE0168E572E00E942B5B882329F0CE01CF
:10B850000E944E5B81E006C082E18983CE010E9496
:10B860004E5B80E0DF91CF9108950F931F93CF93AC
:10B87000DF93EC018B010E94FE5BCE0168E572E074
:10B880000E942B5B882361F0CE016CEFA8010E941F
:10B89000595B882329F0CE010E944E5B81E006C0EF
:10B8A00085E18983CE010E944E5B80E0DF91CF91DC
:10B8B0001F910F910895EF92FF920F931F938C01A8
:10B8C0007B010E94FE5BC801B70140E052E00E948C
:10B8D000985B1F910F91FF90EF900895FF920F9347
:10B8E0001F93DF93CF9300D000D0CDB7DEB78C018C
:10B8F000F62E29833A834B835C830E94FE5BC8014A
:10B9000068E572E00E942B5B8F2D80648EBD0DB4C4
:10B9100007FEFDCFFE0131969E012350304083810A
:10B920008EBD0DB407FEFDCF3197E217F307B9F7CF
:10B93000FF2011F087E801C085E98EBD0DB407FE38
:10B94000FDCF8CE0F81631F48FEF8EBD0DB407FEFD
:10B95000FDCF8EB590E02FEF2EBD0DB407FEFDCFCD
:10B960008EB587FF02C09150B9F7F80183830F901D
:10B970000F900F900F90CF91DF911F910F91FF903B
:10B980000895AF92BF92CF92DF92EF92FF920F9302
:10B990001F93CF93DF93EC015A016B01780189016A
:10B9A00067E320E030E040E050E00E946E5CCE01B2
:10B9B00067E1A80197010E946E5C882311F089E07D
:10B9C00013C08C81833039F089E0AA0CBB1CCC1CDD
:10B9D000DD1C8A95D1F7CE0169E1A60195010E948F
:10B9E0006E5C882339F087E08983CE010E944E5B2C
:10B9F00080E004C0CE010E944E5B81E0DF91CF91D8
:10BA00001F910F91FF90EF90DF90CF90BF90AF907C
:10BA10000895CF92DF92EF92FF920F931F93CF93EF
:10BA2000DF93EC017A018B0169018C81833039F05D
:10BA300099E0EE0CFF1C001F111F9A95D1F7CE0163
:10BA400068E1A80197010E946E5C882319F086E0E6
:10BA500089830CC0CE016EEFA6010E94595B88233A
:10BA600029F0CE010E944E5B81E004C0CE010E940D
:10BA70004E5B80E0DF91CF911F910F91FF90EF908F
:10BA8000DF90CF900895CF93DF93EC016CE020E03E
:10BA900030E040E050E00E946E5C882339F083E0A3
:10BAA0008983CE010E944E5B80E004C0CE010E94DB
:10BAB0004E5B81E0DF91CF910895CF93DF93EC014E
:10BAC0009A01AB018C81833039F069E0220F331F7A
:10BAD000441F551F6A95D1F7CE0162E10E946E5C4A
:10BAE000882339F085E08983CE010E944E5B80E097
:10BAF00004C0CE010E944E5B81E0DF91CF9108959A
:10BB0000CF92DF92EF92FF920F931F93CF93DF9329
:10BB1000EC017A018B0169018C81833039F0B9E045
:10BB2000EE0CFF1C001F111FBA95D1F7CE0161E189
:10BB3000A80197010E946E5C882339F084E0898314
:10BB4000CE010E944E5B80E006C0CE01B60140E00F
:10BB500052E00E94985BDF91CF911F910F91FF906F
:10BB6000EF90DF90CF900895BF92CF92DF92EF9247
:10BB7000FF920F931F93CF93DF93EC01B42E1C829F
:10BB8000198268830E94B6636B01888161E00E941C
:10BB90007C62888161E00E94BB6281E39DE00E943B
:10BBA000165B80E48A8381E39DE060E40E94FC5A96
:10BBB00080E09FEF9EBD0DB407FEFDCF8F5F8A3002
:10BBC000C9F709C00E94B6636C197D09615D7740B1
:10BBD00010F081E063C0CE0160E020E030E040E0A2
:10BBE00050E00E946E5C813069F71FEFCE0168E083
:10BBF0002AEA31E040E050E00E946E5C853011F4AA
:10BC000081E00DC080E01EBD0DB407FEFDCF9EB5E6
:10BC10008F5F8430C1F79B839A3A31F482E08C8342
:10BC20008C81823051F40DC00E94B6636C197D097D
:10BC3000615D7740D8F282E031C0EE24FF248701B5
:10BC40000FC0E12CF12C012D80E4182F09C00E94B7
:10BC5000B6636C197D09615D774010F08AE01EC003
:10BC6000CE0167E320E030E040E050E00E946E5CEF
:10BC7000CE0169E2A80197010E946E5C882339F722
:10BC80008C81823031F5CE016AE320E030E040E083
:10BC900050E00E946E5C882339F088E08983CE01F1
:10BCA0000E944E5B80E01AC08FEF8EBD0DB407FE80
:10BCB000FDCF8EB5807C803C11F483E08C8380E0E6
:10BCC0009FEF9EBD0DB407FEFDCF2EB58F5F833075
:10BCD000C1F7CE010E944E5BBA8281E0DF91CF9125
:10BCE0001F910F91FF90EF90DF90CF90BF9008953C
:10BCF000DB010D900020E9F71197A61BB70B049606
:10BD0000AD010E9415550895DF93CF930F92CDB7E3
:10BD1000DEB769830496BE016F5F7F4F41E050E05C
:10BD20000E94155520E030E0019711F421E030E049
:10BD3000C9010F90CF91DF9108950F931F938C014C
:10BD400004960E947159F801138212828FEB93E0DE
:10BD5000918380831F910F91089581E08093770DE7
:10BD60006093540D1092750D1092760D08952091E8
:10BD7000530D30E08091520D281B3109C9010895FF
:10BD80004091520D8091530D481718F02FEF3FEF5F
:10BD90000AC0E42FF0E0EE5CF24F8081282F30E003
:10BDA0004F5F4093520DC9010895E091520D80916B
:10BDB000530DE81718F0EFEFFFEF06C0F0E0EE5C70
:10BDC000F24F8081E82FF0E0CF010895089510929E
:10BDD0007B0D10927A0D88EE93E0A0E0B0E08093A6
:10BDE0007C0D90937D0DA0937E0DB0937F0D87EC1D
:10BDF00093E09093790D8093780D0895CF92DF9220
:10BE0000EF92FF920F931F93CF93DF937C016B010F
:10BE10008A018091770D8823A1F0C0E0D0E00DC0A9
:10BE2000D701ED91FC91D601AC0FBD1F0190F081BF
:10BE3000E02DC7016C9109952196C017D10780F3B9
:10BE400004C0CB01642F0E943060C801DF91CF9104
:10BE50001F910F91FF90EF90DF90CF900895DF93A7
:10BE6000CF930F92CDB7DEB7FC0169838091770D38
:10BE70008823C9F08091760D803238F081E090E01F
:10BE80009383828320E030E015C08091750DE82F08
:10BE9000F0E0EB5AF24F998190838F5F8093750D9C
:10BEA0008093760D05C0CE01019661E00E9430605E
:10BEB00021E030E0C9010F90CF91DF9108950F93F9
:10BEC000062F8091540D65E57DE04091760D21E0CF
:10BED0000E94DB5F1092750D1092760D1092770D17
:10BEE0000F91089561E00E945F5F0895413208F06C
:10BEF00040E2862F62E37DE00E94925F1092520D35
:10BF00008093530D089521E00E94765F089510926A
:10BF1000520D1092530D1092750D1092760D0E94D5
:10BF2000DC610895382F413210F040E042C080912A
:10BF3000840D8823E1F791E09093840D2093860D82
:10BF40008FEF8093F10D1092AC0D41504093AD0DE9
:10BF50004F5F9093850D8091850D330F832B8093D8
:10BF6000850D8091870D813041F41092870D80916D
:10BF7000850D8093BB0085EC01C085EE8093BC00ED
:10BF80008091840D8130E1F38091AC0D841710F421
:10BF90004091AC0D20E030E00AC0FB01E20FF31F3E
:10BFA000D901A457B24F8C9180832F5F3F4F241744
:10BFB000A0F3842F08950F931F93582F122F41320F
:10BFC00010F081E04AC08091840D8823E1F782E07F
:10BFD0008093840D0093860D8FEF8093F10D109266
:10BFE000AC0D4093AD0DACE8BDE0FB0102C081910A
:10BFF0008D938E2F861B8417D0F31092850D809120
:10C00000850D550F852B8093850D8091870D81308F
:10C0100041F41092870D8091850D8093BB0085ECD3
:10C0200001C085EE8093BC00112321F08091840D26
:10C030008230E1F38091F10D8F3F11F480E00DC06B
:10C040008091F10D803211F482E007C08091F10DF2
:10C05000803311F084E001C083E01F910F910895B7
:10C06000482F613210F081E008958091840D843072
:10C0700011F082E008956093CF0DAEEABDE0842F09
:10C080009C01F90102C081918D938E2F841B86172C
:10C09000D0F380E008951F920F920FB60F921124F3
:10C0A0002F933F934F935F936F937F938F939F93C0
:10C0B000AF93BF93EF93FF938091B90090E0887F97
:10C0C00090708036910509F4F2C081369105CCF567
:10C0D0008832910509F47BC089329105B4F480312E
:10C0E000910509F46FC0813191053CF4009709F482
:10C0F00047C1089709F04FC165C08831910509F41F
:10C1000066C0809709F047C182C08034910509F468
:10C11000A4C08134910544F48033910509F482C0B0
:10C12000C89709F038C189C08035910509F489C0E4
:10C130008835910509F496C08834910509F02BC122
:10C14000AEC08839910509F413C189399105ECF421
:10C150008837910509F4ABC0893791054CF48836CE
:10C16000910509F4A4C08037910509F014C19FC05E
:10C170008838910509F4FCC08039910509F49DC007
:10C180008038910509F007C198C0803B910509F4FA
:10C19000C6C0813B91054CF4803A910509F49FC0DB
:10C1A000883A910509F0F7C0BAC0803C910509F4BE
:10C1B000E3C0883C910509F4DFC0883B910509F094
:10C1C000EAC0C2C08091850D8093BB00CFC0909122
:10C1D000AC0D8091AD0D981768F49091AC0DE92FDE
:10C1E000F0E0E457F24F80818093BB009F5F909313
:10C1F000AC0DBCC08091860D882309F44BC085ED41
:10C200008093BC008091BC0084FDFCCFC2C080E262
:10C210008093F10D85ED8093BC008091BC0084FD7E
:10C22000FCCFB7C080E38093F10D85ED8093BC0017
:10C230008091BC0084FDFCCFACC088E38093F10DFD
:10C240009BC08091AC0D9091BB00E82FF0E0E457CB
:10C25000F24F90838F5F8093AC0D9091AC0D8091E5
:10C26000AD0D82C08091AC0D9091BB00E82FF0E045
:10C27000E457F24F90838F5F8093AC0D8091860DD1
:10C28000882341F085ED8093BC008091BC0084FD43
:10C29000FCCF7FC081E08093870D84EA6EC085ED7E
:10C2A0008093BC008091BC0084FDFCCF72C083E011
:10C2B0008093840D1092F00D59C08091F00D803262
:10C2C00008F056C08091F00D9091BB00E82FF0E08F
:10C2D000E053F24F90838F5F8093F00D47C08091C1
:10C2E000F00D803230F4E091F00DF0E0E053F24FC9
:10C2F000108285ED8093BC008091BC0084FDFCCF52
:10C300001092840D6091F00DE0918A0DF0918B0DEB
:10C3100080ED9DE070E009951092F00D2DC084E055
:10C320008093840D1092CE0D1092CF0DE091880D68
:10C33000F091890D09958091CF0D882329F481E032
:10C340008093CF0D1092AE0D9091CE0DE92FF0E0BD
:10C35000E255F24F80818093BB009F5F9093CE0D9A
:10C360009091CE0D8091CF0D981710F485EC01C0FF
:10C3700085E88093BC000FC085EC8093BC0009C0A9
:10C380001092F10D85ED8093BC008091BC0084FD7E
:10C39000FCCF1092840DFF91EF91BF91AF919F91CF
:10C3A0008F917F916F915F914F913F912F910F905E
:10C3B0000FBE0F901F9018951092840D81E080930E
:10C3C000860D1092870D81E161E00E94BB6280E1E1
:10C3D00061E00E94BB62E9EBF0E080818E7F8083A8
:10C3E00080818D7F808380E28093B80085E4809394
:10C3F000BC000895982F8E3008F09E509770809161
:10C4000050038295880F880F807C892B80937C0055
:10C4100080917A00806480937A0080917A0086FD12
:10C42000FCCF2091780040917900942F80E030E09B
:10C43000282B392BC90108951F93CF93DF93182F11
:10C44000EB0161E00E947C62209709F44AC0CF3F73
:10C45000D10509F449C0E12FF0E0E651F54F849190
:10C460008330C1F0843028F4813051F08230B1F54E
:10C470000CC0863019F1873049F1843079F514C049
:10C4800084B5806884BDC7BD33C084B5806284BD77
:10C49000C8BD2EC080918000806880938000D093BA
:10C4A0008900C093880024C08091800080628093BE
:10C4B0008000D0938B00C0938A001AC08091B00096
:10C4C00080688093B000C093B30012C08091B00028
:10C4D00080628093B000C093B4000AC0C038D10518
:10C4E0001CF4812F60E002C0812F61E00E94BB62DA
:10C4F000DF91CF911F910895CF93DF93482F50E0A4
:10C50000CA018653954FFC0134914655554FFA01A7
:10C510008491882369F190E0880F991FFC01E4570A
:10C52000F54FA591B491FC01EA56F54FC591D49110
:10C53000662351F42FB7F8948C91932F909589230B
:10C540008C93888189230BC0623061F42FB7F894F3
:10C550008C91932F909589238C938881832B88834A
:10C560002FBF06C09FB7F8948C91832B8C939FBFED
:10C57000DF91CF910895482F50E0CA018651954F21
:10C58000FC012491CA018653954FFC0194914655B4
:10C59000554FFA013491332309F440C0222351F15D
:10C5A000233071F0243028F42130A1F0223011F52D
:10C5B00014C02630B1F02730C1F02430D9F404C0C3
:10C5C000809180008F7703C0809180008F7D809361
:10C5D000800010C084B58F7702C084B58F7D84BD84
:10C5E00009C08091B0008F7703C08091B0008F7D2B
:10C5F0008093B000E32FF0E0EE0FFF1FEA56F54FF7
:10C60000A591B4912FB7F894662321F48C9190955D
:10C61000892302C08C91892B8C932FBF0895682F9A
:10C6200070E0CB018651954FFC012491CB018653DC
:10C63000954FFC0144916655754FFB0194919923E8
:10C6400019F420E030E03CC0222351F1233071F096
:10C65000243028F42130A1F0223011F514C0263006
:10C66000B1F02730C1F02430D9F404C080918000AB
:10C670008F7703C0809180008F7D8093800010C0F1
:10C6800084B58F7702C084B58F7D84BD09C0809149
:10C69000B0008F7703C08091B0008F7D8093B00091
:10C6A000892F90E0880F991F8056954FFC01A59126
:10C6B000B4918C9120E030E0842311F021E030E04F
:10C6C000C90108951F920F920FB60F9211242F9354
:10C6D0003F934F935F936F937F938F939F93AF930A
:10C6E000BF932091F60D3091F70D4091F80D5091C8
:10C6F000F90D7091FA0DDA01C9010296A11DB11D63
:10C70000672F6A5F6D3730F06D57DA01C901039604
:10C71000A11DB11D6093FA0D8093F60D9093F70D56
:10C72000A093F80DB093F90D8091F20D9091F30D57
:10C73000A091F40DB091F50D0196A11DB11D80934E
:10C74000F20D9093F30DA093F40DB093F50DBF91FE
:10C75000AF919F918F917F916F915F914F913F9199
:10C760002F910F900FBE0F901F9018958FB7F894D0
:10C770002091F60D3091F70D4091F80D5091F90D83
:10C780008FBFB901CA0108959B01AC017FB7F8942E
:10C790008091F20D9091F30DA091F40DB091F50DF3
:10C7A00066B5A89B05C06F3F19F00196A11DB11D8C
:10C7B0007FBFBA2FA92F982F8827860F911DA11D03
:10C7C000B11D63E0880F991FAA1FBB1F6A95D1F79F
:10C7D000BC012DC0FFB7F8948091F20D9091F30D3C
:10C7E000A091F40DB091F50DE6B5A89B05C0EF3F03
:10C7F00019F00196A11DB11DFFBFBA2FA92F982FC7
:10C8000088278E0F911DA11DB11DE3E0880F991F90
:10C81000AA1FBB1FEA95D1F7861B970B885E934032
:10C82000C8F2215030404040504068517C4F2115A3
:10C8300031054105510571F60895019739F00197C9
:10C8400029F0880F991F01970197F1F708957894BF
:10C8500084B5826084BD84B5816084BD85B5826005
:10C8600085BD85B5816085BDEEE6F0E080818160A3
:10C870008083E1E8F0E010828081826080838081A3
:10C8800081608083E0E8F0E0808181608083E1EB7B
:10C89000F0E0808184608083E0EBF0E08081816063
:10C8A0008083EAE7F0E08081846080838081826019
:10C8B0008083808181608083808180688083109202
:10C8C000C100089508951F920F920FB60F92112480
:10C8D0002F933F934F938F939F93EF93FF934091A9
:10C8E000C60020913B0E30913C0E2F5F3F4F2F73BF
:10C8F000307080913D0E90913E0E2817390759F007
:10C90000E0913B0EF0913C0EE550F24F40833093A6
:10C910003C0E20933B0EFF91EF919F918F914F9191
:10C920003F912F910F900FBE0F901F901895E0919F
:10C930008F0EF091900EE05CFF4F819191912081DC
:10C940003181821B930B8F739070892B11F00E94A1
:10C95000626408951F920F920FB60F9211242F93C5
:10C960003F938F939F93EF93FF9320917F0E30918E
:10C97000800E8091810E9091820E2817390731F434
:10C980008091C1008F7D8093C10014C0E091810E21
:10C99000F091820EE15CF14F20818091810E9091A7
:10C9A000820E01968F7390709093820E8093810E09
:10C9B0002093C600FF91EF919F918F913F912F910E
:10C9C0000F900FBE0F901F901895DC011C96ED91F3
:10C9D000FC911D97E05CFF4F219131918081918105
:10C9E000281B390B2F733070C9010895DC011C9688
:10C9F000ED91FC911D97E05CFF4F20813181E05467
:10CA0000F040DF01AE5BBF4F8D919C9111972817CD
:10CA1000390719F42FEF3FEF07C08D919C91E80F74
:10CA2000F91F8081282F30E0C9010895DC011C9690
:10CA3000ED91FC911D97E05CFF4F20813181E05426
:10CA4000F040DF01AE5BBF4F8D919C91119728178D
:10CA5000390719F42FEF3FEF10C08D919C9111977A
:10CA6000E80FF91F20818D919C91119701968F738A
:10CA7000907011969C938E9330E0C9010895FC014B
:10CA800086859785DC01A05CBF4FFC01EE5BFF4F04
:10CA90002D913C9111978081918128173907C1F719
:10CAA0000895CF93DF93EC01EE85FF85E05CFF4FA7
:10CAB00020813181E054F0402F5F3F4F2F73307061
:10CAC000DF01AE5BBF4F8D919C91119728173907FD
:10CAD000D1F3E05CFF4F80819181E054F040E80F9A
:10CAE000F91F6083EE85FF85E05CFF4F3183208373
:10CAF000EE89FF89208181E090E00D8C02C0880FD3
:10CB0000991F0A94E2F7282B208381E090E0DF91BF
:10CB1000CF9108951092860E1092850E88EE93E0C4
:10CB2000A0E0B0E08093870E9093880EA093890ECA
:10CB3000B0938A0E87ED93E09093840E8093830EDA
:10CB40008BEF9DE09093900E80938F0E8FE39EE08D
:10CB50009093920E8093910E85EC90E09093940EBA
:10CB60008093930E84EC90E09093960E8093950EB4
:10CB700080EC90E09093980E8093970E81EC90E07B
:10CB800090939A0E8093990E86EC90E090939C0E71
:10CB900080939B0E84E080939D0E83E080939E0E95
:10CBA00087E080939F0E85E08093A00E81E08093C4
:10CBB000A10E0895CF92DF92EF92FF920F931F93F1
:10CBC000CF93DF937C016B018A01C0E0D0E00FC0FE
:10CBD000D6016D916D01D701ED91FC910190F0812D
:10CBE000E02DC7010995C80FD91F0150104001154C
:10CBF000110571F7CE01DF91CF911F910F91FF9039
:10CC0000EF90DF90CF900895DC01ED91FC910190C1
:10CC1000F081E02D09950895CF93DF93DB010D900E
:10CC20000020E9F71197A61BB70BEC01E881F98109
:10CC30000280F381E02DAD010995DF91CF91089538
:10CC40004F925F927F928F929F92AF92BF92CF92BC
:10CC5000DF92EF92FF920F931F93DF93CF93CDB7A5
:10CC6000DEB7A1970FB6F894DEBF0FBECDBF2C0183
:10CC7000742ECB01223008F42AE019A231E2C32E2F
:10CC8000D12CCC0EDD1E822E9924AA24BB24672D24
:10CC9000752FA50194010E94F36879018A01C801EA
:10CCA000B701A50194010E94A168472D461B089475
:10CCB000C108D1084A3014F4405D01C0495CF60156
:10CCC0004083E114F1040105110521F07E2C5F2D54
:10CCD000C801DDCFC201B6010E940C66A1960FB655
:10CCE000F894DEBF0FBECDBFCF91DF911F910F91A2
:10CCF000FF90EF90DF90CF90BF90AF909F908F907C
:10CD00007F905F904F900895DC012115310541F42B
:10CD1000ED91FC910190F081E02D642F099508952B
:10CD20000E9420660895EF92FF920F931F939A013D
:10CD30007B0100E010E0B801A7010E9484661F910A
:10CD40000F91FF90EF900895CF92DF92EF92FF92B4
:10CD50000F931F93CF93DF93EC016A017B012115A1
:10CD6000310541F4E881F9810190F081E02D642FD3
:10CD700009951FC02A303105D1F477FF17C0E8812B
:10CD8000F9810190F081E02D6DE209958C01442735
:10CD90005527BA014C195D096E097F09CE012AE0B9
:10CDA0000E9420669801280F391F04C02AE00E94C3
:10CDB00020669C01C901DF91CF911F910F91FF90D7
:10CDC000EF90DF90CF900895EF92FF920F931F9313
:10CDD0007B019A010027F7FC0095102FB801A701ED
:10CDE0000E94A4661F910F91FF90EF9008950E94FA
:10CDF0000C660895CF93DF930E9427640E94252438
:10CE0000C7E9D4E60E949B252097E1F30E9497642E
:10CE1000F9CF0F931F93CF93DF93FC018B01411543
:10CE20005105F9F061157105E1F0848195812817AC
:10CE3000390718F0FB01108214C041505040EC013A
:10CE4000C21BD30B4C175D0708F4EA0160817181A6
:10CE5000620F731FC801AE010E941708C00FD11FD7
:10CE60001882DF91CF911F910F9108950F931F9317
:10CE7000CF93DF93EC018B016F5F7F4F88819981A6
:10CE80000E94B706009711F480E005C0998388835B
:10CE90001B830A8381E0DF91CF911F910F91089549
:10CEA000CF93DF93EC0188819981892B29F08A81C6
:10CEB0009B818617970760F4CE010E94366788230E
:10CEC00041F08C819D81892B19F4E881F9811082D0
:10CED00081E0DF91CF910895EF92FF920F931F931E
:10CEE000CF93DF93EC017B016C817D81E114F10430
:10CEF000C1F04115510599F08A01060F171FB801BD
:10CF00000E945067882369F0888199812C813D8136
:10CF1000820F931FB7010E9402081D830C8381E0DA
:10CF200001C080E0DF91CF911F910F91FF90EF90B2
:10CF30000895EF92FF920F931F93DF93CF93CDB796
:10CF4000DEB72B970FB6F894DEBF0FBECDBF7C01C6
:10CF5000CB01BA018E010F5F1F4FA8012AE030E01C
:10CF60000E949C08F80101900020E9F73197E01B2E
:10CF7000F10BC701B801AF010E946C672B960FB689
:10CF8000F894DEBF0FBECDBFCF91DF911F910F91FF
:10CF9000FF90EF900895EF92FF920F931F93DF930E
:10CFA000CF9300D000D000D0CDB7DEB77C01CB014D
:10CFB0008E010F5F1F4FB8014AE050E00E94C10888
:10CFC000F80101900020E9F73197E01BF10BC70150
:10CFD000B801AF010E946C6726960FB6F894DEBFC9
:10CFE0000FBECDBFCF91DF911F910F91FF90EF90BA
:10CFF0000895EF92FF920F931F93DF93CF9300D08A
:10D0000000D0CDB7DEB77C01862F90E08E010F5F98
:10D010001F4FB8014AE050E00E945E08F8010190FD
:10D020000020E9F73197E01BF10BC701B801AF0110
:10D030000E946C670F900F900F900F90CF91DF912F
:10D040001F910F91FF90EF9008956115710511F4F4
:10D0500080E00895DB010D900020E9F71197A61BF1
:10D06000B70BAD010E946C670895CF93DF93EC017D
:10D0700088819981009711F00E945F0619821882B9
:10D080001D821C821B821A82DF91CF910895EF923C
:10D09000FF920F931F93CF93DF93EC017B018A01E3
:10D0A000BA010E945067882321F4CE010E9435689E
:10D0B00007C01D830C8388819981B7010E940208F3
:10D0C000CE01DF91CF911F910F91FF90EF900895C6
:10D0D000CF93DF93EC01198218821B821A821D8282
:10D0E0001C821E826115710551F0DB010D9000203C
:10D0F000E9F71197A61BB70BAD010E944768DF91B6
:10D10000CF9108950F931F93182F092F6115710563
:10D1100059F0DB010D900020E9F71197A61BB70B22
:10D12000AD010E94476802C00E943568812F902F90
:10D130001F910F910895FC01808191810E945F06EB
:10D140000895629FD001739FF001829FE00DF11D51
:10D15000649FE00DF11D929FF00D839FF00D749F71
:10D16000F00D659FF00D9927729FB00DE11DF91F1D
:10D17000639FB00DE11DF91FBD01CF01112408957A
:10D18000991B79E004C0991F961708F0961B881F19
:10D190007A95C9F780950895AA1BBB1B51E107C07A
:10D1A000AA1FBB1FA617B70710F0A61BB70B881F37
:10D1B000991F5A95A9F780959095BC01CD010895C6
:10D1C00097FB092E07260AD077FD04D0E5DF06D0AD
:10D1D00000201AF4709561957F4F0895F6F79095A9
:10D1E00081959F4F0895A1E21A2EAA1BBB1BFD013A
:10D1F0000DC0AA1FBB1FEE1FFF1FA217B307E40736
:10D20000F50720F0A21BB30BE40BF50B661F771F8D
:10D21000881F991F1A9469F760957095809590956D
:10D220009B01AC01BD01CF01089597FB092E052696
:10D230000ED057FD04D0D7DF0AD0001C38F450952B
:10D240004095309521953F4F4F4F5F4F0895F6F72A
:10D2500090958095709561957F4F8F4F9F4F089562
:10D26000EE0FFF1F0590F491E02D09942F923F924D
:10D270004F925F926F927F928F929F92AF92BF92E6
:10D28000CF92DF92EF92FF920F931F93CF93DF9392
:10D29000CDB7DEB7CA1BDB0B0FB6F894DEBF0FBEEF
:10D2A000CDBF09942A88398848885F846E847D843C
:10D2B0008C849B84AA84B984C884DF80EE80FD803E
:10D2C0000C811B81AA81B981CE0FD11D0FB6F894B4
:0ED2D000DEBF0FBECDBFED010895F894FFCF75
:10D2DE00687474703A2F2F75692E6F70656E737047
:10D2EE0072696E6B6C65722E636F6D2F6A73007050
:10D2FE0069640073756E736574007363616C6500A9
:10D30E00747A0073756E72697365006E7077006360
:10D31E007077006A73700072736E007262740065CB
:10D32E006E007264007077002F00763D5B006E61B8
:10D33E006D650050726F6772616D20002E74787487
:10D34E0000737461727400656E6400005B002C00E3
:10D35E00302C227273222C00302C227264222C006C
:10D36E005D000D0A00616C6C00646179006C6F6386
:10D37E000077746B65790074747400743D5B007390
:10D38E0069640074000D0A0000323030006F706561
:10D39E006E646F6F7200426F73746F6E2C4D41002E
:10D3AE00687474703A2F2F75692E6F70656E737076
:10D3BE0072696E6B6C65722E636F6D2F6A730000EF
:10D3CE002000A60E00007000681173006310760036
:10D3DE00E1197900521A7C00CF1F7F00290C8200C0
:10D3EE0070198500551E8800D5138B00ED108E0028
:10D3FE00830A9100AC219400DB13970010159A005C
:10D40E009E1B9D001A1EA000890AA3003F117B10CF
:10D41E000E0000010A5000D200F9075C07206C07CD
:10D42E0008600701010E086307010113086707C0B2
:10D43E00FF1D086C07A8FF2908700701FF35087447
:10D44E000716FF41087807C0FF4D087C07A8FF5A52
:10D45E0008800701FF6708840701FF7408880750DA
:10D46E00FF81088C0700FF8C08900701018D08943E
:10D47E000700059D0897070101A9089B0700FEB547
:10D48E00089F070008C008A307003CCE08A7073C6A
:10D49E0078DD08AC070001EC08B1070101F908B509
:10D4AE000764FA0809B90701011609BC070001252E
:10D4BE0009C00700FF3309C5076EFF3C09CB07649F
:10D4CE00FF4A09CF0705FF5909D30700C86609D7D8
:10D4DE000700057309DB07CCFF8009DF0709FF8909
:10D4EE0009E40736FF9209E90777FF9B09EE07006B
:10D4FE0001A409F307AF09B309B709BB09BF09C3F3
:10D50E0009C7090069692D31004F70656E5370723D
:10D51E00696E6B6C65722D3030006382536335011A
:10D52E000100000000FC08DA656F0000000000003A
:10D53E00002F6C6F67732F002E6F4F1F1C1F1E1F47
:10D54E001E1F1F1E1F1E1FFFFFFFFFFFFF000007F6
:10D55E000305081000000006091F00151500001F26
:10D56E00111F11131E0014081501050515FFFFFFED
:10D57E00FFFFFF000000004045DA65000040001488
:10D58E0000540000000000EE4DDA6500000000843B
:10D59E005EDA65000000002F5FFE5EB75EC05ED5EE
:10D5AE005EE65E000000005165DA65E5641665F61C
:04D5BE00643F650061
:00000001FF
